:020000040800F2
:1000000000000220F9CB01082D7000082D700008B7
:100010002D7000082D7000082D70000800000000F1
:100020000000000000000000000000002D7000082B
:10003000836B0008000000007D030008290300080E
:100040002D7000082D7000082D7000082D7000081C
:100050002D7000082D7000082D7000082D7000080C
:100060002D7000082D7000082D7000084551010802
:1000700055510108655101082D7000082D700008C8
:100080002D7000082D7000082D7000082D700008DC
:100090002D7000082D7000082D7000082D700008CC
:1000A0002D7000082D7000082D7000082D700008BC
:1000B0002D700008755101082D7000082D70000882
:1000C0002D7000082D7000082D7000082D7000089C
:1000D0002D7000082D7000082D7000088551010852
:1000E0002D7000082D700008000000002D70000821
:1000F0002D7000082D700008955101082D70000822
:100100002D700008A55101082D7000082D70000801
:100110002D7000082D7000082D700008B5510108E1
:100120002D7000082D7000082D7000082D7000083B
:100130002D7000082D7000082D7000082D7000082B
:1001400000000000000000000000000000000000AF
:100150002D7000082D7000082D7000082D7000080B
:100160002D7000082D7000082D7000082D700008FB
:100170002D7000082D7000082D7000080000000090
:100180002D7000082D7000082D7000082D700008DB
:10019000C55101082D7000082D7000082D70000851
:1001A0002D7000082D7000082D7000080000000060
:1001B0002D7000082D7000082D7000082D700008AB
:1001C0002D7000082D7000080000000000000000E5
:1001D00000000000000000002D700008000000007A
:1001E000000000000000000000000000000000000F
:1001F00000000000000000002D7000082D700008B5
:100200002D7000082D700008000000002D700008FF
:100210002D7000082D7000082D7000082D7000084A
:100220002D700008000000002D7000080000000084
:100230002D7000082D700008000000002D700008CF
:100240002D7000082D7000082D7000082D7000081A
:100250002D7000082D7000082D7000082D7000080A
:100260002D7000082D7000082D7000082D700008FA
:100270002D7000082D7000082D700008000000008F
:100280002D7000082D7000082D7000082D700008DA
:10029000000000002D7000082D7000080000000014
:1002A000000000002D7000082D7000082D7000085F
:1002B0002D7000082D7000082D7000082D700008AA
:0C02C0002D7000082D7000082D70000843
:0402CC00000000002E
:1002D00072B64FF0E0201949C0F8081D18481749B8
:1002E000096801601748016841F0010101604FF0A1
:1002F000E020154941614FF0070101614FF0000115
:10030000C0F8181D4FF07F41C0F81C1D0F49C0F800
:10031000201D7047FFF7FEBFFFF7FEBFFFF7FEBFD0
:1003200001B5BDE80140704701B500F091F8BDE8A6
:1003300001407047FFF7FEBFFFF7FEBF0000000857
:10034000BC820024001000E09F8601000000FF40F6
:100350004FF000002A4A1060EFF3148020F00400F0
:1003600080F3148862B64FF080504FF0E021C1F85E
:10037000040DBFF34F8FBFF36F8FFEE72148224A72
:100380004FF00003016891B10360EFF3098C2CE991
:10039000F00F1EF0100F01D12CED108A1B4C4CF801
:1003A00004ED2568C1F808C00DB18D61236072B6F7
:1003B0001168B1B1016062B64F68144C8D6907F1E4
:1003C00001074F602560D1F808C05CF804EB1EF00F
:1003D000100F01D1BCEC108ABCE8F00F8CF3098837
:1003E000704772B61168016009B962B6F9E74FF05B
:1003F00000674FF0E028C8F8047D62B6DCE770477C
:10040000C8820024D8820024D48200248882002458
:10041000026922F00702A2F144026FF002031360A6
:100420004FF0000353609360D36013615361936195
:10043000D361136253629362D362136353634FF0C9
:10044000FF339363D1634FF080731364826070470E
:100450002249086800F101000860214B1A683AB18E
:10046000A2F101021A601AB91E4B4FF00100186088
:100470001D490868026822B11C4B4FF001021A6046
:1004800008E000F104001A4B1A68904201D1194BA0
:1004900018680860134B1A6812B914490868D0B17B
:1004A0002DE901401149086808B11BF085FF0D4B8B
:1004B0001A6872B113F0E8FE0F48016849B90F4895
:1004C00001680F4A13680F484FF08052994200D0DC
:1004D0000260BDE80140BFF34F8F70478C8200245B
:1004E00088820024A8820024B0820024AC820024E8
:1004F000A08200249C820024C8820024D882002488
:08050000D482002404ED00E0A8
:100508002DE9F84F2DED068B84B0B5EE401BF1EECA
:1005180010FA00F09180B4EE411BF1EE10FA80F170
:100528008B80B0EE408B50EC101B420042EAD17138
:1005380011F5001F9FED429B77D2B0EEC89BB0EE3D
:10054800C1ABB4EE4A9BF1EE10FA02D5B0EE489B6F
:100558006BE0B4EE4A9BF1EE10FA05D100F00040D2
:10056800002140EC191B60E002A8B0EE4A0B1CF019
:1005780063FBB4EE4A9BF1EE10FA4FDB59EC1A0B11
:100588000190029F09F0004A4AF0E04040F07F6B7A
:10059800C9F30A556FF31E5940F2FF78B0EE490BC4
:1005A80003A81CF049FB0398C01B691EB0EE4A0B58
:1005B80012D34545B0EE4A0B0ED0431940F2FE72F5
:1005C800002693425A4605DC012B5246A4BF49EA4D
:1005D8000352019E42EC106BB4EE490BF1EE10FA97
:1005E80015DDB0EE4A0B95B14545B0EE4A0B0ED07D
:1005F800014440F2FE7000228142584605DC012980
:100608005046A4BF49EA0150019A40EC102B39EE3C
:10061800409BB4EE4A9BF1EE10FABFDAB5EE408B80
:10062800F1EE10FA48BFB1EE499BB0EE490B04B0A9
:10063800BDEC068BBDE8F88F9FED019BF5E700BF89
:08064800000000000000F87F33
:1006500050EC10CBC0F30A52531E40F2FE718B4295
:1006600051D240F2FE318A4208D8BFEE000B9FED16
:100670002A1BB0F1FF3F31FE000B704740F23241C0
:100680008A4288BF7047F0B5A2F2FF33B3F1200170
:100690004FF48017C3F1200407FA04F540F2000676
:1006A000CFF6F07606FA04F25CBF27FA01F546FAB7
:1006B00001F202EA0C0E27FA03F24EBF1E4100229D
:1006C0004FF0FF36064015EB0E0572412CFA04F48C
:1006D00000FA03F73C43002958BF0CFA01F46FF30A
:1006E0001F540CFA03F148BF0C43B4FA84F14909D2
:1006F0000028A8BF41F0010100291CBF3246754601
:1007000042EC105BF0BD002A04BF00F000409446AC
:1007100040EC10CB704700BF00000000000000005C
:1007200000000000000024400000000000005940CC
:10073000000000000088C3400000000084D79741FB
:100740000080E03779C34143176E05B5B5B89346CD
:10075000F5F93FE9034F384D321D30F94877825A99
:080760003CBF737FDD4F1575EE
:1007680001000000000000000A0000000000000076
:100778006400000000000000E80300000000000022
:100788001027000000000000A08601000000000003
:1007980040420F0000000000809698000000000012
:1007A80000E1F5050000000000CA9A3B00000000C7
:1007B80000E40B540200000000E87648170000002F
:1007C8000010A5D4E800000000A0724E180900002F
:1007D80000407A10F35A00000080C6A47E8D030002
:1007E8000000C16FF286230000008A5D784563012E
:1007F800000064A7B3B6E00D0000E8890423C78AA7
:100808002DE9F84F2DED0A8B8EB006928946804669
:100818000020C8F800000DF11D0003909FEDC6AB45
:10082800B2EE048BB7EE00BB9FEDC5CB19F8011BE8
:10083800252906D0002900F0DA8540461CF034FA54
:10084800F4E70026494619F8012BA2F12003102BE2
:100858000DD88020DFE803F0091B1B191B1B1B1593
:100868001B1B30181B101B1B120040200DE05E2ABA
:100878000DD14FF4805008E0102006E04FF40070CE
:1008880003E04FF4004000E020200643DAE701F1DE
:100898000109A2F1300009284FF000001BD819F80F
:1008A800011B00EB800002EB40003038A1F1300260
:1008B8000A2A0A46F3D30EE0069850F8042B06904D
:1008C800002A104648BF5042102303EAD26216435A
:1008D8004A7801F102092E2A0DD1494611F8012B57
:1008E8002A2A0BD1069999F8012051F804AB0691F0
:1008F80009F1020916E04FF0000A1CE0A2F13003EA
:10090800092B4FF0000A13D811F8013B0AEB8A09AA
:1009180002EB4902A2F1300AA3F130020A2A1A4670
:10092800F2D38946BAF1000F58BF46F4807602E048
:1009380046F4807689466B2A0ADC4C2A03D0682A5A
:1009480018D06A2A28D119F8012B46F0020623E0AC
:100958006C2A05D07A2A14BF742A19F8012B1BE0D7
:10096800494611F8012B6C2A10D199F8012009F198
:100978000209EAE7494611F8012B682A09D199F8D2
:10098800012009F1020946F0080605E046F00106D3
:1009980001E046F00406894620EAE077462A1FDD92
:1009A800A2F1630015282FD8DFE810F060001700C7
:1009B80045002300A40116001700160016001600B3
:1009C8001600700084004E00160016007F00160006
:1009D800480016001600360028E746F4804631E045
:1009E800442A09DD452A24D0462A7FF41FAF46F45D
:1009F800005646F4006B7FE1252A40F065824046A8
:100A080025211CF051F911E7472A00F07181582A75
:100A18007FF40CAF46F40056F0054FEA066048BF75
:100A280026F4007643F25801782A08BF43F2780189
:100A380047E046F4005646F4806B5DE1F00548BF98
:100A480026F4007600213EE03006232101EAE0701A
:100A5800CDE9047046F48076069A002152F8040B1A
:100A680006924FF0080A0DF11E04DEE00698A7F181
:100A7800010A10F8044B069040463146524614F0DD
:100A88005DF8404621461CF00FF9AEE1069951F891
:100A9800040B06913107D8F8001000F11982B2074B
:100AA80052BF0160002206C0C0E6069850F8044B09
:100AB800069079E1F0054FEA066048BF26F4007613
:100AC800302101EAE07170044FEA8670069DCDE995
:100AD800047104D4002808D42B1D00210BE0002841
:100AE80015D455F8040BC11717E0E81D20F00705C9
:100AF80005F1080369680DF11E0428687507069357
:100B080015D416F008051CBFC0B2002132E0E81D5C
:100B180020F00705696855F8080B0DF11E047307E6
:100B280012D4330744BF40F3C01140B20FE080B283
:100B380000211FE000BF00BFA0C8EB85F3CCE17F18
:100B4800000000000000594040F3C03100B2002905
:100B5800069507DBB3060BD47306059D48BF202511
:100B6800059507E00023404263EB01012D2300E0D7
:100B78002B230593F30548BF26F40076F30558BFE9
:100B88004FF0010A00276E2A21DD6F3A092A00F288
:100B98006D80DFE802F0054A6B6B6B6B226B6B4A6A
:100BA80050EA010262D0C20842EA417206251346A1
:100BB80065F3DF00E055013752EAD1004FEAD10171
:100BC8004FEAD20040EA41721846F0D14EE0582A66
:100BD8002BD0642A18BF692A48D150EA010245D0AF
:100BE8000C46054630040AD507F00300032806D151
:100BF8000DF11E0B2C200BF80700013701E00DF159
:100C08001E0B28460A22002303F012FC00EB800288
:100C1800A5EB420242F030020BF807200137D5F16C
:100C280009020022A241DBD320E0002750EA01029A
:100C38001CD0B2044DF6A632C0F601025CBF4DF6D8
:100C4800B632C0F60102030943EA017500F00F004D
:100C58002B46105CE055013755EA11104FEA111187
:100C68004FEA151040EA01751846EFD105994FF083
:100C7800FF30FF2988BF0138AAEB070222EAE27A8F
:100C880007EB0A03049AD41A002918BF0444B005D4
:100C980006D440463146224613F050FF05990024F9
:100CA800FF29039D05D9090A40461BF0FDFF059958
:100CB80000E011B140461BF0F7FF4046314622469E
:100CC80013F03CFF4046302152461CF03DF8012FFE
:100CD80005DBE95D40461BF0E7FF013FF9D8F00668
:100CE8007FF5A4AD4046202122461CF02DF89DE555
:100CF80046F4005646F4406B5FEACB5058BF4FF0BD
:100D0800060A0BF4406006990731A0F5406021F00F
:100D18000701B0FA80F0BAF1000F08BF4FEA501A85
:100D2800D1E9005646EC195B01F108000690B0EED7
:100D3800490B13F0C4FE80B1B5EE409BF1EE10FAFA
:100D48001DD55FEA8B404DF6BA04C0F601045CBFBE
:100D58004DF6BF04C0F6010424E0B0EE490B1BF0C9
:100D68005DFF00284AD05FEA8B404DF6C634C0F6D6
:100D780001045CBF4DF6CA34C0F6010412E01BF44E
:100D880000504DF6C402C0F601024DF6C901C0F686
:100D98000101104612BF541C08464C1C5FEA8B61C7
:100DA80048BF04462BF48076002C04BF4DF27F34F4
:100DB800C0F60104F005204602D41CF07DF802E0DC
:100DC80051461CF08FF8054626F40076A7EB000A7A
:100DD80040463146524613F0B1FE35B114F8011BB6
:100DE80040461BF061FF013DF8D1F0067FF51EADCE
:100DF8004046202152461BF0A7FF17E5B0EE490BED
:100E080013F06AFE002804BF0646054646EC195B47
:100E1800B0EE490B1BF00AFF044686F0004040EC98
:100E2800105B002C09FE009BB0EE490B0DA81BF0CF
:100E380001FF0D9800EB400046F26761C6F266615B
:100E480050FB01F0002C18BF4BF0600B811001EB38
:100E5800D0700D90B5EE409BF1EE10FA16D001302F
:100E68001BF004FFB4EE490BF1EE10FA0D9806D50D
:100E7800411C0D910230F3E70D9801380D901BF0DD
:100E8800F5FEB4EE490BF1EE10FAF5DC0D990BF412
:100E98004064B4F5806F07D0B4F5406F0AD18A4535
:100EA800C8BF11F1050F05DCB1F59A7F13D189EEA2
:100EB8000A9B15E05FEA4B5040F1E7800E2940F3AA
:100EC800C1804FF0000AE0E0002A7FF4AFACA1E255
:100ED8000170FFF7ABBC48421BF0C8FE20EE099B2F
:100EE800B5EE409BF1EE10FA23D0B0EE490B13F0AB
:100EF800E6FD00287FF420AF0D98B4EE489BF1EE94
:100F080010FA08DB89EE089B0130B4EE489BF1EE3D
:100F180010FAF7DA0D90B4EE4B9BF1EE10FA08D503
:100F280029EE089B0138B4EE4B9BF1EE10FAF7D48A
:100F38000D90B4F5406F544608BF013CBAF1000F5C
:100F480018BFA246CAF100001BF090FE4FF0FF3018
:100F580013F0D3FD30EE090BB4EE480BF1EE10FAA6
:100F6800A1BF0D9880EE080B01300D9050EC106B6E
:100F78000290BAF1000F35D005940BF40860B0F573
:100F8800006F31D1BAF1100FA8BF4FF0100A0298C4
:100F980040EC196B50461BF069FE20EE090B51EC32
:100FA800100B03F0F7F90446084300F007820D46DA
:100FB8004CF6CD42CCF6CC42A4FB0201531E04FBF6
:100FC800031105FB0211C20742EA5102C90741EAAF
:100FD8005000D0F1993049F69910C1F69910904116
:100FE80080F0EE81CDF814A0059A0BF08000104334
:100FF800A7EB02000D9D0CBF471F871F01245FEA66
:10100800CB4002D404950299BDE045F25650C5F292
:10101800555055FB00F000EBD07000EB4000281A4B
:1010280002300299DFE800F003A1AB03A10041EC14
:10103800106B20EE080B51EC106B013D0D95013F34
:1010480002249CE0C84350444FF0100A1028B8BF4F
:1010580082465FEA0B6218D4B8B150461BF006FE10
:10106800B6EE001B00EE091BB0EE410BFFF7ECFAE1
:10107800B0EE481BFFF744FAB5EE400BF1EE10FA5C
:1010880002D1BAF1010AE8D10D99CDF814A0CAF13C
:10109800000010398142C8BF08461BF0E7FD4FF039
:1010A800FF3013F02AFD30EE099B0D9801301BF03C
:1010B800DDFDB4EE490BF1EE10FA0D9898BF013042
:1010C800002814D411281AD3A0F110010D91C0F1F1
:1010D80010001BF0CBFD20EE090B51EC100B03F0B8
:1010E80059F905460E460020CDE9010019E050ECFB
:1010F800191BCDE9011000250D95002611E051ECD2
:10110800190B03F047F905460E4603F063F941EC65
:10111800100B39EE400B50EC101BCDE901100020EC
:101128000D902BF4806A40F26870C0F60000083019
:10113800002400F10801013405C8281A76EB0200E2
:101148000846F6D2059AB81A0BF0800111434FF001
:10115800FF321CBF1146013A1BF0600F08BF0A4658
:101168000D99511A0844071B2AE041EC106B20EE38
:101178000C0B51EC106B023D0D95023F032422EA43
:10118800E272CDE904522BF4006A41EC196B304647
:1011980003F000F905460E4603F01CF941EC100B6C
:1011A80039EE400B50EC101BCDE901101BF0600F1D
:1011B80018BF013F04981BF055FD6328C8BF013FC5
:1011C80027EAE77B1AF4047F0DD1012F0BDB40F2ED
:1011D8006877C0F60007404620211BF065FDBBF18B
:1011E800010BF8D103E040F26877C0F600075FEA28
:1011F8008A604FEA4A6003D4002808D5202103E01A
:101208002D21002858BF2B2140461BF04DFD5FEAD9
:10121800CA6009D4BBF1000F06D0404630211BF04C
:1012280043FDBBF1010BF8D1013C07EBC40006C834
:10123800681A76EB0200302006D36D1A9641013009
:101248006B1A76EB0203F8D2C1B240461BF02CFDB4
:10125800002CE9D15FEA0A540BD50D98012808DB68
:1012680001380D90404630211BF01EFD0D980028D6
:10127800F6DC0AF08000059D284343D040462E2125
:101288001BF012FD1020102DB8BF2846002C0D9918
:1012980020EAE077384648BF401A1BF0E7FC012DEA
:1012A80026DBDDE9011040EC111B20EE010B51ECAF
:1012B800100B03F06FF804460D463E46013E40F21F
:1012C8006870C0F6000000EBC60006C8601A75EB2F
:1012D8000200302006D3641A95410130631A75EB79
:1012E8000203F8D2C1B240461BF0DEFC002EE5D165
:1012F8000599C81B06D07C1A404630211BF0D4FC47
:101308000134F9D35FEA4A504BD545215FEA8A4058
:1013180058BF652140461BF0C7FC0D980028404681
:1013280004DB2B211BF0C0FC0D9805E02D211BF0E0
:10133800BBFC0D9840420D90642815DB48F21F5401
:10134800C5F2EB14A0FB0401302000EB511140461C
:101358001BF0AAFC0D9850FB04F14A1102EBD17165
:10136800642201FB12000D9046F26764C6F26664BF
:1013780050FB04F0811001EBD07000F130014046C1
:101388001BF092FC0D9850FB04F18A1002EBD1710E
:1013980001EB8101A0EB410000F1300140461BF058
:1013A80083FCBBF1000F3FF441AA404620211BF00B
:1013B8007BFCBBF1010BF8D1FFF738BA059013E6B7
:1013C800CDF814A0204629460A22002303F030F85D
:1013D80004460D460A22002303F02AF8059801382E
:1013E80005903FF401AE52EA0300EBD0FCE5D8F8D3
:1013F8000C0028B1D8E9001291423CBF00224254A7
:1014080040461BF093FCD8F800000EB0BDEC0A8BE8
:10141800BDE8F88F40461BF089FC4FF0FF30F4E739
:1014280085B0049000208DF80F0004988069E8B911
:101438000498806A0290032817D80299DFE801F01F
:10144800020B0214049890F82F00C00710B1012075
:101458008DF80F0009E00498C06AB0F1C07F02D18E
:1014680001208DF80F0000E0FFE73BE00498806959
:10147800B0F5005F20D10498806A019003281AD83B
:101488000199DFE801F00206020F01208DF80F0034
:1014980011E0049890F82F00C00710B101208DF8D2
:1014A8000F0008E00498C06AB0F1C07F02D10120A3
:1014B8008DF80F00FFE715E00498806A0090032874
:1014C80003D30098032804D00CE001208DF80F0006
:1014D80008E0049890F82F00C00710B101208DF89B
:0C14E8000F00FFE79DF80F0005B07047F3
:1014F4008AB044F21040C5F60200006800F03800DB
:1015040001460191182800F25A810199DFE811F08F
:101514001900570157015701570157015701570146
:10152400350057015701570157015701570157011A
:101534003B00570157015701570157015701570104
:10154400410044F20040C5F602000068C0F34010B8
:1015540068B144F20040C5F602000068C0F3C1015E
:1015640049F20000C0F2D030C840029004E049F2D1
:101574000000C0F2D030029026E140F60010C0F224
:101584003D00029020E147F64000C0F27D10029039
:101594001AE144F22840C5F60200016801F0030193
:1015A40008910068C0F30510079044F22C40C5F67A
:1015B4000200006800F001000690069844F23441ED
:1015C400C5F60201096889B2C908484300EE100A49
:1015D400B8EE400A8DED040A0798002800F0EC806C
:1015E4000898009038B10098012863D00098022828
:1015F40000F08480A6E044F20040C5F602000068D2
:10160400C0F3401090B344F20040C5F602000068F5
:10161400C0F3C10149F20000C0F2D030C8400590C7
:101624009DED050AB8EE400A9DED071AB8EE411A81
:1016340080EE010A44F23040C5F6020000686FF300
:101644005F2001EE100AB8EE411A9DED042A9FEDC9
:10165400613A82EE032A31EE021AB7EE002A31EE25
:10166400021A20EE010A8DED030A22E09DED070A1D
:10167400B8EE401A9FED590A80EE010A44F2304058
:10168400C5F6020000686FF35F2001EE100AB8EEA1
:10169400411A9DED042A9FED4F3A82EE032A31EE62
:1016A400021AB7EE002A31EE021A20EE010A8DED7D
:1016B400030A6AE09DED070AB8EE401A9FED460A58
:1016C40080EE010A44F23040C5F6020000686FF370
:1016D4005F2001EE100AB8EE411A9DED042A9FED39
:1016E4003D3A82EE032A31EE021AB7EE002A31EEB9
:1016F400021A20EE010A8DED030A46E09DED070A69
:10170400B8EE401A9FED320A80EE010A44F23040EE
:10171400C5F6020000686FF35F2001EE100AB8EE10
:10172400411A9DED042A9FED2B3A82EE032A31EEF5
:10173400021AB7EE002A31EE021A20EE010A8DEDEC
:10174400030A22E09DED070AB8EE401A9FED220A33
:1017540080EE010A44F23040C5F6020000686FF3DF
:101764005F2001EE100AB8EE411A9DED042A9FEDA8
:10177400193A82EE032A31EE021AB7EE002A31EE4C
:10178400021A20EE010A8DED030A44F23040C5F638
:101794000200006881B2012000EB512009909DED08
:1017A400030A9DED091AB8EE411A80EE010ABCEE57
:1017B400C00A8DED020A01E00020029004E040F628
:1017C4000010C0F23D00029002980AB0704700BFBA
:1017D40020BCBE4B000000460024744A0024744C14
:1017E40080B59AB0189000208DF857008DF85600F7
:1017F4001898C0780007002840D51898406E1490B7
:1018040060B11498B0F5801F11D01498B0F5001F82
:1018140015D01498B0F5401F19D019E044F22C41AA
:10182400C5F60201086840F40030086013E0189817
:101834000830022109F0B7FB8DF857000BE0189827
:101844002830022109F006FD8DF8570003E002E07C
:1018540001208DF857009DF8570058B944F25041C3
:10186400C5F60201086820F44010189A526E10431D
:10187400086003E09DF857008DF8560018984078EA
:10188400C00700283BD01898806D1390042820D8F6
:101894001399DFE801F0030C141C1D0044F22C41E1
:1018A400C5F60201086840F40030086014E0189896
:1018B4000830002109F077FB8DF857000CE01898E8
:1018C4002830002109F0C6FC8DF8570004E003E03D
:1018D40002E001208DF857009DF8570058B944F2F2
:1018E4005041C5F60201086820F00700189A926D6D
:1018F4001043086003E09DF857008DF856001898CF
:101904004078400700284CD51898D0F8A4001290CD
:10191400A0B11298B0F5001F19D01298B0F5800F3D
:101924001DD01298B0F5C00F21D01298B0F5000F59
:101934001ED01298B0F5200F1BD01BE044F22C41AE
:10194400C5F60201086840F40030086015E01898F4
:101954000830002109F027FB8DF857000DE0189896
:101964002830002109F076FC8DF8570005E004E0EA
:1019740003E002E001208DF857009DF8570060B99C
:1019840044F25841C5F60201086820F46000189A30
:10199400D2F8A4201043086003E09DF857008DF8A6
:1019A400560018984078000700284CD51898D0F8AD
:1019B400A8001190A0B11198B0F1807F19D01198AE
:1019C400B0F1007F1DD01198B0F1407F21D0119863
:1019D400B0F1806F1ED01198B0F1A06F1BD01BE046
:1019E40044F22C41C5F60201086840F40030086056
:1019F40015E018980830002109F0D5FA8DF8570041
:101A04000DE018982830002109F024FC8DF85700C7
:101A140005E004E003E002E001208DF857009DF8A2
:101A2400570060B944F25841C5F60201086820F035
:101A3400E060189AD2F8A8201043086003E09DF8EB
:101A440057008DF856001898C0788007002836D5BE
:101A54001898C06C1090D8B11098102806D010981F
:101A640020280CD01098302811D012E044F22C41D8
:101A7400C5F60201086840F4003008600CE01898CC
:101A84000830022109F08FFA8DF8570004E003E0D2
:101A940002E001208DF857009DF8570058B944F230
:101AA4004C41C5F60201086820F03000189AD26C47
:101AB4001043086003E09DF857008DF8560018980D
:101AC4004078C006002845D51898C06D0F9080B1A5
:101AD4000F98B0F5805F15D00F98B0F5005F19D05E
:101AE4000F98B0F5405F1DD00F98B0F5804F1AD015
:101AF4001AE044F22C41C5F60201086840F40030B3
:101B0400086014E018980830002109F04CFA8DF8A8
:101B140057000CE018982830002109F09BFB8DF841
:101B2400570004E003E002E001208DF857009DF81F
:101B3400570058B944F25041C5F60201086820F430
:101B4400E040189AD26D1043086003E09DF85700F6
:101B54008DF85600189840788006002842D51898C9
:101B6400006E0E90A0B10E98B0F5803F11D00E9883
:101B7400B0F5003F15D00E98B0F5403F19D00E983F
:101B8400B0F5802F16D00E98B0F5A02F13D013E027
:101B940015E018980830012109F005FA8DF857006E
:101BA4000DE018982830012109F054FB8DF85700F6
:101BB40005E004E003E002E001208DF857009DF801
:101BC400570058B944F25041C5F60201086820F4A0
:101BD400E020189A126E1043086003E09DF8570045
:101BE4008DF85600189840784006002844D5189877
:101BF400D0F8AC000D90A0B10D98B0F1805F11D079
:101C04000D98B0F1005F15D00D98B0F1405F19D078
:101C14000D98B0F1804F16D00D98B0F1A04F13D0AD
:101C240013E015E018980830012109F0BCF98DF88B
:101C340057000DE018982830012109F00BFB8DF8AE
:101C4400570005E004E003E002E001208DF85700AE
:101C54009DF8570060B944F25841C5F6020108687E
:101C640020F0E040189AD2F8AC201043086003E05A
:101C74009DF857008DF85600189840780006002803
:101C840034D51898C06E0C90C8B10C98B0F1805F30
:101C940004D00C98B0F1005F09D011E044F22C415B
:101CA400C5F60201086840F4003008600BE018989B
:101CB4000830012109F077F98DF8570003E002E0BC
:101CC40001208DF857009DF8570058B944F250414F
:101CD400C5F60201086820F04050189AD26E1043ED
:101CE400086003E09DF857008DF856001898C078F6
:101CF400C00790B31898806C0B90032817D80B99E1
:101D0400DFE801F014020B1344F22C41C5F6020182
:101D1400086840F4003008600CE01898083002218C
:101D240009F041F98DF8570004E003E002E00120D6
:101D34008DF857009DF8570058B944F24C41C5F648
:101D44000201086820F00300189A926C104308609E
:101D540003E09DF857008DF85600189880784006E7
:101D6400002840F1E6821898D0F8B000B0F5807FE2
:101D740000F03A821898D0F8B000B0F5007F00F077
:101D840033821898D0F8B000B0F50C5F00F02C82C4
:101D94001898D0F8B000B0F54C5F00F02582189880
:101DA400D0F8B000B0F5864F00F01E821898D0F835
:101DB400B000B0F5A64F00F017821898D0F8B00024
:101DC400B0F5C64F00F010821898D0F8B000B0F506
:101DD400E64F00F009821898D0F8B000B0F5034F30
:101DE40000F002821898D0F8B000B0F5134F00F05C
:101DF400FB811898D0F8B000B0F5234F00F0F481BF
:101E04001898D0F8B000B0F5334F00F0ED81189871
:101E1400D0F8B000B0F5434F00F0E6811898D0F840
:101E2400B000B0F5534F00F0DF811898D0F8B0003F
:101E3400B0F5634F00F0D8811898D0F8B000B0F531
:101E4400734F00F0D1811898D0F8B00040F20031FF
:101E5400C0F20101884200F0C7811898D0F8B000A0
:101E640041F20031C0F20101884200F0BD811898AE
:101E7400D0F8B00042F20031C0F20101884200F013
:101E8400B3811898D0F8B00043F20031C0F20101D8
:101E9400884200F0A9811898D0F8B00044F20031CB
:101EA400C0F20101884200F09F811898D0F8B00078
:101EB40045F20031C0F20101884200F09581189882
:101EC400D0F8B00046F20031C0F20101884200F0BF
:101ED4008B811898D0F8B00047F20031C0F20101AC
:101EE400884200F081811898D0F8B00048F200319F
:101EF400C0F20101884200F077811898D0F8B00050
:101F040049F20031C0F20101884200F06D81189855
:101F1400D0F8B0004AF20031C0F20101884200F06A
:101F240063811898D0F8B0004BF20031C0F201017F
:101F3400884200F059811898D0F8B0004CF2003172
:101F4400C0F20101884200F04F811898D0F8B00027
:101F54004DF20031C0F20101884200F04581189829
:101F6400D0F8B0004EF20031C0F20101884200F016
:101F74003B811898D0F8B0004FF20031C0F2010153
:101F8400884200F031811898D0F8B00040F2003156
:101F9400C0F20201884200F027811898D0F8B000FE
:101FA40041F20031C0F20201884200F01D8118980C
:101FB400D0F8B00042F20031C0F20201884200F0D1
:101FC40013811898D0F8B00043F20031C0F2020136
:101FD400884200F009811898D0F8B00044F200312A
:101FE400C0F20201884200F0FF801898D0F8B000D7
:101FF40045F20031C0F20201884200F0F5801898E1
:10200400D0F8B00046F20031C0F20201884200F07C
:10201400EB801898D0F8B00047F20031C0F202010A
:10202400884200F0E1801898D0F8B00048F20031FE
:10203400C0F20201884200F0D7801898D0F8B000AE
:1020440049F20031C0F20201884200F0CD801898B4
:10205400D0F8B0004AF20031C0F20201884200F028
:10206400C3801898D0F8B0004BF20031C0F20201DE
:10207400884200F0B9801898D0F8B0004CF20031D2
:10208400C0F20201884200F0AF801898D0F8B00086
:102094004DF20031C0F20201884200F0A580189888
:1020A400D0F8B0004EF20031C0F20201884200F0D4
:1020B4009B801898D0F8B0004FF20031C0F20201B2
:1020C400884200F091801898D0F8B00040F20031B6
:1020D400C0F20301884200F087801898D0F8B0005D
:1020E40041F20031C0F2030188427DD01898D0F843
:1020F400B00042F20031C0F20301884274D0189853
:10210400D0F8B00043F20031C0F2030188426BD032
:102114001898D0F8B00044F20031C0F203018842AC
:1021240062D01898D0F8B00045F20031C0F2030133
:10213400884259D01898D0F8B00046F20031C0F265
:102144000301884250D01898D0F8B00047F200310B
:10215400C0F20301884247D01898D0F8B00048F282
:102164000031C0F2030188423ED01898D0F8B00084
:1021740049F20031C0F20301884235D01898D0F8F2
:10218400B0004AF20031C0F2030188422CD0189802
:10219400D0F8B0004BF20031C0F20301884223D0E2
:1021A4001898D0F8B0004CF20031C0F20301884214
:1021B4001AD01898D0F8B0004DF20031C0F20301E3
:1021C400884211D01898D0F8B0004EF20031C0F215
:1021D4000301884208D01898D0F8B0004FF20031BB
:1021E400C0F20301884200D107E04DF22A60C0F634
:1021F400010040F27D3104F08CFD44F60001C5F687
:102204000201086840F48070086013F057F81690D3
:1022140044F60000C5F602000068C00500280AD490
:1022240013F04CF81699401A652803D303208DF84F
:10223400570000E0ECE79DF85700002875D144F200
:102244007040C5F60200006800F440701899D1F897
:10225400B01001F44071884211D044F27041C5F6C7
:102264000201086820F440701790086840F4803038
:102274000860086820F4803008601798086018988F
:10228400D0F8B000B0F5807F17D113F017F816908E
:1022940044F27040C5F602000068C0F3400060B923
:1022A40013F00CF81699401A41F28931884203D38D
:1022B40003208DF8570000E0EAE79DF8570078BB4B
:1022C4001898D0F8B00000F44070B0F5407F12D1F7
:1022D40044F21041C5F60201086820F47C50189AB3
:1022E400D2F8B0204FF6F043C0F6FF731A4040EA2C
:1022F4001210086007E044F21041C5F602010868B4
:1023040020F47C5008601898D0F8B0206FF31F3286
:1023140044F27041C5F6020108681043086003E006
:102324009DF857008DF8560003E09DF857008DF88E
:10233400560018980068C007002800F047801898D5
:10234400806F0A9028282BD80A99DFE801F0152914
:1023540029292929292916292929292929291E2907
:1023640029292929292926292929292929292729DE
:10237400292929292929280015E01898083001213C
:1023840008F011FE8DF857000DE01898283001214F
:1023940008F060FF8DF8570005E004E003E002E078
:1023A40001208DF857009DF8570058B944F2544164
:1023B400C5F60201086820F03800189A926F10439D
:1023C400086003E09DF857008DF8560018980078CF
:1023D4008007002834D51898406F0990052819D82B
:1023E4000999DFE801F003040C14151615E0189898
:1023F4000830012108F0D7FD8DF857000DE018983A
:102404002830012108F026FF8DF8570005E004E08C
:1024140003E002E001208DF857009DF8570058B9F9
:1024240044F25441C5F60201086820F00700189AE6
:10243400526F1043086003E09DF857008DF8560072
:10244400189800784007002836D51898D0F89000DE
:102454000890052819D80899DFE801F003040C1442
:10246400151615E018980830012108F09CFD8DF828
:1024740057000DE018982830012108F0EBFE8DF884
:10248400570005E004E003E002E001208DF8570066
:102494009DF8570060B944F25841C5F60201086836
:1024A40020F00700189AD2F890201043086003E047
:1024B4009DF857008DF8560018980078800600287B
:1024C40044D51898D0F88C000790A0B10798B0F1C3
:1024D400805F11D00798B0F1005F15D00798B0F174
:1024E400405F19D00798B0F1804F16D00798B0F12B
:1024F400A04F13D013E015E018980830002108F01D
:1025040052FD8DF857000DE018982830022108F08C
:10251400A1FE8DF8570005E004E003E002E001208D
:102524008DF857009DF8570060B944F25441C5F640
:102534000201086820F0E040189AD2F88C20104379
:10254400086003E09DF857008DF85600189800784D
:102554004006002844D51898D0F898000690A0B1F9
:102564000698B0F5806F11D00698B0F5006F15D0BD
:102574000698B0F5406F19D00698B0F5805F16D074
:102584000698B0F5A05F13D013E015E01898083052
:10259400002108F008FD8DF857000DE01898283048
:1025A400022108F057FE8DF8570005E004E003E02F
:1025B40002E001208DF857009DF8570060B944F2FD
:1025C4005841C5F60201086820F4E050189AD2F880
:1025D40098201043086003E09DF857008DF85600DA
:1025E400189800780006002844D51898D0F89C0064
:1025F4000590A0B10598B0F5005F11D00598B0F52D
:10260400804F15D00598B0F5C04F19D00598B0F596
:10261400004F16D00598B0F5204F13D013E015E005
:1026240018980830002108F0BEFC8DF857000DE022
:1026340018982830022108F00DFE8DF8570005E0A7
:1026440004E003E002E001208DF857009DF85700F4
:1026540060B944F25841C5F60201086820F46040AC
:10266400189AD2F89C201043086003E09DF85700A4
:102674008DF85600189800780007002839D5189866
:10268400D0F88000B0F5805F0FD01898D0F88000A3
:10269400B0F5005F09D01898D0F8800028B11898D8
:1026A400D0F88000B0F5405F00D107E04DF22A6019
:1026B400C0F6010040F2FC4104F02BFB1898D0F85E
:1026C4008000B0F5805F08D118982830022108F006
:1026D400C1FD10B101208DF8560044F25441C5F6F5
:1026E4000201086820F44050189AD2F88020104360
:1026F400086018980078C006002839D51898D0F8D2
:102704009400B0F5807F0FD01898D0F89400B0F5FD
:10271400007F09D01898D0F8940028B11898D0F800
:102724009400B0F5407F00D107E04DF22A60C0F676
:1027340001004FF4A46104F0ECFA1898D0F8940066
:10274400B0F5807F08D118982830022108F082FD66
:1027540010B101208DF8560044F25841C5F602012B
:10276400086820F44070189AD2F894201043086046
:10277400189880780007002835D51898D0F8A0005C
:10278400049040B10498B0F5803F0CD00498B0F5A3
:10279400003F10D010E018980830002108F003FC26
:1027A4008DF857000BE018982830022108F052FDEC
:1027B4008DF8570003E002E001208DF857009DF8E2
:1027C400570060B944F25841C5F60201086820F484
:1027D4004030189AD2F8A0201043086003E09DF816
:1027E40057008DF85600189880784007002838D58F
:1027F4001898D0F884000390B0F5801F08D003988F
:10280400B0F5001F0DD00398B0F5401F11D011E0B2
:1028140044F22C41C5F60201086840F40030086017
:102824000BE018982830012108F014FD8DF85700AA
:1028340003E002E001208DF857009DF8570060B9CD
:1028440044F25441C5F60201086820F44010189A75
:10285400D2F884201043086003E09DF857008DF8F7
:10286400560018988078C007002840D01898006D4A
:1028740020B11898006DB0F5803F00D107E04DF20B
:102884002A60C0F6010040F2865104F042FA18981A
:10289400006D029020B10298B0F5803F09D010E09D
:1028A40044F22C41C5F60201086840F40030086087
:1028B4000AE018980830022108F075FB8DF85700DB
:1028C40002E001208DF857009DF8570058B944F2F2
:1028D4004C41C5F60201086820F48030189A126D44
:1028E4001043086003E09DF857008DF856001898CF
:1028F400C0788006002808D518982830022108F0EE
:10290400A9FC10B101208DF8560018988078800732
:10291400002832D51898C06F0190B8B10198B0F56D
:10292400807F08D00198B0F5007F0DD00198B0F5F4
:10293400407F0AD00BE044F22C41C5F6020108683E
:1029440040F40030086005E004E003E002E0012008
:102954008DF857009DF8570058B944F25441C5F614
:102964000201086820F44070189AD26F104308607E
:1029740003E09DF857008DF8560018988078C0063B
:1029840000281BD51898006F20B11898006FB0F17B
:10299400004F00D107E04DF22A60C0F6010040F27A
:1029A400E55104F0B6F944F25041C5F60201086855
:1029B40020F00040189A126F10430860189880782D
:1029C400800600281BD51898806E20B11898806E58
:1029D400B0F1807F00D107E04DF22A60C0F601001B
:1029E40040F2F95104F095F944F25041C5F6020160
:1029F400086820F08070189A926E10430860189846
:102A0400C0784006002820D51898D0F8B40028B122
:102A14001898D0F8B400B0F5004F00D107E04DF29B
:102A24002A60C0F6010040F20F6104F072F944F22A
:102A34001041C5F60201086820F4004008601898A7
:102A4400D0F8B4200868104308601898C0780006CD
:102A5400002820D51898406D48B11898406DB0F101
:102A6400805F04D01898406DB0F1005F00D107E09A
:102A74004DF22A60C0F6010040F2196104F049F9F0
:102A840044F24C41C5F60201086820F04050189AFF
:102A9400526D10430860189880780006002824D5E9
:102AA4001898D0F8880058B11898D0F88800B0F574
:102AB400800F05D01898D0F88800B0F5000F00D129
:102AC40007E04DF22A60C0F6010040F2236104F0F1
:102AD40020F944F25441C5F60201086820F440008C
:102AE400189AD2F888201043086018980079C00713
:102AF40070B118980830002108F055FA8DF8570085
:102B04009DF8570000B903E09DF857008DF8560072
:102B140018980079800700280ED5189808300121EC
:102B240008F041FA8DF857009DF8570000B903E00A
:102B34009DF857008DF85600189800794007002832
:102B44000ED518980830022108F02DFA8DF8570098
:102B54009DF8570000B903E09DF857008DF8560022
:102B640018980079000700280ED5189828300021FD
:102B740008F070FB8DF857009DF8570000B903E08A
:102B84009DF857008DF8560018980079C006002863
:102B94000ED518982830012108F05CFB8DF85700F9
:102BA4009DF8570000B903E09DF857008DF85600D2
:102BB40018980079800600280ED51898283002212C
:102BC40008F048FB8DF857009DF8570000B903E062
:102BD4009DF857008DF856009DF8560018B900204E
:102BE4008DF8670002E001208DF867009DF867000A
:042BF4001AB080BDD6
:102BF80088B0079044F22840C5F60200016801F049
:102C0800030106910068C0F30510059044F22C40BA
:102C1800C5F60200006800F001000490049844F230
:102C28003441C5F60201096889B2C908484300EE73
:102C3800100AB8EE400A8DED020A0598002800F047
:102C480012810698009038B10098012863D0009846
:102C5800022800F08480A6E044F20040C5F6020095
:102C68000068C0F3401090B344F20040C5F602007B
:102C78000068C0F3C10149F20000C0F2D030C8407A
:102C880003909DED030AB8EE400A9DED051AB8EED3
:102C9800411A80EE010A44F23040C5F6020000688D
:102CA8006FF35F2001EE100AB8EE411A9DED022A7B
:102CB8009FED723A82EE032A31EE021AB7EE002A2D
:102CC80031EE021A20EE010A8DED010A22E09DED97
:102CD800050AB8EE401A9FED6B0A80EE010A44F22D
:102CE8003040C5F6020000686FF35F2001EE100A5D
:102CF800B8EE411A9DED022A9FED603A82EE032A52
:102D080031EE021AB7EE002A31EE021A20EE010A5D
:102D18008DED010A6AE09DED050AB8EE401A9FEDB7
:102D2800580A80EE010A44F23040C5F602000068F5
:102D38006FF35F2001EE100AB8EE411A9DED022AEA
:102D48009FED4E3A82EE032A31EE021AB7EE002AC0
:102D580031EE021A20EE010A8DED010A46E09DEDE2
:102D6800050AB8EE401A9FED440A80EE010A44F2C3
:102D78003040C5F6020000686FF35F2001EE100ACC
:102D8800B8EE411A9DED022A9FED3C3A82EE032AE5
:102D980031EE021AB7EE002A31EE021A20EE010ACD
:102DA8008DED010A22E09DED050AB8EE401A9FED6F
:102DB800350A80EE010A44F23040C5F60200006888
:102DC8006FF35F2001EE100AB8EE411A9DED022A5A
:102DD8009FED2A3A82EE032A31EE021AB7EE002A54
:102DE80031EE021A20EE010A8DED010A9DED010A6D
:102DF80044F23040C5F60200016889B2490A01EE82
:102E0800101AB8EE411AB7EE002A31EE021A80EE17
:102E1800010A0799BCEEC00A81ED000A9DED010A7E
:102E28000168C1F3064101EE101AB8EE411A31EEFD
:102E3800021A80EE010A0799BCEEC00A81ED010A68
:102E48009DED010A0068C0F3066001EE100AB8EEB5
:102E5800411A31EE021A80EE010A0798BCEEC00A48
:102E680080ED020A06E0079900200860079948608B
:102E78000799886008B0704720BCBE4B0000004628
:082E88000024744A0024744C7C
:102E900088B0079044F22840C5F60200016801F0AE
:102EA000030106910068C0F30530059044F22C4000
:102EB000C5F602000068C0F300100490049844F2C4
:102EC0003C41C5F60201096889B2C908484300EED1
:102ED000100AB8EE400A8DED020A0598002800F0AD
:102EE00012810698009038B10098012863D00098AC
:102EF000022800F08480A6E044F20040C5F60200FB
:102F00000068C0F3401090B344F20040C5F60200E0
:102F10000068C0F3C10149F20000C0F2D030C840DF
:102F200003909DED030AB8EE400A9DED051AB8EE38
:102F3000411A80EE010A44F23840C5F602000068EA
:102F40006FF35F2001EE100AB8EE411A9DED022AE0
:102F50009FED723A82EE032A31EE021AB7EE002A92
:102F600031EE021A20EE010A8DED010A22E09DEDFC
:102F7000050AB8EE401A9FED6B0A80EE010A44F292
:102F80003840C5F6020000686FF35F2001EE100ABA
:102F9000B8EE411A9DED022A9FED603A82EE032AB7
:102FA00031EE021AB7EE002A31EE021A20EE010AC3
:102FB0008DED010A6AE09DED050AB8EE401A9FED1D
:102FC000580A80EE010A44F23840C5F60200006853
:102FD0006FF35F2001EE100AB8EE411A9DED022A50
:102FE0009FED4E3A82EE032A31EE021AB7EE002A26
:102FF00031EE021A20EE010A8DED010A46E09DED48
:10300000050AB8EE401A9FED440A80EE010A44F228
:103010003840C5F6020000686FF35F2001EE100A29
:10302000B8EE411A9DED022A9FED3C3A82EE032A4A
:1030300031EE021AB7EE002A31EE021A20EE010A32
:103040008DED010A22E09DED050AB8EE401A9FEDD4
:10305000340A80EE010A44F23840C5F602000068E6
:103060006FF35F2001EE100AB8EE411A9DED022ABF
:103070009FED2A3A82EE032A31EE021AB7EE002AB9
:1030800031EE021A20EE010A8DED010A9DED010AD2
:1030900044F23840C5F60200016889B2490A01EEDF
:1030A000101AB8EE411AB7EE002A31EE021A80EE7D
:1030B000010A0799BCEEC00A81ED000A9DED010AE4
:1030C0000168C1F3064101EE101AB8EE411A31EE63
:1030D000021A80EE010A0799BCEEC00A81ED010ACE
:1030E0009DED010A0068C0F3066001EE100AB8EE1B
:1030F000411A31EE021A80EE010A0798BCEEC00AAE
:1031000080ED020A06E007990020086007994860F0
:103110000799886008B0704720BCBE4B000000468D
:083120000024744A0024744CE1
:1031280088B0079044F22840C5F60200016801F013
:10313800030106910068C0F30550059044F22C4045
:10314800C5F602000068C0F300200490049844F219
:103158004441C5F60201096889B2C908484300EE2E
:10316800100AB8EE400A8DED020A0598002800F012
:1031780012810698009038B10098012863D0009811
:10318800022800F08480A6E044F20040C5F6020060
:103198000068C0F3401090B344F20040C5F6020046
:1031A8000068C0F3C10149F20000C0F2D030C84045
:1031B80003909DED030AB8EE400A9DED051AB8EE9E
:1031C800411A80EE010A44F24040C5F60200006848
:1031D8006FF35F2001EE100AB8EE411A9DED022A46
:1031E8009FED723A82EE032A31EE021AB7EE002AF8
:1031F80031EE021A20EE010A8DED010A22E09DED62
:10320800050AB8EE401A9FED6B0A80EE010A44F2F7
:103218004040C5F6020000686FF35F2001EE100A17
:10322800B8EE411A9DED022A9FED603A82EE032A1C
:1032380031EE021AB7EE002A31EE021A20EE010A28
:103248008DED010A6AE09DED050AB8EE401A9FED82
:10325800580A80EE010A44F24040C5F602000068B0
:103268006FF35F2001EE100AB8EE411A9DED022AB5
:103278009FED4E3A82EE032A31EE021AB7EE002A8B
:1032880031EE021A20EE010A8DED010A46E09DEDAD
:10329800050AB8EE401A9FED440A80EE010A44F28E
:1032A8004040C5F6020000686FF35F2001EE100A87
:1032B800B8EE411A9DED022A9FED3C3A82EE032AB0
:1032C80031EE021AB7EE002A31EE021A20EE010A98
:1032D8008DED010A22E09DED050AB8EE401A9FED3A
:1032E800340A80EE010A44F24040C5F60200006844
:1032F8006FF35F2001EE100AB8EE411A9DED022A25
:103308009FED2A3A82EE032A31EE021AB7EE002A1E
:1033180031EE021A20EE010A8DED010A9DED010A37
:1033280044F24040C5F60200016889B2490A01EE3C
:10333800101AB8EE411AB7EE002A31EE021A80EEE2
:10334800010A0799BCEEC00A81ED000A9DED010A49
:103358000168C1F3064101EE101AB8EE411A31EEC8
:10336800021A80EE010A0799BCEEC00A81ED010A33
:103378009DED010A0068C0F3066001EE100AB8EE80
:10338800411A31EE021A80EE010A0798BCEEC00A13
:1033980080ED020A06E00799002008600799486056
:1033A8000799886008B0704720BCBE4B00000046F3
:0833B8000024744A0024744C47
:1033C00080B596B01490139100208DF84B0013989F
:1033D00020B9149890F83E000F902BE01398042821
:1033E00004D1149890F83F000E9021E0139808281B
:1033F00004D1149890F840000D9017E013980C2811
:1034000004D1149890F841000C900DE01398102806
:1034100004D1149890F842000B9003E0149890F8AF
:1034200043000B900B980C900C980D900D980E90FB
:103430000E980F900F988DF84300139820B91498A8
:1034400090F844000A9017E01398042804D11498C7
:1034500090F8450009900DE01398082804D11498BD
:1034600090F84600089003E0149890F84700089000
:103470000898099009980A900A988DF842001498C3
:1034800000680021C4F20101884217D11398002876
:1034900000F0F6801398042800F0F28013980828B2
:1034A00000F0EE8013980C2800F0EA8013981028A2
:1034B00000F0E6801398142800F0E2801498006869
:1034C000B0F1804F0FD11398002800F0D9801398E5
:1034D000042800F0D5801398082800F0D1801398B4
:1034E0000C2800F0CD801498006840F20041C4F22E
:1034F000000188420FD11398002800F0C180139872
:10350000042800F0BD801398082800F0B9801398B3
:103510000C2800F0B5801498006840F60001C4F251
:10352000000188420FD11398002800F0A980139859
:10353000042800F0A5801398082800F0A1801398B3
:103540000C2800F09D801498006840F60041C4F2F9
:10355000000188420FD11398002800F09180139841
:10356000042800F08D801398082800F089801398B3
:103570000C2800F085801498006840F20041C4F2E5
:103580000101884211D11398002879D0139804289A
:1035900076D01398082873D013980C2870D01398FD
:1035A00010286DD0139814286AD01498006841F63A
:1035B0000001C4F20001884205D1139800285FD0B1
:1035C000139804285CD01498006841F60041C4F2B6
:1035D0000001884202D11398002851D01498006845
:1035E00042F20001C4F20001884202D1139800287F
:1035F00046D01498006844F20001C4F201018842E8
:1036000004D11398E0B31398042839D014980068B3
:1036100044F20041C4F20101884201D1139878B309
:103620001498006844F60001C4F20101884201D1F7
:10363000139828B3149800684EF20001C4F20001F8
:1036400088420AD11398D8B11398042818D0139837
:10365000082815D013980C2812D0149800684EF240
:103660000041C4F20001884211D1139840B113986F
:10367000042805D01398082802D013980C2806D1E6
:103680001398102803D01398142800D007E04DF2A7
:103690005D20C0F6010040F6AC0103F03CFB9DF854
:1036A0004300012803D19DF84200012803D00120E6
:1036B0008DF85700FAE0139820B91499022081F888
:1036C0003E002FE01398042805D11499022081F8B8
:1036D0003F00079025E01398082805D1149902208F
:1036E00081F8400006901AE013980C2805D114992F
:1036F000022081F8410005900FE01398102805D1B1
:103700001499022081F84200049004E014990220E8
:1037100081F8430004900498059005980690069857
:1037200007900798139820B91499022081F8440053
:1037300019E01398042805D11499022081F8450056
:1037400003900FE01398082805D11499022081F8FE
:103750004600029004E01499022081F8470002908C
:10376000029803900398139801900C2825D801998A
:10377000DFE801F0072323230E232323152323232C
:103780001C0014980168C86840F00200C86017E087
:1037900014980168C86840F00400C86010E01498EC
:1037A0000168C86840F00800C86009E01498016822
:1037B000C86840F01000C86002E001208DF84B009E
:1037C0009DF84B0000286DD11498006813990122D0
:1037D00014F07EFE149800680021C4F201018842B2
:1037E00044D014980068B0F1804F3FD0149800681E
:1037F00040F20041C4F20001884237D014980068BA
:1038000040F60001C4F2000188422FD014980068ED
:1038100040F60041C4F20001884227D014980068A5
:1038200040F20041C4F2010188421FD014980068A0
:1038300041F60001C4F20001884217D014980068D4
:1038400044F20001C4F2010188420FD014980068CC
:103850004EF20001C4F20001884207D014980068BB
:103860004EF20041C4F20001884215D1149800685C
:1038700080680721C0F201010840119011980628C4
:1038800009D01198B0F5803F05D0149801680868F8
:1038900040F00100086005E014980168086840F0F5
:1038A000010008609DF84B008DF857009DF8570007
:0438B00016B080BD11
:1038B40080B586B004900391029200208DF8070031
:1038C400029888B1029804280ED0029808280BD0D8
:1038D40002980C2808D00298102805D002981428C1
:1038E40002D002983C2800D107E04DF25D20C0F6DA
:1038F400010041F2B30103F00CFA03980068602858
:103904001FD00398006870281BD0039800684021DA
:10391400C0F20101884214D0039800685021C0F21B
:10392400010188420DD0039800686021C0F20101B2
:10393400884206D0039800687021C0F201018842D1
:1039440000D107E04DF25D20C0F6010041F2B40160
:1039540003F0DFF90398806818B10398806802289F
:1039640000D107E04DF25D20C0F6010041F2B5013F
:1039740003F0CFF90398006918B10398006904288B
:1039840000D107E04DF25D20C0F6010041F2B6011E
:1039940003F0BFF9049890F83C00012803D10220F9
:1039A4008DF8170048E20499012081F83C00029840
:1039B4000090142800F235820099DFE811F0150018
:1039C400320232023202A300320232023202120105
:1039D4003202320232027001320232023202CF016A
:1039E4003202320232020002049800680021C4F25A
:1039F4000101884264D004980068B0F1804F5FD020
:103A04000498006840F20041C4F20001884257D093
:103A14000498006840F60001C4F2000188424FD0C7
:103A24000498006840F60041C4F20001884247D07F
:103A34000498006840F20041C4F2010188423FD07A
:103A44000498006841F60001C4F20001884237D0AE
:103A54000498006841F60041C4F2000188422FD066
:103A64000498006842F20001C4F20001884227D0A1
:103A74000498006844F20001C4F2010188421FD096
:103A84000498006844F20041C4F20101884217D04E
:103A94000498006844F60001C4F2010188420FD082
:103AA400049800684EF20001C4F20001884207D075
:103AB400049800684EF20041C4F20001884200D12B
:103AC40007E04DF25D20C0F601004FF4865103F08B
:103AD40020F904980068039909F0EEFE049801683F
:103AE400886940F00800886104980168886920F0BA
:103AF4000400886103980269049801688869104386
:103B0400886191E1049800680021C4F201018842AF
:103B140044D004980068B0F1804F3FD00498006806
:103B240040F20041C4F20001884237D00498006892
:103B340040F60001C4F2000188422FD004980068C6
:103B440040F60041C4F20001884227D0049800687E
:103B540040F20041C4F2010188421FD00498006879
:103B640041F60001C4F20001884217D004980068AD
:103B740044F20001C4F2010188420FD004980068A5
:103B84004EF20001C4F20001884207D00498006894
:103B94004EF20041C4F20001884200D107E04DF228
:103BA4005D20C0F6010041F2D10103F0B2F804989F
:103BB4000068039914F05AFF04980168886940F476
:103BC4000060886104980168886920F480608861D5
:103BD4000398026904980168886940EA02208861B0
:103BE40022E1049800680021C4F20101884234D023
:103BF40004980068B0F1804F2FD00498006840F218
:103C04000041C4F20001884227D00498006840F6BD
:103C14000001C4F2000188421FD00498006840F6F5
:103C24000041C4F20001884217D00498006840F2B1
:103C34000041C4F2010188420FD0049800684EF29A
:103C44000001C4F20001884207D0049800684EF2D3
:103C54000041C4F20001884200D107E04DF25D202A
:103C6400C0F6010041F2E20103F053F80498006841
:103C7400039909F0F0FE04980168C86940F008004F
:103C8400C86104980168C86920F00400C8610398F9
:103C9400026904980168C8691043C861C4E00498C3
:103CA40000680021C4F20101884234D004980068FD
:103CB400B0F1804F2FD00498006840F20041C4F264
:103CC4000001884227D00498006840F60001C4F23D
:103CD400000188421FD00498006840F60041C4F2F5
:103CE4000001884217D00498006840F20041C4F2F1
:103CF400010188420FD0049800684EF20001C4F21A
:103D04000001884207D0049800684EF20041C4F2D2
:103D14000001884200D107E04DF25D20C0F60100A9
:103D240041F2F30102F0F5FF04980068039909F0E9
:103D34006BFF04980168C86940F40060C861049886
:103D44000168C86920F48060C86103980269049816
:103D54000168C86940EA0220C86165E00498006807
:103D64000021C4F20101884207D00498006840F29F
:103D74000041C4F20101884200D107E04DF25D2008
:103D8400C0F6010041F2041102F0C3FF0498006878
:103D9400039914F045FF04980168486D40F0080049
:103DA400486504980168486D20F00400486503984C
:103DB400026904980168486D1043486534E004982A
:103DC40000680021C4F20101884207D00498006809
:103DD40040F20041C4F20101884200D107E04DF2F3
:103DE4005D20C0F6010041F2151102F092FF049823
:103DF4000068039909F081FF04980168486D40F454
:103E04000060486504980168486D20F48060486546
:103E14000398026904980168486D40EA02204865E5
:103E240002E001208DF807000499002081F83C008D
:103E34009DF807008DF817009DF8170006B080BDA7
:103E440080B584B003900291002001900298009004
:103E54000C2800F278810099DFE811F00D0075015B
:103E6400750175018700750175017501E100750122
:103E7400750175012B01039800680021C4F201014A
:103E8400884264D003980068B0F1804F5FD00398F3
:103E9400006840F20041C4F20001884257D0039800
:103EA400006840F60001C4F2000188424FD0039834
:103EB400006840F60041C4F20001884247D00398EC
:103EC400006840F20041C4F2010188423FD00398E7
:103ED400006841F60001C4F20001884237D003981B
:103EE400006841F60041C4F2000188422FD00398D3
:103EF400006842F20001C4F20001884227D003980E
:103F0400006844F20001C4F2010188421FD0039802
:103F1400006844F20041C4F20101884217D00398BA
:103F2400006844F60001C4F2010188420FD00398EE
:103F340000684EF20001C4F20001884207D00398E1
:103F440000684EF20041C4F20001884200D107E04B
:103F54004DF25D20C0F6010041F2616102F0D9FE2C
:103F640003980068406B0190EDE00398006800211D
:103F7400C4F20101884244D003980068B0F1804F34
:103F84003FD00398006840F20041C4F20001884227
:103F940037D00398006840F60001C4F2000188425B
:103FA4002FD00398006840F60041C4F20001884213
:103FB40027D00398006840F20041C4F2010188420E
:103FC4001FD00398006841F60001C4F20001884242
:103FD40017D00398006844F20001C4F2010188423A
:103FE4000FD0039800684EF20001C4F20001884229
:103FF40007D0039800684EF20041C4F200018842E1
:1040040000D107E04DF25D20C0F6010041F26B6182
:1040140002F07FFE03980068806B019093E00398A0
:1040240000680021C4F20101884234D0039800687A
:10403400B0F1804F2FD00398006840F20041C4F2E1
:104044000001884227D00398006840F60001C4F2BA
:10405400000188421FD00398006840F60041C4F272
:104064000001884217D00398006840F20041C4F26E
:10407400010188420FD0039800684EF20001C4F297
:104084000001884207D0039800684EF20041C4F250
:104094000001884200D107E04DF25D20C0F6010026
:1040A40041F2766102F035FE03980068C06B01901E
:1040B40049E0039800680021C4F20101884234D029
:1040C40003980068B0F1804F2FD00398006840F245
:1040D4000041C4F20001884227D00398006840F6EA
:1040E4000001C4F2000188421FD00398006840F622
:1040F4000041C4F20001884217D00398006840F2DE
:104104000041C4F2010188420FD0039800684EF2C6
:104114000001C4F20001884207D0039800684EF2FF
:104124000041C4F20001884200D107E04DF25D2055
:10413400C0F6010041F2816102F0EBFD03980068D2
:0C414400006C0190FFE7019804B080BD02
:1041500088B00790079845F25931C4F258618842F7
:1041600040F0108148F21C30C2F20040016801F0BA
:104170001F01490006910168C1F3451105910068CE
:10418000C0F3C420049048F23030C2F2004001680D
:1041900001F01F0103910168C1F34311029100680E
:1041A000C0F3462000F2BC70019006980A300690D9
:1041B00006983C28C0F0C8800598069A48F6890100
:1041C000C8F68801A2FB013200EB52100590069858
:1041D000A0FB011251090901A1EB5211A0EB8100D2
:1041E000069005983C28C0F0AF800498059A48F6E0
:1041F0008901C8F68801A2FB013200EB521004903D
:104200000598A0FB011251090901A1EB5211A0EB85
:104210008100059004981828C0F096800020049032
:1042200003980130039002980138014600910B2851
:1042300000F289800099DFE801F0060F252E374053
:1042400049525B646D760398202804D301200390C3
:1042500002980130029077E09DF80400800740B991
:1042600003981E2804D30120039002980130029085
:1042700007E003981D2804D3012003900298013021
:10428000029061E00398202804D301200390029853
:104290000130029058E003981F2804D301200390B6
:1042A0000298013002904FE00398202804D30120A7
:1042B000039002980130029046E003981F2804D32F
:1042C000012003900298013002903DE003982028DD
:1042D00004D30120039002980130029034E0039847
:1042E000202804D3012003900298013002902BE093
:1042F00003981F2804D301200390029801300290F4
:1043000022E00398202804D3012003900298013072
:10431000029019E003981F2804D30120039002980B
:104320000130029010E0039820280BD30120039065
:104330000290019801300190019840F63C018842BA
:1043400000D31FE000E01DE0019948F60000CFF621
:10435000F07000EB4120029940EA411003990843B4
:1043600048F23031C2F2004108600498C002059959
:1043700040EA4110069940EA510048F21C31C2F26D
:084380000041086008B070471D
:10438800034C206804348047FBE702F0F7FBFEE7A4
:0443980050DC0108EC
:10439C000A15C90241EA5051C00241F0004140F2F5
:1043AC001E439A1A08DA20320DD4D141D04048402D
:1043BC009140D14048407047202A28BF202231FA32
:1043CC0002F0002170476FF000010846704700BFF3
:1043DC00F9B140F23D42B1FA81F3D21AC3F1200C8B
:1043EC0030FA0CFC9840994051EA0C0183054FEAD5
:1043FC00D02040EA41504FEAD12101EB025138BFA5
:10440C007047013041F100011B4208BF20F0010050
:10441C00704748B140F21D42B0FA80F3D21A98406E
:0C442C00C10A400501EB0251704700BFBF
:10443800002B35D129B9B0FBF2FC0CFB1202604607
:104448007047914215D22DE9F041B2FA82F39A40B1
:104458009940D3F1200C30FA0CFC51EA0C01984039
:1044680000F04EF8280036FA03F200210023BDE8D8
:10447800F081F0B5B1FBF2FC0CFB1211B2FA82F339
:104488009A409940D3F1200630FA06F63143984015
:1044980000F036F8614628003200DA400023F0BD0B
:1044A800F3B5B3FA83FC49085FEA300013FA0CF35A
:1044B800DCF1200432FA04F423430CB41A0000F0AF
:1044C8001FF80CBC33FA0CF3DCF11F0C35FA0CF5B1
:1044D80018BF013D03BCA5FB026705FB0377801BE2
:1044E800B941904271EB030C05D3821A71EB0303B7
:1044F800681C0021F0BD02000B0028000021F0BD5F
:10450800940D4FF6C2752D02B5FBF4F4D60A0136A8
:1045180004FB04F5A5FB0656F64306EB04165508FE
:1045280032BF00277708013505FB1677A6FB07473A
:104538007F0807EBC63714001500E7FB02457F1B11
:104548004D1C0400E7FB014505FB1206A64284BF8B
:10455800013DB618964224BF0135B61A704700BF10
:104568005AB3844690EA01039B071FD1830707D0FB
:1045780011F8013B00F8013B013AF7D11CE08446F1
:10458800203A09D32DE9F007B1E8F807A0E8F807C1
:10459800203AF9D2BDE8F0071C3205D451F8043BA3
:1045A80040F8043B043AF9D2043205D011F8013B33
:0C45B80000F8013B013AF9D16046704761
:1045C40000220B0011001A0084465AB3830704D05A
:1045D40000F8011B013AF9D124E0C9B241EA0121F2
:1045E40041EA0141202A11D3203A2DE9F0030B4678
:1045F4000C460D460E460F4688468946A0E8FA0347
:10460400203AFBD2BDE8F00320320BD0042A05D3B4
:1046140040F8041B043A05D0042AF9D200F8011B1F
:08462400013AFBD1604670472A
:0C462C00B0D701085846000838460008C6
:1046380085CF0108A5CF0108014D0108B1CF0108B8
:10464800A5CF0108014D0108F34C010851CF01081D
:10465800B2D7010848D9010848D9010848D9010842
:1046680048D9010848D9010848D9010848D901089A
:1046780048D9010848D90108FFFFFFFFFFFFFFFFE6
:10468800FFFFFFFFFFFF000076D70108FAD80108F7
:1046980086D3010817D90108DDD30108E8D8010835
:0846A800F1D80108E4D3010878
:1046B00008B50378BFF35B8F6BB94378012B07D044
:1046C00013F0020302D0054810F021FB02224270D1
:1046D00083F0010008BD0020FCE700BFF3D3010810
:1046E00080B598B0179116901698179980F480703D
:1046F0000843002840F0978044F25040C5F602007D
:10470000006800F007000B900B980890042800F256
:1047100086800899DFE801F00314257D360044F215
:104720000040C5F6020000688001002805D513A8E6
:10473000FEF762FA14980C9001E000200C9070E0F3
:1047400044F20040C5F6020000680001002805D5CB
:1047500010A8FEF79DFB10980C9001E000200C9033
:104760005FE044F20040C5F60200006880000028C7
:1047700005D50DA8FEF7D8FC0D980C9001E000209F
:104780000C904EE044F24C40C5F60200006800F088
:1047900040500A9044F20040C5F60200006840070D
:1047A00000280FD50A9868B944F20040C5F6020007
:1047B0000068C0F3C10149F20000C0F2D030C84027
:1047C0000C9025E044F20040C5F602000068C005E8
:1047D000002809D50A98B0F1805F05D140F6001095
:1047E000C0F23D000C9013E044F20040C5F6020018
:1047F00000688003002809D50A98B0F1005F05D150
:1048000047F64000C0F27D100C9001E000200C90B3
:1048100007E048F20000C0F2BB000C9001E000206D
:104820000C9000F023BC1698179980F48060084320
:10483000002840F09F8044F25840C5F6020000680E
:1048400000F460000B900B98079080B10798B0F5CA
:10485000001F1DD00798B0F5800F2AD00798B0F53B
:10486000C00F7ED00798B0F5000F33D07FE044F240
:104870000040C5F6020000688001002805D513A895
:10488000FEF7BAF914980C9001E000200C9070E04B
:1048900044F20040C5F6020000680001002805D57A
:1048A00010A8FEF7F5FA10980C9001E000200C908B
:1048B0005FE044F20040C5F6020000688000002876
:1048C00005D50DA8FEF730FC0D980C9001E00020F6
:1048D0000C904EE044F24C40C5F60200006800F037
:1048E00040500A9044F20040C5F6020000684007BC
:1048F00000280FD50A9868B944F20040C5F60200B6
:104900000068C0F3C10149F20000C0F2D030C840D5
:104910000C9025E044F20040C5F602000068C00596
:10492000002809D50A98B0F1805F05D140F6001043
:10493000C0F23D000C9013E044F20040C5F60200C6
:1049400000688003002809D50A98B0F1005F05D1FE
:1049500047F64000C0F27D100C9001E000200C9062
:1049600007E048F20000C0F2BB000C9001E000201C
:104970000C907BE31698179980F400600843002898
:1049800040F09F8044F25840C5F60200006800F0F5
:10499000E0600B900B98069080B10698B0F1807F94
:1049A0001DD00698B0F1007F2AD00698B0F1407F64
:1049B0007ED00698B0F1806F33D07FE044F20040A3
:1049C000C5F6020000688001002805D513A8FEF78F
:1049D00013F914980C9001E000200C9070E044F260
:1049E0000040C5F6020000680001002805D510A8A7
:1049F000FEF74EFA10980C9001E000200C905FE05A
:104A000044F20040C5F6020000688000002805D589
:104A10000DA8FEF789FB0D980C9001E000200C908A
:104A20004EE044F24C40C5F60200006800F04050F1
:104A30000A9044F20040C5F60200006840070028D2
:104A40000FD50A9868B944F20040C5F60200006824
:104A5000C0F3C10149F20000C0F2D030C8400C9050
:104A600025E044F20040C5F602000068C0050028B9
:104A700009D50A98B0F1805F05D140F60010C0F268
:104A80003D000C9013E044F20040C5F602000068BF
:104A90008003002809D50A98B0F1005F05D147F6D8
:104AA0004000C0F27D100C9001E000200C9007E067
:104AB00048F20000C0F2BB000C9001E000200C9016
:104AC000D4E21698179980F480500843002840F0EB
:104AD0009F8044F25040C5F60200006800F4E040B8
:104AE00009900998059080B10598B0F5805F1DD0B8
:104AF0000598B0F5005F2AD00598B0F5405F7ED0EC
:104B00000598B0F5804F33D07FE044F20040C5F601
:104B1000020000688001002805D513A8FEF76CF894
:104B200014980C9001E000200C9070E044F20040DA
:104B3000C5F6020000680001002805D510A8FEF7A0
:104B4000A7F910980C9001E000200C905FE044F26F
:104B50000040C5F6020000688000002805D50DA8B9
:104B6000FEF7E2FA0D980C9001E000200C904EE068
:104B700044F24C40C5F60200006800F040500A9034
:104B800044F20040C5F602000068400700280FD537
:104B90000A9868B944F20040C5F602000068C0F304
:104BA000C10149F20000C0F2D030C8400C9025E0AD
:104BB00044F20040C5F602000068C005002809D58F
:104BC0000A98B0F1805F05D140F60010C0F23D00B8
:104BD0000C9013E044F20040C5F602000068800328
:104BE000002809D50A98B0F1005F05D147F64000CA
:104BF000C0F27D100C9001E000200C9007E048F21C
:104C00000000C0F2BB000C9001E000200C902DE2EF
:104C10001698179980F400500843002840F08480CB
:104C200044F25040C5F60200006800F4E02009900C
:104C300009980490A0B10498B0F5803F14D004986E
:104C4000B0F5003F21D00498B0F5403F2ED0049835
:104C5000B0F5802F43D00498B0F5A02F50D060E07D
:104C600006F07DF90C905EE044F20040C5F60200CB
:104C700000680001002805D510A8FEF709F9119871
:104C80000C9001E000200C904DE044F20040C5F68D
:104C9000020000688000002805D50DA8FEF744FA40
:104CA0000E980C9001E000200C903CE044F2004093
:104CB000C5F602000068400700280DD544F2004008
:104CC000C5F602000068C0F3C10149F20000C0F25D
:104CD000D030C8400C9001E000200C9023E044F25A
:104CE0000040C5F602000068C005002805D540F662
:104CF0000010C0F23D000C9001E000200C9012E08A
:104D000044F20040C5F6020000688003002805D583
:104D100047F64000C0F27D100C9001E000200C909E
:104D200001E000200C90A1E11698179980F4002072
:104D30000843002840F0808044F25840C5F6020045
:104D4000006800F4403009900998039040B103983E
:104D5000B0F5803F15D00398B0F5003F22D068E051
:104D600044F20040C5F6020000680001002805D5A5
:104D700010A8FEF78DF810980C9001E000200C9020
:104D800059E044F20040C5F60200006880000028A7
:104D900005D50DA8FEF7C8F90F980C9001E000208A
:104DA0000C9048E044F24C40C5F60200006800F068
:104DB00040500A9044F20040C5F6020000684007E7
:104DC00000280FD50A9868B944F20040C5F60200E1
:104DD0000068C0F3C10149F20000C0F2D030C84001
:104DE0000C9025E044F20040C5F602000068C005C2
:104DF000002809D50A98B0F1805F05D140F600106F
:104E0000C0F23D000C9013E044F20040C5F60200F1
:104E100000688003002809D50A98B0F1005F05D129
:104E200047F64000C0F27D100C9001E000200C908D
:104E300001E000200C9019E11698179980F4803059
:104E40000843A0BB44F24C40C5F60200006800F4E1
:104E5000803009900998029020B10298B0F5803F07
:104E600011D021E044F20040C5F602000068800144
:104E7000002805D513A8FDF7BFFE14980C9001E09B
:104E800000200C9012E044F20040C5F602000068D9
:104E90000001002805D510A8FDF7FAFF12980C9024
:104EA00001E000200C9001E000200C90DEE016985C
:104EB000179980F480400843002840F0848044F231
:104EC0005840C5F60200006800F0E04009900998DB
:104ED0000190A0B10198B0F1805F14D00198B0F1B9
:104EE000005F21D00198B0F1405F2ED00198B0F161
:104EF000804F43D00198B0F1A04F50D060E006F051
:104F000006FB0C905EE044F20040C5F6020000682B
:104F10000001002805D510A8FDF7BAFF11980C90E4
:104F200001E000200C904DE044F20040C5F6020084
:104F300000688000002805D50DA8FEF7F5F80E984A
:104F40000C9001E000200C903CE044F20040C5F6DB
:104F500002000068400700280DD544F20040C5F665
:104F600002000068C0F3C10149F20000C0F2D03075
:104F7000C8400C9001E000200C9023E044F2004077
:104F8000C5F602000068C005002805D540F60010EF
:104F9000C0F23D000C9001E000200C9012E044F2C1
:104FA0000040C5F6020000688003002805D547F6DA
:104FB0004000C0F27D100C9001E000200C9001E058
:104FC00000200C9052E01698179980F40040084396
:104FD000002849D144F25040C5F60200006800F0B4
:104FE000405009900998009040B10098B0F1805F5E
:104FF00015D00098B0F1005F22D032E044F20040BA
:10500000C5F6020000688003002805D547F6400079
:10501000C0F27D100C9001E000200C9023E044F2DF
:105020000040C5F6020000688001002805D513A8DD
:10503000FDF7E2FD14980C9001E000200C9012E0C6
:1050400044F20040C5F6020000680001002805D5C2
:1050500010A8FDF71DFF11980C9001E000200C90A6
:1050600001E000200C9001E000200C900C9818B09A
:0250700080BD01
:1050720080B594B01290002311931298109010985A
:105082000FA94FF480620FF0FCF91190119840B112
:105092004DF28640C0F601000FF061FD11981390A9
:1050A20002E14DF2B470C0F601000B900B990F981B
:1050B2006A46B4239361012353614FF0000CC2F896
:1050C20010C04FF01F0CC2F80CC0C2F808C04FF459
:1050D200806CC2F804C0106047F26070C2F20040F7
:1050E20044F6B962C0F6010217F03BFC1190119828
:1050F20048B10B994CF6DC70C0F601000FF02FFDA1
:1051020011981390D0E010980EA94FF480620023FA
:105112000FF0B7F91190119840B14DF28640C0F6E8
:1051220001000FF01CFD11981390BDE04CF6EF70DA
:10513200C0F601000A900A990E986A46B423936158
:10514200012353614FF0000CC2F810C04FF01F0C46
:10515200C2F80CC0C2F808C04FF4806CC2F804C098
:10516200106047F61400C2F2004046F6B502C0F6DF
:10517200000217F0F6FB1190119848B10A994CF60B
:10518200DC70C0F601000FF0EAFC119813908BE07E
:1051920010980DA94FF4806200230FF072F911905C
:1051A200119840B14DF28640C0F601000FF0D7FCD5
:1051B2001198139078E04DF2A840C0F601000990D2
:1051C20009990D986A46B4239361012353614FF004
:1051D200000CC2F810C04FF01F0CC2F80CC0C2F88D
:1051E20008C04FF4806CC2F804C0106047F6C800D3
:1051F200C2F2004046F22132C0F6000217F0B1FBC3
:105202001190119848B109994CF6DC70C0F6010072
:105212000FF0A5FC1198139046E010980CA94FF4DA
:10522200007200230FF02DF91190119840B14DF248
:105232008640C0F601000FF092FC1198139033E003
:105242004CF6FA70C0F60100089008990C986A466C
:10525200B4239361012353614FF0000CC2F810C0D4
:105262004FF01F0CC2F80CC0C2F808C04FF4007C0B
:10527200C2F804C0106047F63020C2F2004044F683
:105282002152C0F6010217F06CFB1190119848B13F
:1052920008994CF6DC70C0F601000FF060FC119822
:0E52A200139001E011981390139814B080BD82
:1052B00080B59EB01D9000208DF867001D98406855
:1052C0004BF62041C0F2BE01884200D807E04DF6FF
:1052D000A220C0F6010040F6E23101F01CFD1D984D
:1052E0008068B0F1805F07D01D98806820B11D985C
:1052F0008068B0F5805F00D107E04DF6A220C0F6CF
:10530000010040F6E33101F006FD1D98006840F60B
:105310000041C5F60001884211D11D98C06820B136
:105320001D98C068B0F5005F00D107E04DF6A220DF
:10533000C0F6010040F6E63101F0EDFC2BE01D98CF
:10534000C068B0F5805F0CD01D98C06848B11D984A
:10535000C068B0F5405F04D01D98C068B0F5005F2C
:1053600000D107E04DF6A220C0F6010040F6EA3178
:1053700001F0D1FC1D98006A20B11D98006AB0F5BB
:10538000006F00D107E04DF6A220C0F6010040F604
:10539000EB3101F0C0FC1D98006948B11D9800690F
:1053A000B0F5806F04D01D980069B0F5C06F00D1D2
:1053B00007E04DF6A220C0F6010040F6EE3101F004
:1053C000AAFC1D9840696FF00C01084203D11D989A
:1053D000406900B107E04DF6A220C0F6010040F69A
:1053E000EF3101F098FC1D98806970B11D988069BB
:1053F000B0F5807F09D01D988069B0F5007F04D09A
:105400001D988069B0F5407F00D107E04DF6A220DD
:10541000C0F601004FF43F6101F07DFC1D98C069AA
:1054200020B11D98C069B0F5004F00D107E04DF6DE
:10543000A220C0F6010040F6F13101F06CFC1D988D
:10544000406A58B31D98406A012827D01D98406AC9
:10545000022823D01D98406A03281FD01D98406A57
:1054600004281BD01D98406A052817D01D98406A53
:10547000062813D01D98406A07280FD01D98406A4F
:1054800008280BD01D98406A092807D01D98406A4B
:105490000A2803D01D98406A0B2800D107E04DF67A
:1054A000A220C0F6010040F6F23101F034FC1D9953
:1054B00088680B694A69C9691843104308431C90FE
:1054C0001D980068006846F6F311CCF6FF7108409D
:1054D0001C9908431D99096808601D980068406878
:1054E00020F440501D9A1168D268104348601D98FE
:1054F00080691C901D98006840F60041C5F60001C7
:10550000884204D01D98016A1C9808431C901D987D
:10551000006880684FF2FF41C1F2FF1108401C99FA
:1055200008431D99096888601D980068C06A20F0CA
:105530000F001D9A1168526A1043C8621D980068D6
:1055400041F20001C4F20101884240F03F8044F280
:105550005440C5F60200006800F038000146109182
:1055600028282FD81099DFE801F0152D2D2D2D2D8D
:105570002D2D192D2D2D2D2D2D2D1D2D2D2D2D2D7F
:105580002D2D212D2D2D2D2D2D2D252D2D2D2D2D5F
:105590002D2D290001208DF86D0016E004208DF8D6
:1055A0006D0012E008208DF86D000EE010208DF8DF
:1055B0006D000AE020208DF86D0006E040208DF897
:1055C0006D0002E080208DF86D004DE21D980068AE
:1055D00044F20041C4F2000188422CD144F254400C
:1055E000C5F60200006800F0070001460F9105288B
:1055F0001DD80F99DFE801F003070B0F13170020E8
:105600008DF86D0016E004208DF86D0012E0082082
:105610008DF86D000EE010208DF86D000AE020205E
:105620008DF86D0006E040208DF86D0002E08020CE
:105630008DF86D0018E21D98006844F60001C4F270
:10564000000188422CD144F25440C5F602000068A3
:1056500000F0070001460E9105281DD80E99DFE8DD
:1056600001F003070B0F131700208DF86D0016E0F3
:1056700004208DF86D0012E008208DF86D000EE01A
:1056800010208DF86D000AE020208DF86D0006E0F6
:1056900040208DF86D0002E080208DF86D00E3E180
:1056A0001D98006844F60041C4F2000188422CD1E4
:1056B00044F25440C5F60200006800F007000146BD
:1056C0000D9105281DD80D99DFE801F003070B0F98
:1056D000131700208DF86D0016E004208DF86D0082
:1056E00012E008208DF86D000EE010208DF86D009E
:1056F0000AE020208DF86D0006E040208DF86D0056
:1057000002E080208DF86D00AEE11D98006845F242
:105710000001C4F2000188422CD144F25440C5F685
:105720000200006800F0070001460C9105281DD812
:105730000C99DFE801F003070B0F131700208DF819
:105740006D0016E004208DF86D0012E008208DF841
:105750006D000EE010208DF86D000AE020208DF81D
:105760006D0006E040208DF86D0002E080208DF88D
:105770006D0079E11D98006841F20041C4F2010119
:10578000884240F03F8044F25440C5F60200006871
:1057900000F0380001460B9128282FD80B99DFE83C
:1057A00001F0152D2D2D2D2D2D2D192D2D2D2D2DBE
:1057B0002D2D1D2D2D2D2D2D2D2D212D2D2D2D2D35
:1057C0002D2D252D2D2D2D2D2D2D290001208DF850
:1057D0006D0016E004208DF86D0012E008208DF8B1
:1057E0006D000EE010208DF86D000AE020208DF88D
:1057F0006D0006E040208DF86D0002E080208DF8FD
:105800006D0031E11D98006847F60001C4F2000107
:1058100088422CD144F25440C5F60200006800F0E2
:10582000070001460A9105281DD80A99DFE801F012
:1058300003070B0F131700208DF86D0016E00420EE
:105840008DF86D0012E008208DF86D000EE010203C
:105850008DF86D000AE020208DF86D0006E04020F4
:105860008DF86D0002E080208DF86D00FCE01D9841
:10587000006847F60041C4F2000188422CD144F28E
:105880005440C5F60200006800F007000146099187
:1058900005281DD80999DFE801F003070B0F13173E
:1058A00000208DF86D0016E004208DF86D0012E0E8
:1058B00008208DF86D000EE010208DF86D000AE0D4
:1058C00020208DF86D0006E040208DF86D0002E08C
:1058D00080208DF86D00C7E01D98006841F600013A
:1058E000C4F20101884240F03F8044F25440C5F6C2
:1058F0000200006800F038000146089128282FD8DF
:105900000899DFE801F0152D2D2D2D2D2D2D192DA8
:105910002D2D2D2D2D2D1D2D2D2D2D2D2D2D212DD3
:105920002D2D2D2D2D2D252D2D2D2D2D2D2D2900E0
:1059300001208DF86D0016E004208DF86D0012E056
:1059400008208DF86D000EE010208DF86D000AE043
:1059500020208DF86D0006E040208DF86D0002E0FB
:1059600080208DF86D007FE01D98006841F60041B1
:10597000C4F20101884240F03F8044F25440C5F631
:105980000200006800F038000146079128282FD84F
:105990000799DFE801F0152D2D2D2D2D2D2D192D19
:1059A0002D2D2D2D2D2D1D2D2D2D2D2D2D2D212D43
:1059B0002D2D2D2D2D2D252D2D2D2D2D2D2D290050
:1059C00001208DF86D0016E004208DF86D0012E0C6
:1059D00008208DF86D000EE010208DF86D000AE0B3
:1059E00020208DF86D0006E040208DF86D0002E06B
:1059F00080208DF86D0037E01D98006840F600416A
:105A0000C5F6000188422CD144F25840C5F6020088
:105A1000006800F007000146069105281DD8069988
:105A2000DFE801F003070B0F131702208DF86D005C
:105A300016E004208DF86D0012E008208DF86D004E
:105A40000EE010208DF86D000AE020208DF86D002A
:105A500006E040208DF86D0002E080208DF86D009A
:105A600002E080208DF86D001D98006840F600412E
:105A7000C5F60001884240F09E809DF86D00014609
:105A8000059102280FD00598042810D00598082801
:105A900013D00598102816D0059820282FD00598E7
:105AA000402832D035E005F032FD119036E015A8DF
:105AB000FDF7EEF91698119030E012A8FDF734FBCF
:105AC000139811902AE044F20040C5F602000068E5
:105AD000C0F3401068B144F20040C5F6020000680F
:105AE000C0F3C10149F20000C0F2D030C8401190AB
:105AF00004E049F20000C0F2D03011900EE040F610
:105B00000010C0F23D00119008E04FF400401190E9
:105B100004E00020119001208DF867001198002802
:105B200048D011981D994A6A4CF6E031C0F601013F
:105B300031F81210B0FBF1F0189018981D994968CF
:105B400001EB4101884205D318981D994968B0EBD3
:105B5000013F03D901208DF867002BE011981D99B2
:105B60004A6803924A6A4CF6E031C0F6010131F806
:105B70001220002304931946FEF75EFC039A049B4F
:105B8000090241EA1061000210EB520041F10001EC
:105B9000FEF752FC1A901A98B0F5407F07D31A9876
:105BA000000D20B91A981D990968C86002E001200B
:105BB0008DF867002DE11D98C069B0F5004F40F0E9
:105BC0009C809DF86D0001460291402800F25E80A5
:105BD0000299DFE801F021255B5B295B5B5B2F5BB2
:105BE0005B5B5B5B5B5B355B5B5B5B5B5B5B5B5B2B
:105BF0005B5B5B5B5B5B515B5B5B5B5B5B5B5B5BFF
:105C00005B5B5B5B5B5B5B5B5B5B5B5B5B5B5B5BE4
:105C10005B5B5B5B5B5B570005F0A1F911903AE0C1
:105C200005F0B0F9119036E015A8FDF731F9169896
:105C3000119030E012A8FDF777FA139811902AE03E
:105C400044F20040C5F602000068C0F3401068B19D
:105C500044F20040C5F602000068C0F3C10149F2F9
:105C60000000C0F2D030C840119004E049F20000BA
:105C7000C0F2D03011900EE040F60010C0F23D00AE
:105C8000119008E04FF40040119004E000201190C2
:105C900001208DF86700119870B311981D9A516812
:105CA000536A4CF6E032C0F6010232F81320B0FB22
:105CB000F2F0400000EB5100B0FBF1F01A901A989E
:105CC000102816D3BDF86A0098B91A9820F00F0072
:105CD000ADF86E001A9800F00E01BDF86E0040EAB3
:105CE0005100ADF86E00BDF86E001D990968C860DE
:105CF00002E001208DF867008BE09DF86D00014601
:105D00000191402800F25E800199DFE801F0212531
:105D10005B5B295B5B5B2F5B5B5B5B5B5B5B355B57
:105D20005B5B5B5B5B5B5B5B5B5B5B5B5B5B515BCD
:105D30005B5B5B5B5B5B5B5B5B5B5B5B5B5B5B5BB3
:105D40005B5B5B5B5B5B5B5B5B5B5B5B5B5B570002
:105D500005F005F911903AE005F014F9119036E0DC
:105D600015A8FDF795F81698119030E012A8FDF7E8
:105D7000DBF9139811902AE044F20040C5F60200C6
:105D80000068C0F3401068B144F20040C5F602005C
:105D90000068C0F3C10149F20000C0F2D030C84031
:105DA000119004E049F20000C0F2D03011900EE0F2
:105DB00040F60010C0F23D00119008E04FF40040A2
:105DC000119004E00020119001208DF867001198D7
:105DD000F8B111981D9A5168536A4CF6E032C0F63A
:105DE000010232F81320B0FBF2F000EB5100B0FBDF
:105DF000F1F01A901A98102808D3BDF86A0028B953
:105E0000BDF868001D990968C86002E001208DF89E
:105E100067001D990120A1F86A001D99A1F868008A
:105E20001D99002048671D9988679DF867001EB07E
:025E300080BD33
:105E320080B586B044F2D840C5F60200016841F050
:105E420001010160006800F00100059005980B2037
:105E5200019000220392114601F018FC01980FF004
:105E62008CFA039A0C200290114601F00FFC029862
:105E72000FF083FA039A0D200490114601F006FCFC
:0A5E820004980FF07AFA06B080BD14
:105E8C0080B586B0059048F28420C2F200400068CC
:105E9C00012808D1002013F069FE20B1059990204B
:105EAC00C1F88C00F1E00598D0F8900000F00300E8
:105EBC0003900598D0F888000090082800F2E18043
:105ECC000099DFE801F06074888D0592DED13F0007
:105EDC0005990020C1F88C0048F23820C2F200402D
:105EEC004DF68801C0F60101002220230EF091FC32
:105EFC0060B948F21820C2F200404DF6A101C0F67C
:105F0C000101002220230EF084FC18B10599902089
:105F1C00C1F88C0048F28420C2F20040006880B9BD
:105F2C00002013F007FE0490049830B948F2842145
:105F3C00C2F200410120086003E005999020C1F8ED
:105F4C008C00A2E005990020C1F88C000BF0D4FB6A
:105F5C000490049820B105999020C1F88C0005E0BC
:105F6C0048F28421C2F200410020086048F2382037
:105F7C00C2F200400EF0E4FC48F21820C2F20040DD
:105F8C000EF0DEFC81E005999020C1F88C0005989C
:105F9C00036FD0F89410D0F898201944039B0BF0A1
:105FAC0000FC18B905990020C1F88C006DE005992A
:105FBC009020C1F88C000598036FD0F89410D0F89D
:105FCC0098201944039B0BF0A9FC18B905990020E3
:105FDC00C1F88C0059E005990020C1F88C0054E000
:105FEC0005990020C1F88C004FE00598D0F8982056
:105FFC00039B00210BF0D5FB0490049820B104986E
:10600C000599C1F88C0040E0002102910598D0F868
:10601C00900002AA01AB13F04BFE0490049820B13F
:10602C0005999020C1F88C002FE00298B8B100209F
:10603C0013F09CFD20B105999020C1F88C0024E050
:10604C0005980299D0F89820039B0BF0AAFB0490BA
:10605C00049820B104980599C1F88C0015E00599B5
:10606C000020C1F88C0010E00598D0F89820039B14
:10607C0000210BF053FC049004980599C1F88C0096
:0E608C0003E005999020C1F88C0006B080BD9D
:10609A0080B59AB000201990189017901690159014
:1060AA0044F2E040C5F60200016841F010010160C7
:1060BA00006800F010001490149844F2E040C5F60D
:1060CA000200016841F004010160006800F0040068
:1060DA001390139844F2E040C5F60200016841F0BB
:1060EA0020010160006800F020001290129844F22A
:1060FA00E040C5F60200016841F0800101600068D5
:10610A0000F080001190119844F2E040C5F60200B8
:10611A00016841F001010160006800F0010010907F
:10612A00109844F2E040C5F60200016841F002010D
:10613A000160006800F002000F900F9844F2E040FE
:10614A00C5F60200016841F040010160006800F0F4
:10615A0040000E900E9844F2E040C5F60200016835
:10616A0041F008010160006800F008000D900D98E8
:10617A0041F20000C5F6020001904AF2C001009106
:10618A000022099211F079F9099A41F20040C5F604
:10619A00020003904FF40041029111F06EF9099A3E
:1061AA0041F60000C5F6020008904BF6036104911F
:1061BA0011F063F9099A40F60040C5F6020006900C
:1061CA004FF49061059111F058F90198099940F23C
:1061DA003F721592032207921692179115A90C91F4
:1061EA0003F0BAF8009B0198099A0C9915930123B8
:1061FA000A9316931792189203F0AEF8079A099821
:10620A000C9942F23F0315931692179040F600003C
:10621A00C5F6020003F0A0F80398079B099A0C99A7
:10622A0047F6FF7CCDF854C01693179203F094F802
:10623A00079A09980C9949F6FF63159316921790D5
:10624A000020C5F602000B9003F086F8079A099819
:10625A000C994FF6FF7315931692179040F200406F
:10626A00C5F6020003F078F8DDF808C00398099A29
:10627A000A9B0C99CDF854C016931792189203F002
:10628A006BF8DDF810C00898099A0A9B0C99CDF8AA
:10629A0054C016931792189203F05EF8DDF814C0F2
:1062AA000698099A0A9B0C99CDF854C0169317922E
:1062BA00189203F051F80698099A0C994FF4005372
:1062CA0015931692179203F047F80698079B099AB6
:1062DA000C994CF27B0CCDF854C01693179203F02C
:1062EA003BF8079B0898099A0C9944F2FC1CCDF8D4
:1062FA0054C01693179203F02FF8099B0A9A0B9829
:10630A000C994FF4807CCDF854C01693179203F081
:06631A0023F81AB080BD5B
:1063200080B586B0059048F25830C2F2004000783F
:10633000BFF35F8FC00728BB48F25830C2F200405D
:10634000FEF7B6F9F0B169463C20486028200860A5
:1063500048F22410C2F200404DF2C571C0F60101AE
:1063600046F6B803C2F2004301220EF0A1F948F24A
:106370004C31C2F20041086048F25830C2F200408D
:1063800016F026FE48F24C30C2F20040006828B1F8
:106390004DF2D270C0F601000EF0E2FB47F640402D
:1063A000C2F2004040F20011C3F200014FF48072CB
:1063B0000AF04FFB47F65070C2F20040006810210F
:1063C000C4F20201884200F0A18047F65070C2F288
:1063D000004000682821C4F20201884200F0968043
:1063E00047F65070C2F2004000684021C4F202013A
:1063F000884200F08B8047F65070C2F2004000687F
:106400005821C4F20201884200F0808047F65070A3
:10641000C2F2004000687021C4F20201884275D0C7
:1064200047F65070C2F2004000688821C4F20201B1
:1064300088426BD047F65070C2F200400068A0213D
:10644000C4F20201884261D047F65070C2F20040A7
:106450000068B821C4F20201884257D047F6507054
:10646000C2F20040006840F21041C4F202018842CA
:106470004CD047F65070C2F20040006840F228410C
:10648000C4F20201884241D047F65070C2F2004087
:10649000006840F24041C4F20201884236D047F61B
:1064A0005070C2F20040006840F25841C4F202014C
:1064B00088422BD047F65070C2F20040006840F28C
:1064C0007041C4F20201884220D047F65070C2F2F7
:1064D0000040006840F28841C4F20201884215D0B1
:1064E00047F65070C2F20040006840F2A041C4F28A
:1064F000020188420AD047F65070C2F2004000689C
:1065000040F2B841C4F20201884209D147F6507006
:10651000C2F200400168086820F00800086008E046
:1065200047F65070C2F200400168086820F004008D
:10653000086048F24C30C2F200400068002865D183
:1065400048F22410C2F2004048F24831C2F2004141
:106550004FF0FF3216F060F904900498002850D1F3
:1065600048F24830C2F2004000680068B0F5807F11
:1065700007D948F24830C2F2004001684FF48070F9
:10658000086048F24830C2F20040006801684DF2ED
:106590000500C0F601000EF0E3FA00200390039816
:1065A00048F24831C2F2004109680968884221D2A4
:1065B00048F24830C2F2004000680399084400796C
:1065C000202809DB48F24830C2F2004000680399F5
:1065D00008440079029001E05F2002900298C1B265
:1065E0004DF21800C0F601000EF0BAFA039801301F
:1065F0000390D4E74DF21B00C0F601000EF0B0FA94
:1066000003E04FF47A7015F0BDFD03E042F2107024
:0666100015F0B8FD8DE756
:1066160080B588B0039040F20010C3F200000790E6
:106626004FF480700690069801281CDB069807999F
:1066360001F01F010844059007980490BFF34F8F9F
:1066460004984EF65C71CEF2000108600498203082
:10665600049005982038059005980028F0DCBFF3D3
:106666004F8FBFF36F8F48F25030C2F20040006880
:106676004CF6CD41CCF6CC41A0FB0121C90801EB7B
:106686008101A0EB410048F24431C2F200410860AA
:106696000020029002980399884218D2029A40F28A
:1066A6000010C3F20000805C48F24431C2F200419F
:1066B600096801EB811346F63811C2F2004101EB7D
:1066C600830111440871029801300290E2E7039AAF
:1066D60048F24431C2F20041086800EB801346F6E6
:1066E6003810C2F2004040F82320096801EB8111FE
:1066F60000EB8100019048F22410C2F2004001A98B
:10670600002216F0CCF848F25031C2F20041086877
:106716000130086047F64040C2F2004040F20011E6
:10672600C3F200014FF480720AF090F947F65070F8
:10673600C2F2004000681021C4F20201884200F053
:10674600A18047F65070C2F2004000682821C4F2CA
:106756000201884200F0968047F65070C2F200406F
:1067660000684021C4F20201884200F08B8047F69F
:106776005070C2F2004000685821C4F202018842FB
:1067860000F0808047F65070C2F200400068702129
:10679600C4F20201884275D047F65070C2F200403A
:1067A60000688821C4F2020188426BD047F6507017
:1067B600C2F200400068A021C4F20201884261D002
:1067C60047F65070C2F200400068B821C4F20201D8
:1067D600884257D047F65070C2F20040006840F237
:1067E6001041C4F2020188424CD047F65070C2F202
:1067F6000040006840F22841C4F20201884241D0BC
:1068060047F65070C2F20040006840F24041C4F2C0
:106816000201884236D047F65070C2F20040006846
:1068260040F25841C4F2020188422BD047F650701C
:10683600C2F20040006840F27041C4F20201884290
:1068460020D047F65070C2F20040006840F28841FE
:10685600C4F20201884215D047F65070C2F20040D9
:10686600006840F2A041C4F2020188420AD047F60D
:106876005070C2F20040006840F2B841C4F2020112
:10688600884209D147F65070C2F200400168086894
:1068960020F00800086008E047F65070C2F2004099
:0E68A6000168086820F00400086008B080BD9A
:1068B400B0B58CB00B900EF0B9FA42F2107015F02E
:1068C4005FFC4FF47A7015F05BFC48F24030C2F282
:1068D4000040026848F6A330CBF62E20A2FB00103D
:1068E4000009162100FB11200A900A9948F26C70E5
:1068F400C2F2004000EB4110007EC00758B10A9973
:1069040048F26C70C2F2004000EB4110407EC007B8
:10691400002840F08B800A9A48F26C70C2F2004062
:1069240000EB4211520182584B688868D1F80CC0C0
:10693400D1F810E04C694DF2C045C0F60105694636
:106944000D61CC60C1F808E0C1F804C0086040F2F1
:106954000020C3F2000007904DF21E01C0F60101B1
:1069640016F00EFA079816F0A9FA0990099800286B
:106974005CD009994DF2C240C0F601000EF0EEF869
:10698400002008900898099988421DD2089940F27D
:106994000020C3F20000405C202807DB089940F285
:1069A4000020C3F20000405C069001E05F200690E6
:1069B4000698C1B24DF22D00C0F601000EF0CEF8DB
:1069C400089801300890DDE74DF23000C0F6010070
:1069D4000EF0C4F840F20020C3F20000059016F057
:1069E4006DFA059982B247F64040C2F2004012F0B7
:1069F400E9FC0A9948F26C70C2F2004000EB4110C5
:106A0400007EC00740B10A9948F26C70C2F200409F
:106A140000EB4111012048760A9948F26C70C2F2E9
:106A2400004000EB4110408B15F0AAFB0A9948F294
:106A34006C70C2F2004000EB4110808B08B30A98DE
:106A440048F26C71C2F2004101EB4012D08B01306C
:106A5400D08380B20A9A01EB4211898B88420FDB02
:106A64000A9948F26C70C2F2004000EB4111002018
:106A7400C88348F24031C2F200410868013008601E
:106A840006E048F24031C2F2004108680130086073
:026A940017E702
:106A960080B586B00490012003900398052835DC64
:106AA6004DF63400C0F601000EF057F840F60040EF
:106AB600C5F6020001904FF480610091012210F0AA
:106AC600DEFC322015F05BFB00990198002210F0E5
:106AD600D6FC0DF10B0000F020F858B103994DF2E9
:106AE6005F00C0F6010005220EF037F801208DF890
:106AF60017000EE003994DF28E00C0F60100052244
:106B06000EF02BF8039801300390C6E700208DF8AD
:0A6B160017009DF8170006B080BDBF
:106B200080B584B002900DF02DFC01900DF02AFC90
:106B30000199401A42F20F7188421BD8642015F067
:106B400021FB40F60040C5F602004FF4005110F062
:106B500075FC01280DD10DF015FC0199411A4DF27B
:106B60002450C0F601000DF0FBFF01208DF80F004E
:106B700003E0DBE700208DF80F009DF80F0004B064
:026B800080BDD6
:026B820070475A
:106B840080B584B0002000904DF65500C0F6010099
:106B94004DF66E01C0F601014DF6FA12C0F601027F
:106BA4000DF0DCFF00F07BF84EF61450CEF200003E
:106BB40000688003002800D519E0BFF34F8FBFF3AE
:106BC4006F8F4EF65071CEF2000100200860BFF3C3
:106BD4004F8FBFF36F8F4EF61451CEF20001086849
:106BE40040F400300860BFF34F8FBFF36F8F4EF651
:106BF4001450CEF200000068C003002800D537E02E
:106C04004EF68451CEF2000100200860BFF34F8F8E
:106C14004EF68050CEF20000006803900398C0F353
:106C24004E3002900398C0F3C90001900299019874
:106C3400800761F34D104EF66071CEF200010860DA
:106C44000198411E01910028F0D10298411E029141
:106C54000028E7D1BFF34F8F4EF61451CEF2000156
:106C6400086840F480300860BFF34F8FBFF36F8F24
:106C740000F087FC0EF040F9FFF70DFAFFF7D7F8A4
:106C840000F04CF800F034F9FFF779FF00F085FBD1
:0E6C940000F086FA0EF09CFA0EF03CF8FEE7D7
:106CA20080B586B000200190059004900390029078
:106CB20000F038FD019801218DF808108DF80900C7
:106CC20003901F228DF8102087228DF811208DF855
:106CD20012008DF813008DF814108DF815108DF830
:106CE20016008DF8170002A80EF0BBFB04200EF070
:066CF200A0FB06B080BD0E
:106CF80080B582B001900198006841F20041C4F269
:0E6D08000001884201D100F075FC02B080BD90
:0A6D160082B00190009102B07047B6
:106D200080B582B048F2F410C2F20040019044F203
:106D30000001C5F600010160002141607F228260F0
:106D4000FF22C26001618161C161416104F0F2FB17
:0A6D500008B10EF03BF902B080BD5F
:106D5A0080B5B0B02F906846B821FDF72EFC2F9869
:106D6A00006844F20001C5F60001884215D10020EE
:106D7A0001904FF4800000904FF480702C90684688
:106D8A00FAF72BFD08B10EF01CF944F27041C5F672
:0E6D9A000201086840F40040086030B080BD7F
:106DA80080B5BEB03D9000203C903B903A90399021
:106DB80038900AA8B821FDF701FC3D98006847F211
:106DC8000001C5F20021884267D100200B904FF4E2
:106DD80080310A911E900AA8FAF700FD08B10EF05A
:106DE800F1F844F2D440C5F60200016841F480315C
:106DF8000160006800F480300990099844F2E0408E
:106E0800C5F60200016841F004010160006800F065
:106E180004000890089844F2E040C5F602000168B2
:106E280041F008010160006800F008000790079829
:106E38004FF4F850389002200190399000200590C6
:106E48003A90032002903B900C2003903C9040F62F
:106E58000000C5F6020038A9049102F07EFADDF8B8
:106E680004C0029A03980499059B4FF0040ECDF8CC
:106E7800E0E0CDF8E4C03A933B923C9040F6004005
:106E8800C5F6020002F069FA059A3120069011460B
:0E6E980000F0F9FB06980EF06DFA3EB080BDDA
:106EA60080B582B001900198006847F20001C5F2F2
:106EB6000021884219D144F2D441C5F6020108687E
:106EC60020F48030086040F60000C5F602004FF45A
:106ED600F85102F00CFD40F60040C5F60200042110
:0E6EE60002F005FD31200EF072FA02B080BD00
:106EF40080B582B047F6D440C2F20040009043F21D
:106F04000041C4F2010101604FF4800141604FF47B
:106F1400C02181600821C1600021019101614161AA
:106F24004FF0005282614FF08052C26101624162AF
:106F34008162C1624FF0804242638163C163016434
:106F440041648164C16401654165816505F070FB3C
:0A6F540008B10EF039F802B080BD5C
:106F5E0080B590B00E900E980F280FD80E9937204E
:106F6E000090002200F08CFB00980EF000FA0E98B4
:106F7E0048F64021C2F20041086003E001208DF87E
:106F8E003F0048E044F2E840C5F60200016841F0D7
:106F9E0020010160006800F020000190019806A811
:106FAE0002A910F012FB0B980490049818B903F084
:106FBE00CFFF059003E003F0CBFF4000059005984E
:106FCE004DF68361C4F21B31A0FB01014FF0FF307F
:106FDE0000EB9140039048F28C00C2F2004041F267
:106FEE000041C4F20001016040F2E731C160039933
:106FFE00416000210161816005F0A2FE40B948F2B6
:10700E008C00C2F2004011F052F98DF83F0002E000
:0E701E0001208DF83F009DF83F0010B080BDAE
:02702C00FEE77D
:10702E0080B582B00190ADF802100198006844F668
:10703E000001C4F20001884203D1BDF80200FFF73F
:06704E00E3FA02B080BD70
:1070540080B582B001900198006840F20041C4F20A
:0E7064000101884201D10DF0CDFE02B080BDC9
:107072004EF68851CEF20001086840F470000860B4
:1070820042F20000C5F20020006800F00F0006285E
:1070920008D842F20001C5F200210868072262F313
:1070A2000300086044F20041C5F60201086840F09E
:1070B2000100086044F21042C5F60202002010608E
:1070C20008684EF67F52CEF6F6221040086042F271
:1070D2000000C5F20020006800F00F00082808D365
:1070E20042F20001C5F200210868072262F30300A0
:1070F200086044F21841C5F602010020086044F21B
:107102001C41C5F60201086044F22041C5F60201A5
:10711200086044F22842C5F6020240F20021C0F2A1
:107122000221116044F22C42C5F602020021C0F293
:10713200FF11116044F23042C5F6020240F2802192
:10714200C0F20111116044F23442C5F6020210602D
:1071520044F23842C5F60202116044F23C42C5F6DE
:107162000202106044F24042C5F60202116044F28B
:107172004441C5F60201086044F20042C5F602022B
:10718200116821F48021116044F26041C5F60201C8
:10719200086044F20001C5F2002143F2D200086007
:0271A200704734
:1071A40080B590B0002101910F910E910D910C9139
:1071B4000B910A9109910891079106910591049107
:1071C4000391029148F2D800C2F2004040F200421A
:1071D400C4F2000202600322426081604FF47A72BA
:1071E400C26001618021816105F0AFFD08B10DF03D
:1071F400EBFE4FF480500C9048F2D800C2F20040ED
:107204000CA907F0D0F808B10DF0DEFE48F2D80062
:10721400C2F2004005F0B3FF08B10DF0D5FE002026
:1072240009900B9048F2D800C2F2004009A911F06D
:107234001FFE08B10DF0C8FE60200290C820039024
:10724400022004900020069048F2D800C2F20040C8
:1072540002A90422FCF72CFB08B10DF0B5FE48F29C
:0E726400D800C2F2004000F002F810B080BD69
:1072720080B588B007900020069005900490039096
:1072820002900798006840F20041C4F2000188426F
:107292001BD144F2E040C5F60200016841F004014E
:1072A2000160006800F004000190019880200290C3
:1072B20002200390002104910591069040F60000FF
:0E72C200C5F6020002A902F04BF808B080BD2C
:1072D00080B58CB00B9000200A9009900890079020
:1072E00006900B98006840F20041C4F20001884209
:1072F00016D144F2E840C5F60200016841F00201EF
:107300000160006800F00200059005981D200290C1
:107310000022114600F0BBF902980EF02FF83CE075
:107320000B98006840F20041C4F20101884234D158
:1073300044F2F040C5F60200016841F0020101602C
:10734000006800F002000490049844F2E040C5F6A2
:107350000200016841F004010160006800F00400CF
:107360000390039840200690022007900120089087
:1073700000200090099003200A9040F60000C5F616
:10738000020006A901F0EDFF009A2E2001900F21C6
:0E73900000F07DF901980DF0F1FF0CB080BD0A
:10739E0080B582B047F64040C2F20040019044F6FC
:1073AE000001C4F2000101604FF4E131416000219F
:1073BE008160C16001610C2242618161C161016223
:1073CE004162282181624FF4004181634FF40051E4
:1073DE00016408F0DFF808B10DF0F1FD47F640400A
:1073EE00C2F20040002109F0AFF908B10DF0E7FD3F
:1073FE0047F64040C2F20040002109F064FA08B19D
:10740E000DF0DDFD47F64040C2F2004009F003F9F1
:0A741E0008B10DF0D4FD02B080BDEE
:1074280080B5BAB0399000203890379036903590B2
:10743800349006A8B821FDF7C1F83998006844F6D9
:107448000001C4F20001884240F0978000210791B2
:107458000220069019221092C82211921290082236
:107468001392149015914FF400721692179123906D
:1074780006A8FAF7B3F908B10DF0A4FD44F2E84004
:10748800C5F60200016841F480210160006800F43B
:1074980080200590059844F2E040C5F60200016896
:1074A80041F008010160006800F0080004900498A9
:1074B8004FF4D85034900220359000200290369036
:1074C80037900720389040F60040C5F6020034A9EE
:1074D80001F043FF029947F65070C2F20040039052
:1074E8002822C4F2020202602D2242608160C1603B
:1074F8004FF48062026141618161C1610162416250
:1075080000F01EF908B10DF05DFD399847F650718D
:10751800C2F20041C0F880103998886347F6D860F5
:10752800C2F2004001904021C4F2020101602E2104
:107538004160402181600021C1604FF48062026196
:1075480041618161C1614FF400320262416200F021
:10755800F7F808B10DF036FD399847F6D861C2F250
:107568000041C1673998886327200090002211469E
:0E75780000F089F800980DF0FDFE3AB080BDDD
:1075860080B582B0032000F060F8F9F7B0FF44F24E
:107596001842C5F602021168C1F303234DF6922183
:1075A600C0F60101CB5C03F01F03D84000900098A1
:1075B600126802F00F02895C01F01F01C84048F60C
:1075C6005421C2F200410860009848F65821C2F2E0
:1075D600004108600F20FFF7BFFC18B101208DF8AD
:1075E600070004E00DF09BFD00208DF807009DF8D4
:0675F600070002B080BD99
:1075FC0048F6BA20C2F20040027848F27021C2F27A
:0A760C000041086810440860704750
:1076160080B584B003900DF050FE0290039801905F
:107626000198013038B148F6BA20C2F2004001781C
:107636000198084401900DF040FE0299401A019904
:0A764600884200D2F7E704B080BDCF
:1076500080B582B00190019807280BD001980628C8
:1076600008D00198052805D00198042802D0019877
:10767000032800D106E04DF25650C0F601009121DA
:0E768000FFF749FB01980DF021FE02B080BD1E
:10768E0080B586B0ADF816000491039203980F28CA
:10769E0000D806E04DF25650C0F60100A921FFF7C2
:1076AE0033FB04980F2800D806E04DF25650C0F672
:1076BE000100AA21FFF728FB0DF01FFE0290BDF975
:1076CE001600019002980499039A0DF01EFE0146D1
:0A76DE00019800F002F806B080BD2C
:1076E80082B0ADF806000091BDF90600002809D463
:1076F80000980001BDF906104EF20042CEF20002D9
:1077080088540AE000980001BDF8061001F00F0146
:0E7718004EF61452CEF20002885402B07047B2
:10772600BFF35F8F4EF62451CEF20001086820F4B5
:10773600803008604EF69451CEF2000100200860B9
:0277460070478A
:1077480010B58EB00C900DF0B7FD0A900C9820B9CA
:1077580001208DF8370000F0F6BD0C980068102164
:10776800C4F20201884200F0B8800C980068282111
:10777800C4F20201884200F0B0800C9800684021F1
:10778800C4F20201884200F0A8800C9800685821D1
:10779800C4F20201884200F0A0800C9800687021B1
:1077A800C4F20201884200F098800C980068882191
:1077B800C4F20201884200F090800C980068A02171
:1077C800C4F20201884200F088800C980068B82151
:1077D800C4F20201884200F080800C98006840F2F0
:1077E8001041C4F20201884277D00C98006840F238
:1077F8002841C4F2020188426FD00C98006840F218
:107808004041C4F20201884267D00C98006840F2F7
:107818005841C4F2020188425FD00C98006840F2D7
:107828007041C4F20201884257D00C98006840F2B7
:107838008841C4F2020188424FD00C98006840F297
:10784800A041C4F20201884247D00C98006840F277
:10785800B841C4F2020188423FD00C98006845F252
:107868000841C5F60201884237D00C98006845F2F5
:107878001C41C5F6020188422FD00C98006845F2D9
:107888003041C5F60201884227D00C98006845F2BD
:107898004441C5F6020188421FD00C98006845F2A1
:1078A8005841C5F60201884217D00C98006845F285
:1078B8006C41C5F6020188420FD00C98006845F269
:1078C8008041C5F60201884207D00C98006845F24D
:1078D8009441C5F60201884200D106E04DF2C1008C
:1078E800C0F60100E621FFF712FA0C98806838B15B
:1078F8000C988068402803D00C988068802800D1B4
:1079080006E04DF2C100C0F60100E721FFF7FFF9DC
:107918000C98C068B0F5007F02D00C98C06800B918
:1079280006E04DF2C100C0F60100E821FFF7EFF9CB
:107938000C980069B0F5806F02D00C98006900B906
:1079480006E04DF2C100C0F60100E921FFF7DFF9BA
:107958000C98406948B10C984069B0F5006F04D0A4
:107968000C984069B0F5805F00D106E04DF2C10087
:10797800C0F60100EA21FFF7CAF90C98806948B1FE
:107988000C988069B0F5005F04D00C988069B0F558
:10799800804F00D106E04DF2C100C0F60100EB2196
:1079A800FFF7B5F90C98C06990B10C98C069B0F5AB
:1079B800807F0DD00C98C069202809D00C98C06928
:1079C800B0F5802F04D00C98C069B0F5402F00D1D5
:1079D80006E04DF2C100C0F60100EC21FFF797F96F
:1079E8000C98006A70B10C98006AB0F5803F09D015
:1079F8000C98006AB0F5003F04D00C98006AB0F506
:107A0800403F00D106E04DF2C100C0F60100ED2173
:107A1800FFF77DF90C98016801201022C4F20202D8
:107A28009142079000F091800C980168012028226B
:107A3800C4F202029142079000F087800C98016816
:107A480001204022C4F20202914207907DD00C9896
:107A5800016801205822C4F202029142079074D0B2
:107A68000C98016801207022C4F20202914207902A
:107A78006BD00C98016801208822C4F2020291425E
:107A8800079062D00C9801680120A022C4F202027B
:107A98009142079059D00C9801680120B822C4F28D
:107AA80002029142079050D00C980168012040F2E0
:107AB8001042C4F202029142079046D00C98016825
:107AC800012040F22842C4F20202914207903CD0C1
:107AD8000C980168012040F24042C4F2020291422F
:107AE800079032D00C980168012040F25842C4F245
:107AF80002029142079028D00C980168012040F2B8
:107B08007042C4F20202914207901ED00C9801689C
:107B1800012040F28842C4F202029142079014D038
:107B28000C980168012040F2A042C4F2020291427E
:107B380007900AD00C9800684FF64831CBF6FD71D3
:107B48000844B0FA80F0400907900798C007002859
:107B580000F0B1810C984068892800D806E04DF201
:107B6800C100C0F60100F121FFF7D1F80C98406A76
:107B780018B10C98406A042800D106E04DF2C10003
:107B8800C0F60100F221FFF7C2F80C98406A0028FD
:107B98004AD00C98806A58B10C98806A012807D09E
:107BA8000C98806A022803D00C98806A032800D1B8
:107BB80006E04DF2C100C0F60100F721FFF7A7F873
:107BC8000C98C06A70B10C98C06AB0F5000F09D063
:107BD8000C98C06AB0F1807F04D00C98C06AB0F1EC
:107BE800C07F00D106E04DF2C100C0F60100F821C7
:107BF800FFF78DF80C98006B70B10C98006BB0F51E
:107C0800001F09D00C98006BB0F5800F04D00C98B9
:107C1800006BB0F5C00F00D106E04DF2C100C0F610
:107C28000100F921FFF773F80C99022081F835005B
:107C38000C99002081F834000C9800681021C4F2D7
:107C48000201884270D00C9800682821C4F2020111
:107C5800884269D00C9800684021C4F20201884229
:107C680062D00C9800685821C4F2020188425BD0A7
:107C78000C9800687021C4F20201884254D00C9814
:107C880000688821C4F2020188424DD00C9800682F
:107C9800A021C4F20201884246D00C980068B8219D
:107CA800C4F2020188423FD00C98006840F21041AB
:107CB800C4F20201884237D00C98006840F228418B
:107CC800C4F2020188422FD00C98006840F240416B
:107CD800C4F20201884227D00C98006840F258414B
:107CE800C4F2020188421FD00C98006840F270412B
:107CF800C4F20201884217D00C98006840F288410B
:107D0800C4F2020188420FD00C98006840F2A041EA
:107D1800C4F20201884207D00C98006840F2B841CA
:107D2800C4F20201884206D10C980168086820F064
:107D38000100086005E00C980168086820F001005F
:107D480008600C9800680068C00788B10DF0B4FAA4
:107D58000A99401A06280AD30C99202048650C99DC
:107D6800032081F8350001208DF83700EBE2E8E7C1
:107D78000C98006800680B900B9848F23F01CFF60A
:107D8800106108400B900C998868D1F80CC00B69F9
:107D98004A6940EA0C00184310438A691043CA69CB
:107DA8001043096A01430B9808430B900C98406AEA
:107DB800042806D10C99C86A096B01430B9808433B
:107DC8000B900C984068292805D30C98416801202D
:107DD8002F2906902CD30C9840683F2805D30C987F
:107DE800416801204329069022D30C98406847280F
:107DF80005D30C98416801204929069018D30C989E
:107E080040684F2805D30C984168012053290690F3
:107E18000ED30C98416800207429059006D30C985D
:107E280041680020782938BF012005900598069000
:107E38000698C00718B10B9840F480100B900B9867
:107E48000C99096808600C98006840690B900B98B9
:107E580020F007000B900C98416A0B9808430B9090
:107E68000C98406A042815D10C98816A0B9808432D
:107E78000B900C98C06A68B10C98F9F7D1FA48B120
:107E88000C99402048650C99012081F835008DF83F
:107E9800370058E20B980C99096848610C9800F073
:107EA80056FA09900C98C06D00F01F013F208840D9
:107EB800099988601BE10C980168012045F2084285
:107EC800C5F602029142049046D00C980168012040
:107ED80045F21C42C5F60202914204903CD00C982F
:107EE8000168012045F23042C5F602029142049031
:107EF80032D00C980168012045F24442C5F60202CE
:107F08009142049028D00C980168012045F258420B
:107F1800C5F60202914204901ED00C980168012017
:107F280045F26C42C5F602029142049014D00C98B6
:107F38000168012045F28042C5F602029142049090
:107F48000AD00C9800684AF66C31CAF2FD710844F0
:107F5800B0FA80F0400904900498C007002800F0A7
:107F6800BB800C980168012045F20842C5F6020260
:107F78009142039046D00C980168012045F21C42BA
:107F8800C5F60202914203903CD00C98016801208A
:107F980045F23042C5F602029142039032D00C9865
:107FA8000168012045F24442C5F60202914203905D
:107FB80028D00C980168012045F25842C5F6020203
:107FC800914203901ED00C980168012045F26C4242
:107FD800C5F602029142039014D00C980168012062
:107FE80045F28042C5F60202914203900AD00C98ED
:107FF80000684AF66C31CAF2FD710844B0FA80F0A4
:10800800400903900398C00760B10C984068112894
:1080180000D807E04DF2C100C0F6010040F26B1134
:10802800FEF775FE0C99022081F835000C990020A6
:1080380081F834000C98006800680B900B986FF377
:1080480010100B900C988068402802D110200290E4
:1080580007E00C9880688038B0FA80F04009800307
:10806800029002980C99CA680B69D1F814C0D1F82B
:1080780018E0CC694EEA040E4CEA0E0C43EA0C03F5
:108088001A4340EAD200096A40EA11110B980843E2
:108098000B900B980C99096808600C9908684AF6C7
:1080A800F832CAF2FD7210444CF6CD42CCF6CC42FE
:1080B800A0FB02026FF0030000EA9200C8650C986A
:1080C80000F045F908900C98C06D00F01F010120E0
:1080D8008840089948600AE00C99402048650C9946
:1080E800032081F8350001208DF837002BE10C982A
:1080F800016801201022C4F202029142019000F0AE
:10810800EA800C98016801202822C4F202029142F8
:10811800019000F0E0800C98016801204022C4F230
:1081280002029142019000F0D6800C98016801206B
:108138005822C4F202029142019000F0CC800C98BF
:10814800016801207022C4F202029142019000F0FD
:10815800C2800C98016801208822C4F20202914270
:10816800019000F0B8800C9801680120A022C4F2A8
:1081780002029142019000F0AE800C980168012043
:10818800B822C4F202029142019000F0A4800C9837
:108198000168012040F21042C4F2020291420190AB
:1081A80000F099800C980168012040F22842C4F23E
:1081B80002029142019000F08E800C980168012023
:1081C80040F24042C4F202029142019000F08380E2
:1081D8000C980168012040F25842C4F20202914210
:1081E800019078D00C980168012040F27042C4F2E6
:1081F8000202914201906ED00C980168012040F271
:108208008842C4F202029142019064D00C9801683D
:10821800012040F2A042C4F20202914201905AD0D9
:108228000C980168012040F2B842C4F2020291425F
:10823800019050D00C980168012045F20842C5F61B
:1082480002029142019046D00C980168012045F243
:108258001C42C5F60202914201903CD00C9801687C
:10826800012045F23042C5F602029142019032D017
:108278000C980168012045F24442C5F60202914279
:10828800019028D00C980168012045F25842C5F6A3
:108298000202914201901ED00C980168012045F21B
:1082A8006C42C5F602029142019014D00C98016804
:1082B800012045F28042C5F60202914201900AD09F
:1082C8000C9800684AF66C31CAF2FD710844B0FA9D
:1082D80080F0400901900198C00758B30C9800F04D
:1082E80005F90C988068802802D10C990020486014
:1082F8000C990879096E08600C98416E806E486088
:108308000C98406878B10C98406808280BD80C98ED
:108318000DF036FA0C98C16E002008600C98016FB9
:10832800406F486006E00C990020C8660C99086701
:108338000C9948670C99002048650C9A012182F82D
:0E83480035108DF837009DF837000EB010BDCF
:1083560083B002900298016801201022C4F2020242
:108366009142009000F09180029801680120282235
:10837600C4F202029142009000F0878002980168E0
:1083860001204022C4F20202914200907DD0029860
:10839600016801205822C4F202029142009074D072
:1083A6000298016801207022C4F2020291420090F4
:1083B6006BD00298016801208822C4F20202914221
:1083C600009062D0029801680120A022C4F2020245
:1083D6009142009059D0029801680120B822C4F257
:1083E60002029142009050D002980168012040F2AA
:1083F6001042C4F202029142009046D002980168EF
:10840600012040F22842C4F20202914200903CD080
:1084160002980168012040F24042C4F202029142F1
:10842600009032D002980168012040F25842C4F20E
:1084360002029142009028D002980168012040F281
:108446007042C4F20202914200901ED00298016866
:10845600012040F28842C4F202029142009014D0F8
:1084660002980168012040F2A042C4F20202914241
:1084760000900AD0029800684FF64831CBF6FD719D
:108486000844B0FA80F0400900900098C00728B36D
:108496000298007810384AF6AB21CAF6AA21A0FB4A
:1084A600011000090190019800F007014DF6222005
:1084B600C0F60100405C0299C8650198042806D3FD
:1084C60002990868042262F30900886505E00299AA
:1084D600086840F2FF329043886504E00299086814
:0E84E60020F0FF0088650298806D03B070479B
:1084F40084B00390039800680190039801680120F8
:1085040045F20842C5F602029142009046D0039813
:108514000168012045F21C42C5F602029142009016
:108524003CD003980168012045F23042C5F60202AE
:108534009142009032D003980168012045F24442F0
:10854400C5F602029142009028D0039801680120E8
:1085540045F25842C5F60202914200901ED003989B
:108564000168012045F26C42C5F602029142009076
:1085740014D003980168012045F28042C5F6020236
:10858400914200900AD0039800684AF66C31CAF20E
:10859400FD710844B0FA80F0400900900098C007CB
:1085A40008B30398007808384CF6CD41CCF6CC419A
:1085B400A0FB011000090290029945F60000C5F6DF
:1085C400020000EB810003990866039945F68000D8
:1085D400C5F602004866029800F01F010120884099
:1085E4000399886631E00398007810384AF6AB2185
:1085F400CAF6AA21A0FB011000090290019840F2DA
:10860400B841C4F20201884209D8019840F21041ED
:10861400C4F20201884202D30298083002900299FF
:1086240040F60000C4F2020000EB810003990866E2
:10863400039940F68000C4F202004866029800F0F4
:0E8644001F01012088400399886604B070472A
:1086520089B008900791069205930898806D04905E
:108662000898806D03900898016801201022C4F2D6
:1086720002029142029000F0EA800898016801200B
:108682002822C4F202029142029000F0E08008988F
:10869200016801204022C4F202029142029000F0DD
:1086A200D6800898016801205822C4F20202914241
:1086B200029000F0CC800898016801207022C4F278
:1086C20002029142029000F0C280089801680120E3
:1086D2008822C4F202029142029000F0B880089807
:1086E20001680120A022C4F202029142029000F02D
:1086F200AE80089801680120B822C4F202029142B9
:10870200029000F0A48008980168012040F2104213
:10871200C4F202029142029000F099800898016826
:10872200012040F22842C4F202029142029000F07B
:108732008E8008980168012040F24042C4F2020291
:108742009142029000F0838008980168012040F273
:108752005842C4F202029142029078D0089801680D
:10876200012040F27042C4F20202914202906ED0A5
:1087720008980168012040F28842C4F20202914244
:10878200029064D008980168012040F2A042C4F22D
:108792000202914202905AD008980168012040F2E8
:1087A200B842C4F202029142029050D00898016885
:1087B200012045F20842C5F602029142029046D0DB
:1087C20008980168012045F21C42C5F60202914256
:1087D20002903CD008980168012045F23042C5F66B
:1087E20002029142029032D008980168012045F2BB
:1087F2004442C5F602029142029028D008980168CC
:10880200012045F25842C5F60202914202901ED062
:1088120008980168012045F26C42C5F602029142B5
:10882200029014D008980168012045F28042C5F6F2
:108832000202914202900AD0089800684AF66C310E
:10884200CAF2FD710844B0FA80F040090290029821
:10885200C00750B10898416E806E48600898C06E9B
:1088620018B10898016F406F4860089801680120AC
:108872001022C4F202029142019000F09180089805
:10888200016801202822C4F202029142019000F004
:1088920087800898016801204022C4F202029142B6
:1088A20001907DD00898016801205822C4F202028A
:1088B2009142019074D00898016801207022C4F29C
:1088C2000202914201906BD008980168012088222F
:1088D200C4F202029142019062D00898016801201C
:1088E200A022C4F202029142019059D00898016874
:1088F2000120B822C4F202029142019050D008989D
:108902000168012040F21042C4F202029142019039
:1089120046D008980168012040F22842C4F20202BF
:10892200914201903CD008980168012040F24042F7
:10893200C4F202029142019032D0089801680120EB
:1089420040F25842C4F202029142019028D00898A3
:108952000168012040F27042C4F202029142019089
:108962001ED008980168012040F28842C4F2020237
:108972009142019014D008980168012040F2A0426F
:10898200C4F20202914201900AD0089800684FF6A0
:108992004831CBF6FD710844B0FA80F040090190ED
:1089A2000198C00738B30898C06D00F01F013F203E
:1089B20088400499886008980168086820F480203B
:1089C20008600598089909684860089880684028F6
:1089D20008D1069808990968886007980899096873
:1089E200C86007E00798089909688860069808999E
:1089F2000968C86075E008980168012045F20842DC
:108A0200C5F602029142009046D008980168012002
:108A120045F21C42C5F60202914200903CD00898F1
:108A22000168012045F23042C5F6020291420090EF
:108A320032D008980168012045F24442C5F602028C
:108A42009142009028D008980168012045F25842CE
:108A5200C5F60202914200901ED0089801680120DA
:108A620045F26C42C5F602029142009014D0089879
:108A72000168012045F28042C5F60202914200904F
:108A82000AD0089800684AF66C31CAF2FD710844AF
:108A9200B0FA80F0400900900098C00708B3089827
:108AA200C06D00F01F0101208840039948600598BD
:108AB20008990968486008988068402808D1069893
:108AC200089909688860079808990968C86007E0EA
:108AD2000798089909688860069808990968C86023
:068AE200FFE709B0704738
:108AE80080B58AB008900CF0E7FB0490089820B98C
:108AF80001208DF8270000F02CBC089890F835006C
:108B080002280BD00899802048650899002081F830
:108B1800340001208DF8270000F01BBC089801687C
:108B280001201022C4F202029142039000F09180C9
:108B38000898016801202822C4F202029142039099
:108B480000F087800898016801204022C4F20202E0
:108B5800914203907DD00898016801205822C4F200
:108B680002029142039074D0089801680120702293
:108B7800C4F20202914203906BD008980168012068
:108B88008822C4F202029142039062D008980168D8
:108B98000120A022C4F202029142039059D0089801
:108BA80001680120B822C4F202029142039050D019
:108BB80008980168012040F21042C4F20202914272
:108BC800039046D008980168012040F22842C4F278
:108BD8000202914203903CD008980168012040F2BB
:108BE8004042C4F202029142039032D008980168D0
:108BF800012040F25842C4F202029142039028D068
:108C080008980168012040F27042C4F202029142C1
:108C180003901ED008980168012040F28842C4F2EF
:108C280002029142039014D008980168012040F292
:108C3800A042C4F20202914203900AD00898006848
:108C48004FF64831CBF6FD710844B0FA80F0400980
:108C580003900398C00778B108980168086820F065
:108C68001E00086008980168486920F08000486183
:108C780008980068059008E008980168086820F0DE
:108C88000E0008600898006805900898016801209F
:108C98001022C4F202029142029000F0EA80089881
:108CA800016801202822C4F202029142029000F0D9
:108CB800E0800898016801204022C4F20202914233
:108CC800029000F0D6800898016801205822C4F26A
:108CD80002029142029000F0CC80089801680120BD
:108CE8007022C4F202029142029000F0C2800898F9
:108CF800016801208822C4F202029142029000F029
:108D0800B880089801680120A022C4F202029142AA
:108D1800029000F0AE80089801680120B822C4F2E1
:108D280002029142029000F0A48008980168012094
:108D380040F21042C4F202029142029000F099807F
:108D480008980168012040F22842C4F202029142C8
:108D5800029000F08E8008980168012040F240429D
:108D6800C4F202029142029000F0838008980168E0
:108D7800012040F25842C4F202029142029078D097
:108D880008980168012040F27042C4F20202914240
:108D980002906ED008980168012040F28842C4F21F
:108DA80002029142029064D008980168012040F2C2
:108DB800A042C4F20202914202905AD00898016877
:108DC800012040F2B842C4F202029142029050D00F
:108DD80008980168012045F20842C5F6020291424E
:108DE800029046D008980168012045F21C42C5F659
:108DF8000202914202903CD008980168012045F295
:108E08003042C5F602029142029032D008980168B9
:108E1800012045F24442C5F602029142029028D050
:108E280008980168012045F25842C5F602029142AD
:108E380002901ED008980168012045F26C42C5F6E0
:108E480002029142029014D008980168012045F26C
:108E58008042C5F60202914202900AD00898006842
:108E68004AF66C31CAF2FD710844B0FA80F0400944
:108E780002900298C00728B10898016E086820F48B
:108E880080700860089800681021C4F202018842C6
:108E980070D0089800682821C4F20201884269D07D
:108EA800089800684021C4F20201884262D00898FC
:108EB80000685821C4F2020188425BD00898006813
:108EC8007021C4F20201884254D0089800688821B1
:108ED800C4F2020188424DD008980068A021C4F26B
:108EE8000201884246D008980068B821C4F20201FD
:108EF80088423FD00898006840F21041C4F202014D
:108F0800884237D00898006840F22841C4F202012C
:108F180088422FD00898006840F24041C4F202010C
:108F2800884227D00898006840F25841C4F20201EC
:108F380088421FD00898006840F27041C4F20201CC
:108F4800884217D00898006840F28841C4F20201AC
:108F580088420FD00898006840F2A041C4F202018C
:108F6800884207D00898006840F2B841C4F202016C
:108F7800884206D108980168086820F00100086056
:108F880005E008980168086820F001000860059865
:108F98000068C007A8B10CF08FF90499401A062898
:108FA8000ED30899202048650899032081F83500D8
:108FB8000899002081F8340001208DF82700C8E1C5
:108FC800E5E70898016801201022C4F202029142E4
:108FD800019000F091800898016801202822C4F2CD
:108FE80002029142019000F08780089801680120F0
:108FF8004022C4F20202914201907DD00898016893
:1090080001205822C4F202029142019074D00898BB
:10901800016801207022C4F20202914201906BD0D3
:109028000898016801208822C4F202029142019046
:1090380062D0089801680120A022C4F2020291427D
:10904800019059D0089801680120B822C4F20202A0
:109058009142019050D008980168012040F21042D6
:10906800C4F202029142019046D00898016801209A
:1090780040F22842C4F20202914201903CD0089882
:109088000168012040F24042C4F20202914201907C
:1090980032D008980168012040F25842C4F2020216
:1090A8009142019028D008980168012040F270424E
:1090B800C4F20202914201901ED008980168012072
:1090C80040F28842C4F202029142019014D00898FA
:1090D8000168012040F2A042C4F2020291420190CC
:1090E8000AD0089800684FF64831CBF6FD7108445D
:1090F800B0FA80F0400901900198C00758B108986B
:10910800806D07900898C06D00F01F013F208840CF
:10911800079988600AE00898806D06900898C06DE5
:1091280000F01F01012088400699486008980168EE
:1091380001201022C4F202029142009000F0EA805D
:109148000898016801202822C4F202029142009086
:1091580000F0E0800898016801204022C4F2020271
:109168009142009000F0D6800898016801205822AA
:10917800C4F202029142009000F0CC800898016885
:1091880001207022C4F202029142009000F0C280D5
:109198000898016801208822C4F2020291420090D6
:1091A80000F0B880089801680120A022C4F20202E9
:1091B8009142009000F0AE80089801680120B82222
:1091C800C4F202029142009000F0A480089801685D
:1091D800012040F21042C4F202029142009000F0D5
:1091E800998008980168012040F22842C4F20202DE
:1091F8009142009000F08E8008980168012040F2AA
:109208004042C4F202029142009000F08380089824
:109218000168012040F25842C4F2020291420090D3
:1092280078D008980168012040F27042C4F2020226
:10923800914200906ED008980168012040F288425F
:10924800C4F202029142009064D00898016801209B
:1092580040F2A042C4F20202914200905AD008980B
:109268000168012040F2B842C4F202029142009023
:1092780050D008980168012045F20842C5F602025C
:109288009142009046D008980168012045F21C429E
:10929800C5F60202914200903CD00898016801206E
:1092A80045F23042C5F602029142009032D0089849
:1092B8000168012045F24442C5F60202914200903D
:1092C80028D008980168012045F25842C5F60202E4
:1092D800914200901ED008980168012045F26C4226
:1092E800C5F602029142009014D008980168012046
:1092F80045F28042C5F60202914200900AD00898D1
:1093080000684AF66C31CAF2FD710844B0FA80F080
:10931800400900900098C00780B10898416E806E9F
:1093280048600898C06E48B10898C16E086820F473
:10933800807008600898016F406F486008990120A4
:1093480081F835000899002081F8340000208DF854
:0A93580027009DF827000AB080BD31
:1093620080B590B00F900E9100200D908020C5F630
:1093720000000A900F980021C5F6020188423ED0F3
:109382000F9840F20041C5F60201884237D00F988B
:1093920040F60001C5F60201884230D00F9840F62F
:1093A2000041C5F60201884229D00F9841F200011E
:1093B200C5F60201884222D00F9841F20041C5F65B
:1093C200020188421BD00F9841F60001C5F6020146
:1093D200884214D00F9841F60041C5F60201884236
:1093E2000DD00F9842F20041C5F60201884206D024
:1093F2000F9842F60001C5F60201884200D106E04C
:109402004DF62A20C0F60100B321FDF783FC0E9829
:10941200008818B10E98408800B906E04DF62A205F
:10942200C0F60100B421FDF775FC0E98406888B3C0
:109432000E98406801282DD00E984068112829D036
:109442000E984068022825D00E984068122821D034
:109452000E984068B0F5881F1CD00E984068B0F591
:10946200041F17D00E984068B0F5441F12D00E9812
:109472004068B0F5901F0DD00E984068B0F5081FF7
:1094820008D00E984068B0F5481F03D00E98406887
:10949200032800D106E04DF62A20C0F60100B521CE
:1094A200FDF738FC0E9800680D99C840002800F0BE
:1094B2001E820E9800680D9A0121914008400C907E
:1094C2000C98002800F00F820E98406800F003000C
:1094D200012805D00E98406800F00300022844D10C
:1094E2000E98C06858B10E98C068012807D00E982F
:1094F200C068022803D00E98C068032800D106E095
:109502004DF62A20C0F60100C421FDF703FC0F9896
:1095120080680B900D984100032000FA01F10B982E
:1095220088430B900E98C0680D99490000FA01F12A
:109532000B9808430B900B980F9988600F9840681E
:109542000B900D99012000FA01F10B9888430B90C2
:109552000E984068C0F300100D9900FA01F10B98C3
:1095620008430B900B980F9948600E98406800F0E2
:109572000300032829D00E98806838B10E988068BD
:10958200012803D00E988068022800D106E04DF62B
:109592002A20C0F60100D621FDF7BCFB0F98C06857
:1095A2000B900D984100032000FA01F10B988843BB
:1095B2000B900E9880680D99490000FA01F10B9802
:1095C20008430B900B980F99C8600E98406800F002
:1095D200030002287DD10F980021C5F602018842BE
:1095E2003ED00F9840F20041C5F60201884237D0C2
:1095F2000F9840F60001C5F60201884230D00F985C
:1096020040F60041C5F60201884229D00F9841F286
:109612000001C5F60201884222D00F9841F20041B2
:10962200C5F6020188421BD00F9841F60001C5F62B
:109632000201884214D00F9841F60041C5F602019A
:1096420088420DD00F9842F20041C5F602018842CD
:1096520006D00F9842F60001C5F60201884200D1F9
:1096620006E04DF62A20C0F60100E321FDF752FB89
:109672000E9800690F2800D806E04DF62A20C0F6A1
:109682000100E421FDF746FB0F980D996FF00302EC
:1096920002EA51010844006A0B900D9800F007009D
:1096A20081000F2000FA01F10B9888430B900E986D
:1096B20000690D9901F00701890000FA01F10B9888
:1096C20008430B900B980F990D9B02EA5302114429
:1096D20008620F9800680B900D984100032000FA71
:1096E20001F10B9888430B900E98406800F003003C
:1096F2000D99490000FA01F10B9808430B900B9861
:109702000F9908600E9880798007002800F0EB809E
:1097120044F2F440C5F60200016841F00201016022
:10972200006800F00200099009980D9820F00300EB
:1097320040F20841C5F6000140580B900D9800F028
:10974200030081000F2000FA01F10B9888430B906F
:109752000F980021C5F60201884202D1002008902C
:109762005DE00F9840F20041C5F60201884202D145
:109772000120079051E00F9840F60001C5F6020162
:10978200884202D10220069045E00F9840F600413F
:10979200C5F60201884202D10320059039E00F98F4
:1097A20041F20001C5F60201884202D10420049070
:1097B2002DE00F9841F20041C5F60201884202D124
:1097C2000520039021E00F9841F60001C5F6020141
:1097D200884202D10620029015E00F9841F600411E
:1097E200C5F60201884202D10720019009E00F99D3
:1097F20042F20042C5F602020A20914208BF092045
:1098020001900198029002980390039804900498A2
:109812000590059806900698079007980890089872
:109822000D9901F00301890000FA01F10B98084338
:109832000B900B980D9921F0030140F20842C5F6F6
:10984200000288504FF0B04000680B900C990B98C2
:1098520088430B900E988079C006002803D50C9996
:109862000B9808430B900B984FF0B041086004200E
:10987200C5F6000000680B900C990B9888430B907A
:109882000E9880798006002803D50C990B9808431E
:109892000B900B980421C5F6000108600A984068F5
:1098A2000B900C990B9888430B900E988079800747
:1098B200002803D50C990B9808430B900B980A9932
:1098C20048600A9800680B900C990B9888430B909B
:1098D2000E988079C00718B10C990B9808430B9029
:1098E2000B980A9908600D9801300D90DAE510B0D6
:0298F20080BD37
:1098F40080B590B00F900E9100200D908020C5F699
:1099040000000A900F980021C5F6020188423ED05B
:109914000F9840F20041C5F60201884237D00F98F3
:1099240040F60001C5F60201884230D00F9840F697
:109934000041C5F60201884229D00F9841F2000186
:10994400C5F60201884222D00F9841F20041C5F6C3
:10995400020188421BD00F9841F60001C5F60201AE
:10996400884214D00F9841F60041C5F6020188429E
:109974000DD00F9842F20041C5F60201884206D08C
:109984000F9842F60001C5F60201884200D107E0B3
:109994004DF62A20C0F601004FF49E71FDF7B9F987
:1099A400BDF8380018B1BDF83A0000B907E04DF62B
:1099B4002A20C0F6010040F23D11FDF7AAF90E98E5
:1099C4000D99C840002800F0EE800E980D9A0121F0
:1099D400914008400C900C98002800F0E0800D980D
:1099E40020F0030040F20841C5F6000140580B90F6
:1099F4000D9800F0030081000F2000FA01F10B988C
:109A040008400B900B9809900F980021C5F60201AD
:109A1400884202D1002008905DE00F9840F2004196
:109A2400C5F60201884202D10120079051E00F9847
:109A340040F60001C5F60201884202D102200690D8
:109A440045E00F9840F60041C5F60201884202D174
:109A54000320059039E00F9841F20001C5F6020198
:109A6400884202D1042004902DE00F9841F2004175
:109A7400C5F60201884202D10520039021E00F9827
:109A840041F60001C5F60201884202D10620029087
:109A940015E00F9841F60041C5F60201884202D153
:109AA4000720019009E00F9942F20042C5F6020234
:109AB4000A20914208BF092001900198029002985F
:109AC40003900398049004980590059806900698CE
:109AD400079007980890099808990D9A02F00302D4
:109AE40092009140884228D10C9A0A9908689043C0
:109AF40008600C9A0A994868904348600C9A0421BB
:109B0400C5F600010868904308600C9A4FF0B04114
:109B14000868904308600D9800F0030081000F204E
:109B240088400B900B9B0D9820F0030140F20842F3
:109B3400C5F600028858984388500D9841000320C8
:109B440000FA01F30F9A116819431160DDF834C06B
:109B54000CF007018A000F2101FA02F30F996FF04C
:109B6400030202EA5C020A44116A994311620D99E4
:109B7400490000FA01F30F9AD1689943D1600D9A14
:109B8400012101FA02F30F9A5168994351600D992A
:109B9400490000FA01F20F998868904388600D9893
:0A9BA40001300D900BE710B080BDFA
:109BAE0044F60001C5F60201086840F480700860B2
:029BBE007047EE
:109BC00080B58CB00A900A9820B901208DF82F003A
:109BD00000F0C1BD0A98006800B30A980078C00779
:109BE000E0B90A98006800F00200022816D00A982E
:109BF000006800F01000102810D00A98006800F0EB
:109C0000080008280AD00A98006800F00400042818
:109C100004D00A9800788006002800D507E04DF2AD
:109C20002810C0F6010040F2A111FDF774F80A985F
:109C30000078C007002800F0AE800A98406848B15C
:109C40000A984068B0F5803F04D00A984068B0F5A3
:109C5000A02F00D107E04DF22810C0F601004FF40C
:109C6000D371FDF758F844F21040C5F602000068C1
:109C700000F03800069044F22840C5F60200006863
:109C800005900698102807D00698182815D1059831
:109C900000F00300022810D144F20040C5F6020093
:109CA0000068C0F3404038B10A98406820B90120EC
:109CB0008DF82F0000F04FBD6DE00A984068B0F5B8
:109CC000803F08D144F20041C5F60201086840F423
:109CD000803008602DE00A98406860B944F2004185
:109CE000C5F60201086820F480300860086820F496
:109CF000802008601DE00A984068B0F5A02F0CD1C4
:109D000044F20041C5F60201086840F48020086072
:109D1000086840F4803008600BE044F20041C5F66A
:109D20000201086820F480300860086820F4802070
:109D300008600A984068B8B10BF0C2FA099044F282
:109D40000040C5F602000068C0F3404058B90BF06F
:109D5000B7FA0999401A652804D303208DF82F001B
:109D600000F0F9BCEBE716E00BF0AAFA099044F218
:109D70000040C5F602000068C0F3404058B10BF047
:109D80009FFA0999401A652804D303208DF82F0003
:109D900000F0E1BCEBE70A9800788007002840F16A
:109DA000D5800A98C06898B10A98C06801280FD079
:109DB0000A98C06801280BD00A98C068092807D003
:109DC0000A98C068112803D00A98C068192800D1E1
:109DD00007E04DF22810C0F601004FF4ED71FCF7DA
:109DE0009AFF0A9800697F2800D807E04DF22810F2
:109DF000C0F6010040F2DB11FCF78DFF44F2104089
:109E0000C5F60200006800F03800049044F22840D3
:109E1000C5F6020000680390049838B10498182829
:109E200043D19DF80C00800700283ED144F2004049
:109E3000C5F602000068C0F3800038B10A98C06817
:109E400020B901208DF82F0000F085BC44F20041BC
:109E5000C5F60201086820F019000A9AD26810437A
:109E600008600BF02DFA099044F20040C5F602009C
:109E70000068C0F3800058B90BF022FA0999401A23
:109E8000032804D303208DF82F0000F064BCEBE717
:109E900044F20441C5F60201086820F0FE400A9A27
:109EA000126940EA0260086050E00A98C06870B326
:109EB00044F20041C5F60201086820F019000A9A30
:109EC000D268104308600BF0FBF9099044F200409F
:109ED000C5F602000068C0F3800058B90BF0F0F935
:109EE0000999401A032804D303208DF82F0000F0AD
:109EF00032BCEBE744F20441C5F60201086820F0E9
:109F0000FE400A9A126940EA026008601EE044F2CC
:109F10000041C5F60201086820F0010008600BF05E
:109F2000CFF9099044F20040C5F602000068C0F382
:109F3000800058B10BF0C4F90999401A032804D3E2
:109F400003208DF82F0000F006BCEBE70A9800789C
:109F5000C006002840F19F800A98C06918B10A988D
:109F6000C069802800D107E04DF22810C0F601003A
:109F700040F22B21FCF7CFFE0A98006A3F2800D858
:109F800007E04DF22810C0F601004FF40B71FCF70A
:109F9000C2FE44F21040C5F60200006800F038002E
:109FA000029044F22840C5F6020000680190029831
:109FB000082807D00298182821D1019800F0030042
:109FC00001281CD144F20040C5F602000068C0F32D
:109FD000002038B10A98C069802803D001208DF88C
:109FE0002F00B8E344F20C41C5F60201086820F0E6
:109FF0007C500A9A126A40EA026008604BE00A98B4
:10A00000C06950B344F20041C5F60201086840F04F
:10A01000800008600BF054F9099044F20040C5F646
:10A0200002000068C0F3002050B90BF049F909990B
:10A03000401A032803D303208DF82F008BE3ECE7AD
:10A0400044F20C41C5F60201086820F07C500A9ADF
:10A05000126A40EA026008601DE044F20041C5F661
:10A060000201086820F0800008600BF029F90990CF
:10A0700044F20040C5F602000068C0F3002050B171
:10A080000BF01EF90999401A032803D303208DF819
:10A090002F0060E3ECE70A980078000700284FD50E
:10A0A0000A98406918B10A984069012800D107E070
:10A0B0004DF22810C0F6010040F26D21FCF72BFE96
:10A0C0000A984069F0B144F27441C5F6020108688B
:10A0D00040F0010008600BF0F3F8099044F274407E
:10A0E000C5F602000068C0F3400050B90BF0E8F874
:10A0F0000999401A032803D303208DF82F002AE37F
:10A10000ECE71DE044F27441C5F60201086820F056
:10A11000010008600BF0D4F8099044F27440C5F6D1
:10A1200002000068C0F3400050B10BF0C9F8099973
:10A13000401A032803D303208DF82F000BE3ECE72C
:10A140000A980078800600284FD50A98806918B1CF
:10A150000A988069012800D107E04DF22810C0F666
:10A1600001004FF42671FCF7D6FD0A988069F0B122
:10A1700044F20041C5F60201086840F480500860CE
:10A180000BF09EF8099044F20040C5F6020000680A
:10A19000C0F3403050B90BF093F80999401A0328E6
:10A1A00003D303208DF82F00D5E2ECE71DE044F245
:10A1B0000041C5F60201086820F4805008600BF0E9
:10A1C0007FF8099044F20040C5F602000068C0F331
:10A1D000403050B10BF074F80999401A032803D3AA
:10A1E00003208DF82F00B6E2ECE70A9800784007CC
:10A1F000002840F1A0800A98806838B10A988068E9
:10A20000012803D00A988068052800D107E04DF2A4
:10A210002810C0F6010040F2C221FCF77CFD44F694
:10A220000001C5F60201086840F4807008600BF078
:10A2300047F8099044F60000C5F602000068C00522
:10A2400000280AD40BF03CF80999401A652803D37A
:10A2500003208DF82F007EE2ECE70A988068012841
:10A2600008D144F27041C5F60201086840F00100CF
:10A2700008602CE00A98806860B944F27041C5F625
:10A280000201086820F001000860086820F004005E
:10A2900008601CE00A98806805280CD144F27041DF
:10A2A000C5F60201086840F004000860086840F044
:10A2B000010008600BE044F27041C5F60201086835
:10A2C00020F001000860086820F0040008600A9887
:10A2D0008068C0B10AF0F4FF099044F27040C5F6FE
:10A2E00002000068C0F3400060B90AF0E9FF099974
:10A2F000401A41F28931884203D303208DF82F00A0
:10A3000029E2EAE717E00AF0DBFF099044F2704027
:10A31000C5F602000068C0F3400060B10AF0D0FF4B
:10A320000999401A41F28931884203D303208DF8FC
:10A330002F0010E2EAE70A98406A38B10A98406AAA
:10A34000012803D00A98406A022800D107E04DF2A4
:10A350002810C0F601004FF43D71FCF7DCFC0A98B0
:10A36000406A002800F0F48144F21040C5F6020073
:10A37000006800F03800182800F068810A98406AE8
:10A38000022840F044810A98806A01280AD00A987D
:10A39000806A38B10A98806A032803D00A98806AD4
:10A3A000022800D107E04DF22810C0F6010040F26B
:10A3B000FD21FCF7B0FC0A98006C58B10A98006CBB
:10A3C000042807D00A98006C082803D00A98006C6B
:10A3D0000C2800D107E04DF22810C0F6010040F231
:10A3E000FE21FCF798FC0A98406C18B10A98406C62
:10A3F000022800D107E04DF22810C0F6010040F21B
:10A40000FF21FCF788FC0A98C06A20B10A98C06A4C
:10A410003F2800D807E04DF22810C0F601004FF4A5
:10A420004071FCF778FC0A98006B042805D30A9861
:10A43000006BB0F5007F00D807E04DF22810C0F6A1
:10A44000010040F20131FCF766FC0A98406B20B134
:10A450000A98406B802800D807E04DF22810C0F61B
:10A46000010040F20231FCF756FC0A98806B20B1E3
:10A470000A98806B802800D807E04DF22810C0F6BB
:10A48000010040F20331FCF746FC0A98C06B20B192
:10A490000A98C06B802800D807E04DF22810C0F65B
:10A4A00001004FF44171FCF736FC0A98806C400BB8
:10A4B00000B907E04DF22810C0F6010040F2053166
:10A4C000FCF729FC44F20041C5F60201086820F0BF
:10A4D000807008600AF0F4FE099044F20040C5F66E
:10A4E00002000068C0F3406050B10AF0E9FE09992B
:10A4F000401A032803D303208DF82F002BE1ECE74B
:10A5000044F22841C5F60201086840F2F332904354
:10A510000A9B9A6ADB6A42EA0312104308600A99AE
:10A52000086BD1F834C08B6BCA6B01386FF35F20B6
:10A530004FF60061CFF6FF7101EB4C2189B2084460
:10A540000021CFF6FF7101EB034101F4FE01084445
:10A550004FF07F4101EB026101F0FE41084444F2FB
:10A560003041C5F60201086044F22C41C5F60201F3
:10A570000091086820F00100086044F23442C5F6FA
:10A58000020210684FF6F87398430A9B9B6C40EAEE
:10A59000C3001060086820F00C000A9A126C104387
:10A5A0000860086820F002000A9A526C10430860A4
:10A5B000086840F480300860086840F400300860A3
:10A5C000086840F480200860086840F001000860D6
:10A5D00044F20041C5F60201086840F0807008604E
:10A5E0000AF06EFE099044F20040C5F602000068D1
:10A5F000C0F3406050B90AF063FE0999401A03287D
:10A6000003D303208DF82F00A5E0ECE71DE044F212
:10A610000041C5F60201086820F0807008600AF069
:10A620004FFE099044F20040C5F602000068C0F3F6
:10A63000406050B10AF044FE0999401A032803D340
:10A6400003208DF82F0086E0ECE781E044F22840FB
:10A65000C5F602000068089044F23040C5F60200DA
:10A66000006807900A98406A01282DD0089800F0E9
:10A6700003000A99896A884226D10898C0F3051117
:10A680000A98C06A88421FD107986FF35F200A9921
:10A69000096B0139884217D1BDF81C00410A0A989C
:10A6A000406B013888420FD10798C0F306410A98E1
:10A6B000806B0138884207D10798C0F306610A9879
:10A6C000C06B0138884203D001208DF82F0042E092
:10A6D00044F23440C5F60200006880B2C008089019
:10A6E0000A98806C0899884232D00A98806C400B96
:10A6F00000B907E04DF22810C0F601004FF45B717D
:10A70000FCF709FB44F22C41C5F60201086820F071
:10A71000010008600AF0D4FD09900AF0D1FD099902
:10A72000401A00B9F9E744F23441C5F6020108685D
:10A730004FF6F87290430A9A926C40EAC2000860A1
:10A7400044F22C41C5F60201086840F0010008609F
:0EA7500000208DF82F009DF82F000CB080BD6A
:10A75E0080B586B004900391049818B901208DF845
:10A76E001700C6E30498006820B1049800683F28DB
:10A77E0000D807E04DF22810C0F6010040F2A731D4
:10A78E00FCF7C2FA039860B30398012829D0039806
:10A79E00022826D00398032823D00398042820D01B
:10A7AE00039805281DD0039806281AD00398072869
:10A7BE0017D00398082814D00398092811D00398AD
:10A7CE000A280ED003980B280BD003980C2808D01B
:10A7DE0003980D2805D003980E2802D003980F2851
:10A7EE0000D107E04DF22810C0F601004FF46A7157
:10A7FE00FCF78AFA039842F20001C5F200210968BB
:10A80E0001F00F01884213D942F20000C5F2002078
:10A81E00016821F00F01039A11430160006800F0F6
:10A82E000F000399884203D001208DF8170060E3D2
:10A83E00049800784007002831D50498006944F246
:10A84E001841C5F60201096801F07001884226D947
:10A85E000498006978B10498006940280BD00498D8
:10A86E000069502807D004980069602803D0049826
:10A87E000069702800D107E04DF22810C0F60100E3
:10A88E004FF47171FCF740FA44F21841C5F602011B
:10A89E00086820F07000049A12691043086004984A
:10A8AE0000780007002831D50498406944F21C4115
:10A8BE00C5F60201096801F07001884226D9049894
:10A8CE00406978B10498406940280BD004984069DB
:10A8DE00502807D004984069602803D00498406936
:10A8EE00702800D107E04DF22810C0F6010040F2AA
:10A8FE00D631FCF709FA44F21C41C5F6020108688C
:10A90E0020F07000049A5269104308600498007891
:10A91E00C006002835D50498806944F21C41C5F65E
:10A92E000201096801F4E06188422AD9049880691D
:10A93E0098B104988069B0F5806F0ED00498806944
:10A94E00B0F5A06F09D004988069B0F5C06F04D03F
:10A95E0004988069B0F5E06F00D107E04DF2281041
:10A96E00C0F6010040F2E731FCF7CEF944F21C418B
:10A97E00C5F60201086820F4E060049A926910435B
:10A98E000860049800788006002831D50498C069C4
:10A99E0044F22041C5F60201096801F070018842B7
:10A9AE0026D90498C06978B10498C06940280BD0A4
:10A9BE000498C069502807D00498C069602803D055
:10A9CE000498C069702800D107E04DF22810C0F637
:10A9DE00010040F2F931FCF797F944F22041C5F637
:10A9EE000201086820F07000049AD26910430860D2
:10A9FE00049800788007002841D50498C06844F276
:10AA0E001841C5F60201096801F00F01884236D9D6
:10AA1E000498C068F8B10498C06808281BD0049840
:10AA2E00C068092817D00498C0680A2813D0049863
:10AA3E00C0680B280FD00498C0680C280BD004985F
:10AA4E00C0680D2807D00498C0680E2803D004985B
:10AA5E00C0680F2800D107E04DF22810C0F60100A3
:10AA6E0040F20C41FCF750F944F21841C5F60201D0
:10AA7E00086820F00F00049AD2681043086004980A
:10AA8E000078C007002800F0BD800498806838B3B5
:10AA9E0004988068B0F5006F22D004988068B0F5F5
:10AAAE00106F1DD004988068B0F5206F18D00498F0
:10AABE008068B0F5306F13D004988068B0F5406FA1
:10AACE000ED004988068B0F5506F09D00498806855
:10AADE00B0F5606F04D004988068B0F5706F00D147
:10AAEE0007E04DF22810C0F6010040F21C41FCF7C1
:10AAFE000BF90498406801280AD00498406838B1D0
:10AB0E0004984068022803D004984068032800D1B6
:10AB1E0007E04DF22810C0F6010040F21D41FCF78F
:10AB2E00F3F844F21841C5F60201086820F470608B
:10AB3E00049A9268104308600498406802280CD169
:10AB4E0044F20040C5F602000068C0F3404018B958
:10AB5E0001208DF81700CCE12DE004984068032801
:10AB6E000CD144F20040C5F602000068C0F340600C
:10AB7E0018B901208DF81700BBE11CE0049840685D
:10AB8E0001280CD144F20040C5F602000068C0F363
:10AB9E00002018B901208DF81700AAE10BE044F24D
:10ABAE000040C5F602000068C0F3800018B901200D
:10ABBE008DF817009DE144F21041C5F602010868B8
:10ABCE0020F00700049A5268104308600AF071FBE7
:10ABDE00019044F21040C5F60200006800F0380003
:10ABEE0004994968C90088420CD00AF062FB0199A9
:10ABFE00401A41F28931884203D303208DF81700A1
:10AC0E0077E1E6E7049800788007002841D504989C
:10AC1E00C06844F21841C5F60201096801F00F013F
:10AC2E00884236D20498C068F8B10498C0680828E3
:10AC3E001BD00498C068092817D00498C0680A2849
:10AC4E0013D00498C0680B280FD00498C0680C2845
:10AC5E000BD00498C0680D2807D00498C0680E2841
:10AC6E0003D00498C0680F2800D107E04DF22810D9
:10AC7E00C0F6010040F25E41FCF746F844F218417E
:10AC8E00C5F60201086820F00F00049AD26810433E
:10AC9E000860039842F20001C5F20021096801F034
:10ACAE000F01884213D242F20000C5F20020016863
:10ACBE0021F00F01039A11430160006800F00F00AC
:10ACCE000399884203D001208DF8170011E10498F2
:10ACDE0000784007002831D50498006944F21841E5
:10ACEE00C5F60201096801F07001884226D2049867
:10ACFE00006978B10498006940280BD00498006967
:10AD0E00502807D004980069602803D00498006981
:10AD1E00702800D107E04DF22810C0F6010040F275
:10AD2E007F41FBF7F1FF44F21841C5F602010868B6
:10AD3E0020F07000049A126910430860049800789D
:10AD4E000007002831D50498406944F21C41C5F62D
:10AD5E000201096801F07001884226D20498406908
:10AD6E0078B10498406940280BD004984069502867
:10AD7E0007D004984069602803D004984069702871
:10AD8E0000D107E04DF22810C0F6010040F29141CB
:10AD9E00FBF7BAFF44F21C41C5F60201086820F029
:10ADAE007000049A52691043086004980078C00637
:10ADBE00002835D50498806944F21C41C5F602017D
:10ADCE00096801F4E06188422AD20498806998B13A
:10ADDE0004988069B0F5806F0ED004988069B0F544
:10ADEE00A06F09D004988069B0F5C06F04D00498A4
:10ADFE008069B0F5E06F00D107E04DF22810C0F683
:10AE0E00010040F2A341FBF77FFF44F21C41C5F65F
:10AE1E000201086820F4E060049A92691043086009
:10AE2E00049800788006002831D50498C06944F251
:10AE3E002041C5F60201096801F07001884226D250
:10AE4E000498C06978B10498C06940280BD0049862
:10AE5E00C069502807D00498C069602803D00498B0
:10AE6E00C069702800D107E04DF22810C0F601002D
:10AE7E0040F2B541FBF748FF44F22041C5F602010E
:10AE8E00086820F07000049AD26910430860F6F743
:10AE9E002AFB44F21842C5F602021168C1F30323DD
:10AEAE004DF69221C0F60101CB5C03F01F03D84092
:10AEBE0000900098126802F00F02895C01F01F01E9
:10AECE00C84048F65421C2F200410860009848F686
:10AEDE005821C2F20041086048F64020C2F20040FC
:10AEEE000068FCF735F88DF80B009DF80B008DF817
:0AAEFE0017009DF8170006B080BD94
:10AF080080B582B0F6F7F2FA44F21842C5F60202AA
:10AF18001168C1F303234DF69221C0F60101CB5C01
:10AF280003F01F03D84001900198126802F00F0245
:10AF3800895C01F01F0120FA01F148F65420C2F2A1
:10AF480000400160019948F65822C2F2004211609F
:06AF5800006802B080BD9C
:10AF5E0080B5FFF7D2FF44F21C41C5F60201096825
:10AF6E00C1F302124DF69221C0F60101895C01F087
:06AF7E001F01C84080BD68
:10AF840080B5FFF7BFFF44F21C41C5F60201096812
:10AF9400C1F302224DF69221C0F60101895C01F051
:06AFA4001F01C84080BD42
:10AFAA0080B586B00490039100208DF807000498BC
:10AFBA00006820B1049800683F2800D807E04DF2E5
:10AFCA002A60C0F6010040F67261FBF79FFE049802
:10AFDA004068042805D304984068B0F5007F00D87B
:10AFEA0007E04DF22A60C0F6010040F67361FBF7F4
:10AFFA008DFE0498806820B104988068802800D863
:10B00A0007E04DF22A60C0F6010040F67461FBF7D2
:10B01A007DFE0498006920B104980069802800D850
:10B02A0007E04DF22A60C0F6010040F67561FBF7B1
:10B03A006DFE0498C06820B10498C068802800D8C2
:10B04A0007E04DF22A60C0F6010040F67661FBF790
:10B05A005DFE0498406958B104984069402807D0B9
:10B06A0004984069802803D004984069C02800D118
:10B07A0007E04DF22A60C0F6010040F67761FBF75F
:10B08A0045FE0498806918B104988069202800D187
:10B09A0007E04DF22A60C0F6010040F67861FBF73E
:10B0AA0035FE0498C069400B00B907E04DF22A60EA
:10B0BA00C0F6010040F67961FBF728FE44F2284009
:10B0CA00C5F60200006800F00300032803D101203E
:10B0DA008DF81700B7E044F20041C5F6020108688E
:10B0EA0020F0806008600AF0E6F8029044F200401E
:10B0FA00C5F602000068C0F3C06050B10AF0DBF880
:10B10A000299401A032803D303208DF817009AE006
:10B11A00ECE744F22841C5F60201086820F47C30C5
:10B12A00049A126840EA0230086004994868D1F823
:10B13A0008C0CB680A6901386FF35F204FF60061D7
:10B14A00CFF6FF7101EB4C2189B208440021CFF6FA
:10B15A00FF7101EB034101F4FE0108444FF07F4106
:10B16A0001EB026101F0FE41084444F23841C5F6A0
:10B17A000201086044F22C41C5F6020100910868F8
:10B18A0020F0C000049A526910430860086820F051
:10B19A002000049A926910430860086820F01000A1
:10B1AA00086044F23C42C5F6020210684FF6F87392
:10B1BA009843049BDB6940EAC3001060086840F0CA
:10B1CA0010000860039840B944F22C41C5F6020108
:10B1DA00086840F40020086013E00398012808D1A9
:10B1EA0044F22C41C5F60201086840F48010086058
:10B1FA0007E044F22C41C5F60201086840F4001049
:10B20A00086044F20041C5F60201086840F0806017
:10B21A0008600AF050F8029044F20040C5F60200B5
:10B22A000068C0F3C06050B90AF045F80299401AA4
:10B23A00032803D303208DF8170004E0ECE79DF8F8
:0EB24A0007008DF817009DF8170006B080BDB4
:10B2580080B586B00490039100208DF8070004980B
:10B26800006820B1049800683F2800D807E04DF234
:10B278002A60C0F6010040F6DA61FBF748FD049841
:10B288004068042805D304984068B0F5007F00D8CA
:10B2980007E04DF22A60C0F6010040F6DB61FBF7DB
:10B2A80036FD0498806820B104988068802800D80A
:10B2B80007E04DF22A60C0F6010040F6DC61FBF7BA
:10B2C80026FD0498006920B104980069802800D8F8
:10B2D80007E04DF22A60C0F6010040F6DD61FBF799
:10B2E80016FD0498C06820B10498C068802800D86A
:10B2F80007E04DF22A60C0F6010040F6DE61FBF778
:10B3080006FD0498406970B104984069B0F5806FF3
:10B3180009D004984069B0F5006F04D004984069DA
:10B32800B0F5406F00D107E04DF22A60C0F6010089
:10B3380040F6DF61FBF7EBFC0498806920B10498C4
:10B348008069B0F5007F00D107E04DF22A60C0F6B1
:10B3580001004FF46E61FBF7DAFC0498C069400BFA
:10B3680000B907E04DF22A60C0F6010040F6E1613D
:10B37800FBF7CDFC44F22840C5F60200006800F057
:10B388000300032803D101208DF81700B7E044F229
:10B398000041C5F60201086820F08050086009F0F5
:10B3A8008BFF029044F20040C5F602000068C0F32B
:10B3B800407050B109F080FF0299401A032803D366
:10B3C80003208DF817009AE0ECE744F22841C5F60F
:10B3D8000201086820F07C70049A126840EA025062
:10B3E800086004994868D1F808C0CB680A69013830
:10B3F8006FF35F204FF60061CFF6FF7101EB4C2130
:10B4080089B208440021CFF6FF7101EB034101F432
:10B41800FE0108444FF07F4101EB026101F0FE415B
:10B42800084444F24041C5F60201086044F22C4148
:10B43800C5F602010091086820F44060049A526938
:10B4480010430860086820F40070049A9269104359
:10B458000860086820F48070086044F24442C5F629
:10B46800020210684FF6F8739843049BDB6940EAC0
:10B47800C3001060086840F480700860039840B901
:10B4880044F22C41C5F60201086840F480000860C7
:10B4980013E00398012808D144F22C41C5F60201B3
:10B4A800086840F40000086007E044F22C41C5F643
:10B4B8000201086840F08070086044F20041C5F657
:10B4C8000201086840F08050086009F0F5FE02901B
:10B4D80044F20040C5F602000068C0F3407050B95D
:10B4E80009F0EAFE0299401A032803D303208DF8D5
:10B4F800170004E0ECE79DF807008DF817009DF8A9
:06B50800170006B080BD33
:10B50E0080B5FFF7FAFC44F22041C5F60201096846
:10B51E00C1F302124DF69221C0F60101895C01F0D1
:06B52E001F01C84080BDB2
:10B5340080B582B0019001208DF8030001980028A5
:10B5440000F0E9800198006844F20001C5F60001AA
:10B55400884200D106E04DF28F10C0F60100FD21B3
:10B56400FBF7D7FB01984068402802D00198406857
:10B5740000B906E04DF28F10C0F60100FE21FBF782
:10B58400C8FB019880687F2800D806E04DF28F1030
:10B59400C0F60100FF21FBF7BCFB0198C068C00B9B
:10B5A40000B907E04DF28F10C0F601004FF480712E
:10B5B400FBF7AFFB0198006970B101980069B0F521
:10B5C400001F09D001980069B0F5800F04D00198DC
:10B5D4000069B0F5C00F00D107E04DF28F10C0F63E
:10B5E400010040F20111FBF794FB0198406918B186
:10B5F40001984069022800D107E04DF28F10C0F68F
:10B6040001004FF48171FBF784FB0198806920B13C
:10B6140001988069B0F5801F00D107E04DF28F10CA
:10B62400C0F6010040F20311FBF773FB0198C069F7
:10B6340018B10198C069012800D107E04DF28F10BC
:10B64400C0F601004FF48271FBF763FB019890F898
:10B65400210030B90199002081F820000198FBF7FE
:10B664007AFB0199022081F8210001980068C068E2
:10B67400C0F30010002844D101980168CA20486230
:10B684000198016853204862019800F048F88DF849
:10B6940003009DF80300F0B90198016888684FF62B
:10B6A400BF72CFF68F7210408860019A116850689B
:10B6B40013699269184302438868104388600198AB
:10B6C40001688268C06840EA02400861019800F09D
:10B6D4005DF88DF803009DF8030068B901980168CE
:10B6E400C86C20F00300C864019801684269C0690D
:10B6F4000243C86C1043C86401980168FF20486283
:10B7040002E000208DF803009DF8030018B90199A8
:0EB71400012081F821009DF8030002B080BDE5
:10B7220080B584B0039000208DF80700039800686C
:10B73200C0684006002826D4039801684FF0FF3005
:10B74200C86009F0BCFD029003980068C16800203F
:10B7520049060029009005D49DF80700033818BF58
:10B76200012000900098C00768B109F0A8FD029975
:10B77200401AB0F57A7F05D903208DF807000399A6
:0EB7820081F82100E0E79DF8070004B080BDCB
:10B7900080B582B0019000208DF8030044F20C01C6
:10B7A000C5F60001086820F08000086044F2080037
:10B7B000C5F600000068800600280AD401980BF046
:10B7C0004FFF28B10199032081F821008DF8030073
:10B7D00019E044F20801C5F60001086820F02000D5
:10B7E000086001980BF03CFF28B10199032081F813
:10B7F00021008DF8030044F20801C5F60001086835
:0EB8000040F0200008609DF8030002B080BDFB
:10B80E0080B58AB00890089818B901208DF82700E5
:10B81E00DBE00898006847F20001C5F2002188427B
:10B82E0007D00898006842F20041C4F6020188422F
:10B83E0000D107E04DF29460C0F601004FF4B071F4
:10B84E00FBF762FA0898406820B108984068B0F596
:10B85E00803F00D107E04DF29460C0F6010040F247
:10B86E006111FBF751FA0898806820B1089880683A
:10B87E00B0F5805F00D107E04DF29460C0F6010094
:10B88E004FF4B171FBF740FA0898C06848B10898B8
:10B89E00C068B0F5804F04D00898C068B0F5004F6E
:10B8AE0000D107E04DF29460C0F6010040F2631142
:10B8BE00FBF72AFA0898006920B108980069B0F5DC
:10B8CE00003F00D107E04DF29460C0F601004FF446
:10B8DE00B271FBF719FA08984069800A00B907E0BF
:10B8EE004DF29460C0F6010040F26511FBF70CFAC0
:10B8FE00089890F8300028B9089900200876089822
:10B90E00FBF74BFA0899042081F8300008980BF0E9
:10B91E00C6FE18B101208DF8270056E0089803A93D
:10B92E000BF04FFF18B101208DF827004DE09DF868
:10B93E001C0002909DF81D0001900898806B012854
:10B94E0008D1029808B9019820B108994FF40070F7
:10B95E0088650BE00898806B012804D108994FF494
:10B96E008070886502E00899002088650898C16893
:10B97E0000F02FF818B101208DF8270025E009F00E
:10B98E0098FC009008980BF0B0FF042812D009F034
:10B99E0090FC0099401A013058B908994FF00040B8
:10B9AE0048630899012081F8300003208DF82700A4
:10B9BE000BE0E7E70899002048630899C862089AE7
:10B9CE00012182F830108DF827009DF827000AB06B
:02B9DE0080BD2A
:10B9E00010B58CB00B900A9100208DF80B000A98CE
:10B9F00038B10A98B0F5804F03D00A98B0F5004FDF
:10BA000000D107E04DF29460C0F6010040F66711E6
:10BA1000FBF781F90B99032081F830000B98806BBC
:10BA2000032829D00A98B0F5004F05D10B99486B2F
:10BA300040F0805048631EE00A98B0F5804F09D16D
:10BA40000B980BF095FF0490049A0B99486B1043E8
:10BA5000486310E00A9848B90B9800F0EEF804909B
:10BA6000049A0B99486B1043486304E00B99486BA8
:10BA700040F00060486304E00B99486B40F0805050
:10BA800048630B98406B50B10B98016840F6FF700B
:10BA9000C1F6E070886301208DF80B00ADE04FF433
:10BAA00080300021F8F71CFE03900398002800F076
:10BAB0009C800B98406805900B98806806900A98C7
:10BAC00007900B98006908900B984069039943F61A
:10BAD0008932C5F2E652A1FB0221B0EB116F03D30C
:10BAE0000B984069099070E00B98806DB0F5007F6D
:10BAF00003D10B984069099067E00B98806DB0F511
:10BB0000807F31D10B984069A0B903984FF2810131
:10BB1000C0F2FA21884209D3039843F68931C5F26D
:10BB2000E651A0FB0110400E099002E00B9840691D
:10BB3000099018E003980B9949694900B0FBF1F0AE
:10BB40004FF28101C0F2FA21884209D3039843F6EB
:10BB50008931C5F2E651A0FB0110400E099002E0C8
:10BB60000B984069099030E00B984069A0B90398A0
:10BB700047F64101C0F27D11884209D3039843F68C
:10BB80008931C5F2E651A0FB0110000E099002E0D8
:10BB90000B984069099018E003980B99496949008E
:10BBA000B0FBF1F047F64101C0F27D11884209D3A4
:10BBB000039843F68931C5F2E651A0FB0110000E4F
:10BBC000099002E00B98406909900B98006805996C
:10BBD000069A079BDDF820C0099CEE46CEF804408B
:10BBE000CEF800C004F08AFF07E00B99486B40F0E4
:10BBF0000060486301208DF80B000B9800684FF43B
:10BC0000007105F052F90490049870B10B98016826
:10BC100040F6FF70C1F6E0708863049A0B99486B98
:10BC20001043486301208DF80B000B99012081F827
:0ABC300030009DF80B000CB010BDB1
:10BC3A0080B586B0049000210391029104980068AF
:10BC4A0005F064F88001002803D54FF400600590E0
:10BC5A002AE0049802A90BF0C6FE0190019810B1DF
:10BC6A000198059020E09DF80E00C007C8B104991C
:10BC7A000868496C090405F0EFFA0190019810B1BF
:10BC8A000198059010E004980068002105F01EFB59
:10BC9A000190019810B10198059005E000200590E7
:0EBCAA0002E04FF080600590059806B080BD66
:10BCB80080B58EB00C900B9109F0FEFA03900B98AA
:10BCC80001900C980068002105F021F880010028F7
:10BCD80003D54FF400600D90A2E00C980068402155
:10BCE80005F0DFF80490049828B10C99486B486374
:10BCF80004980D9094E00C990868496C090405F0C3
:10BD0800ACFA0490049828B10C99486B48630498DD
:10BD18000D9085E04FF0FF300590402006906020A0
:10BD28000790022008900020099001200A900C98A2
:10BD3800006805A905F00CF80C98006805F03BFCB4
:10BD48000490049828B10C99486B486304980D90A6
:10BD580066E00C980068406B10F4957F22D10C982F
:10BD68000068406B0004002811D50020029002985A
:10BD780007280CD80C98006804F043FF0199086064
:10BD8800019804300190029801300290EFE709F021
:10BD980093FA0399401A013018B94FF000400D90FA
:10BDA8003EE0D6E70C980068406B0007002802D5F3
:10BDB80008200D9034E00C980068406B800700283C
:10BDC80002D502200D902BE00C980068406B80068D
:10BDD800002802D520200D9022E00C980068406BC6
:10BDE800C004002813D50C98006804F00AFF0199D4
:10BDF800086001980430019009F05EFA0399401A2E
:10BE0800013018B94FF000400D9009E0E5E70C98B3
:10BE1800016840F63A70C1F60000886300200D9072
:06BE28000D980EB080BD74
:10BE2E0080B588B006900020059004900390069887
:10BE3E0000680DF07EFD0290029810B102980790F6
:10BE4E007AE00698006805F0EAF902900298B0F1DF
:10BE5E00004F0DD106990020C863069800680DF0BA
:10BE6E0068FD0290029810B10298079064E002E01B
:10BE7E0006990120C8630698C06B01280BD106985D
:10BE8E000068002105F0E6F90290029818B14FF013
:10BE9E008050079050E0059900204FF6FE729142B7
:10BEAE00019004D80398B0FA80F0400901900198EF
:10BEBE00C00758B306980068002105F0CBF9029030
:10BECE00029810B10298079036E00698006800219B
:10BEDE00CCF2101105F0DDF90290029818B14FF076
:10BEEE008050079028E006980068002104F00CFFAF
:10BEFE00049004994FF0FF3000EBD170B0FA80F04F
:10BF0E0040090390059801300590C4E705984FF657
:10BF1E00FF71884203D34FF0807007900CE00699B2
:10BF2E00002088639DF813004006002802D506996C
:0EBF3E000120886300200790079808B080BD9E
:10BF4C0083B0019000910198C06D800F009908702A
:10BF5C000198C06DC0F38360009948700198C06D62
:10BF6C00C0F30160009988700198B0F85E000099E8
:10BF7C00C8700198C06D000A009908710198C06DD5
:10BF8C00009948710198006E000D0099C8800198C5
:10BF9C00006EC0F30340009908720198B0F860007D
:10BFAC00C00B009948720198006EC0F38030009964
:10BFBC0088720198006EC0F340300099C8720198E5
:10BFCC00006EC0F30030009908730099002048738C
:10BFDC000198806B00284AD10199086E496E6FF365
:10BFEC009F20800040EA9170009908610198406E92
:10BFFC00C0F3C260009908750198406EC0F30260EE
:10C00C00009948750198406EC0F3425000998875AC
:10C01C000198406EC0F382400099C8750198406E3B
:10C02C00C0F3C2300099087600980069013001997C
:10C03C0088640098007E00F00700811C012000FA43
:10C04C0001F3019A916C594391640099097A01F0BA
:10C05C000F0188400199C8640199886CCA6C520A16
:10C06C005043086501994FF40070486533E001981E
:10C07C00806B01281CD10198016E01F03F01B0F8D2
:10C08C00660040EA014000990861009801694FF48C
:10C09C00806000EB8120019988640199886C0865A7
:10C0AC0001994FF40070C8640199C86C486512E09E
:10C0BC000198016840F6FF70C1F6E0708863019941
:10C0CC00486B40F0805048630199012081F83000A2
:10C0DC008DF80B0071E00198406EC0F38030009930
:10C0EC0048760198406EC0F3C61000998876019886
:10C0FC00406E00F07F000099C8760198806EC00FEA
:10C10C00009908770198806EC0F3417000994877C8
:10C11C000198806EC0F38260009988770198806ED8
:10C12C00C0F383500099C8770198806EC0F34050DB
:10C13C00009981F820000099002081F821000199D4
:10C14C00896EC1F30041009A82F822100199B1F86E
:10C15C006810C90B009A82F823100199896EC1F3FB
:10C16C008031009A82F824100199896EC1F3403114
:10C17C00009A82F825100199896EC1F30031009A5A
:10C18C0082F826100199896EC1F38121009A82F8F8
:10C19C0027100199896EC1F30121009A82F82810A9
:10C1AC00019991F868104908009A82F82910009AB0
:10C1BC00012182F82A108DF80B009DF80B0003B0BA
:02C1CC007047BA
:10C1CE0080B582B00190019800680DF06CFB02B052
:02C1DE0080BD22
:10C1E00080B58EB00C900B910A9209930A98019039
:10C1F0000B9840B90C99486B40F0006048630120EF
:10C200008DF8370089E00C9890F83000012840F054
:10C2100081800C99002048630198099908440C9981
:10C22000096D884208D90C99486B40F0007048634A
:10C2300001208DF8370070E00C99032081F8300060
:10C240000C9801680020C8620B980C994862099804
:10C2500040020C9988620C98806B012802D00198EA
:10C26000400201904FF0FF30039009984002049083
:10C2700090200590022006900020079008900C98CE
:10C28000006803A904F068FD0C980168C86840F0D4
:10C290004000C8600B980C99096888650C98016883
:10C2A000012008650998022809D30C998220C862E8
:10C2B0000C980068019904F03DFF029008E00C9989
:10C2C0008120C8620C980068019904F014FF029064
:10C2D0000298A8B10C98016840F6FF70C1F6E070B2
:10C2E0008863029A0C99486B104348630C990120AB
:10C2F00081F830000C9A0021D1628DF837000CE0F3
:10C300000C980168C86B40F49570C86300208DF8E4
:10C31000370002E002208DF837009DF837000EB09C
:02C3200080BDDE
:10C3220080B584B003900398C06A019003980068B6
:10C33200406B80B2C00B40B19DF80400000700289A
:10C3420003D503980BF08FFD71E103980068406BF1
:10C35200C0F30020002800F09F80039801684FF48A
:10C362008070886303980168C86B4CF23A1290435C
:10C37200C86303980168C86B20F08050C8630398B3
:10C382000168C86820F04000C8609DF804000007FA
:10C39200002837D59DF804008007002804D49DF8B2
:10C3A2000400800600280ED5039800680DF093FA69
:10C3B2000290029838B1029A0399486B104348637D
:10C3C20003980BF08CFD0398016840F63A70C1F6B1
:10C3D200000088630399012081F83000039900204E
:10C3E200C8629DF80400C00720B99DF804008007C8
:10C3F200002803D5039805F0CEF902E0039805F072
:10C40200BFF948E09DF804000006002843D50398D0
:10C4120001680020886203990968C8620399096863
:10C4220008659DF804008007002804D49DF80400E4
:10C43200800600280ED5039800680DF04CFA029091
:10C44200029838B1029A0399486B104348630398E3
:10C452000BF045FD0399012081F83000039900207B
:10C46200C8629DF80400C006002804D49DF80400A8
:10C472008006002802D5039805F082F99DF8040091
:10C48200C00720B99DF804008007002802D5039850
:10C4920005F081F9FFE7CAE003980068406BC0F33A
:10C4A200803040B19DF804000007002803D50398AE
:10C4B2000BF019FDBBE003980068406B10F03A0FD7
:10C4C20000F08A8003980068406BC0F3400020B1FE
:10C4D2000399486B40F00200486303980068406B80
:10C4E200C0F3C00020B10399486B40F008004863D4
:10C4F20003980068406BC0F3401020B10399486B69
:10C5020040F02000486303980068406BC0F30010BD
:10C5120020B10399486B40F010004863039801680A
:10C5220040F63A70C1F60000886303980168C86B50
:10C5320020F49D70C86303980168C86820F0400029
:10C54200C86003980168C86A40F40050C862039842
:10C552000168C86840F08000C860039800680DF068
:10C56200BAF902460399486B10434863039801687D
:10C57200C86820F08000C860039801684FF400602A
:10C5820088639DF80400000700280AD5039901205A
:10C5920081F8300003990020C86203980BF09FFCD9
:10C5A20019E09DF804000006002814D50398406B9A
:10C5B20080B103980168C86B20F08050C86303986B
:10C5C2000168002008650399012081F83000039872
:10C5D2000BF085FCFFE72AE003980068406BC0F38C
:10C5E200007020B3039801684FF08050886303986D
:10C5F2000068006D400700280CD49DF804008006F6
:10C60200002803D503980BF06AFC02E003980BF0B4
:10C6120066FC0BE09DF804008006002803D5039811
:10C622000BF05DFC02E003980BF059FCFFE704B04D
:02C6320080BDC9
:10C6340080B586B00490049818B901208DF81700CD
:10C64400EBE20498006843F20001C4F2010188425D
:10C6540027D00498006843F60001C4F20001884220
:10C664001FD00498006843F60041C4F200018842D8
:10C6740017D00498006843F20041C4F201018842D3
:10C684000FD00498006845F20001C4F20101884209
:10C6940007D00498006841F20041C5F600018842C1
:10C6A40000D106E04DF2F610C0F60100FE21FAF7C3
:10C6B40030FB0498406820B104984068B0F5800FBE
:10C6C40000D106E04DF2F610C0F60100FF21FAF7A2
:10C6D40020FB0498806870B104988068B0F5802FBE
:10C6E40009D004988068B0F5C02F04D004988068FD
:10C6F400B0F5003F00D107E04DF2F610C0F601009E
:10C704004FF48071FAF705FB0498C0681F2873D0B2
:10C714000498C0681E286FD00498C0681D286BD088
:10C724000498C0681C2867D00498C0681B2863D08C
:10C734000498C0681A285FD00498C06819285BD090
:10C744000498C068182857D00498C068172853D094
:10C754000498C06816284FD00498C06815284BD098
:10C764000498C068142847D00498C068132843D09C
:10C774000498C06815283FD00498C06812283BD09C
:10C784000498C068112837D00498C068102833D0A2
:10C794000498C0680F282FD00498C0680E282BD0A6
:10C7A4000498C0680D2827D00498C0680C2823D0AA
:10C7B4000498C0680B281FD00498C0680A281BD0AE
:10C7C4000498C068092817D00498C068082813D0B2
:10C7D4000498C06807280FD00498C06806280BD0B6
:10C7E4000498C068052807D00498C068042803D0BA
:10C7F4000498C068032800D107E04DF2F610C0F693
:10C80400010040F20111FAF784FA0498C06B002881
:10C8140043D00498C06B20283FD00498C06B4028B4
:10C824003BD00498C06B602837D00498C06B802834
:10C8340033D00498C06BA0282FD00498C06BC028B4
:10C844002BD00498C06BE02827D00498C06BB0F5B7
:10C85400807F22D00498C06BB0F5907F1DD00498DF
:10C86400C06BB0F5A07F18D00498C06BB0F5B07F52
:10C8740013D00498C06BB0F5C07F0ED00498C06B81
:10C88400B0F5D07F09D00498C06BB0F5E07F04D038
:10C894000498C06BB0F5F07F00D107E04DF2F610BC
:10C8A400C0F601004FF48171FAF733FA04988069F5
:10C8B400B0F1806F07D00498806920B10498806932
:10C8C400B0F1005F00D107E04DF2F610C0F60100B0
:10C8D40040F20311FAF71DFA0498406BB0F1804F4F
:10C8E40002D00498406B00B907E04DF2F610C0F690
:10C8F40001004FF48271FAF70CFA0498C06910B37E
:10C904000498C069B0F1805F1DD00498C069B0F18B
:10C91400005F18D00498C069B0F1405F13D0049848
:10C92400C069B0F1804F0ED00498C069B0F1A04F37
:10C9340009D00498C069B0F1C04F04D00498C0690C
:10C94400B0F1E04F00D107E04DF2F610C0F601005F
:10C9540040F20511FAF7DDF90498006A20B1049851
:10C96400006AB0F5000F00D107E04DF2F610C0F6F2
:10C9740001004FF48371FAF7CCF90498406A20B1AE
:10C984000498406AB0F5002F00D107E04DF2F6108C
:10C99400C0F6010040F20711FAF7BBF90498406AA7
:10C9A40008BB0498006920B104980069B0F1007FC5
:10C9B40000D107E04DF2F610C0F601004FF4857186
:10C9C400FAF7A7F90498406920B104984069B0F1D6
:10C9D400807F00D107E04DF2F610C0F6010040F26E
:10C9E4000B11FAF796F904990020886204980068FC
:10C9F40043F20001C4F20101884217D00498006890
:10CA040043F60001C4F2000188420FD00498006884
:10CA140043F60041C4F20001884207D00498C0687C
:10CA2400102803D301208DF81700F6E0049800F0D5
:10CA3400F8F802900498006843F20001C4F201017E
:10CA4400884212D00498006843F60001C4F2000141
:10CA540088420AD00498006843F60041C4F20001F9
:10CA6400884202D0029808281AD80498006843F231
:10CA74000001C4F2010188420FD00498006843F613
:10CA84000001C4F20001884207D00498006843F60C
:10CA94000041C4F20001884206D10298112803D350
:10CAA40001208DF81700B8E0049890F8810030B99F
:10CAB4000499002081F88000049808F0AFFA0499E2
:10CAC400022081F8810004980168086820F00100C0
:10CAD400086004980068806800F4F81003900498D3
:10CAE4008069B0F1806F15D104984068B0F5800F6B
:10CAF40002D10498806B38B10498406850B9049806
:10CB0400806BB0F1805F05D104980168086840F437
:10CB14008050086004988079400600280ED5049857
:10CB2400C06807280AD304980068006820F480705D
:10CB3400049A1168126D1043086005E004980168B6
:10CB4400086820F480700860049B1968DA68D86962
:10CB5400D3F828C040EA0C00DDF80CC040EA0C0011
:10CB6400DB6B184310438860049A0192506B516A3E
:10CB74000843916B0843916908431168D2F804C0D3
:10CB84009368D2F810E040EA0E00D2F814E040EACC
:10CB94000E00D2F820E040EA0E0040EA0C00D2F881
:10CBA4004CC040EA0C001843936C1843926D104338
:10CBB400C8600498406888B90498006880680121B6
:10CBC40061F3CC200499096888600498006880683F
:10CBD400022161F34A200499096888600498016875
:10CBE400086D20F00100086504988079400600284B
:10CBF40009D504980068C06820F00040049A1168C0
:10CC0400526D1043C86004990020C1F88400049A4E
:10CC1400012182F881108DF817009DF8170006B0E5
:02CC240080BDD1
:10CC260083B002900298C16B012000EB5110019075
:10CC36000298C0680130009000980730C008009044
:0ACC460000980199484303B07047BD
:10CC500082B00190019800684069009001980168D5
:10CC6000886940F00800886101980168886940F08F
:10CC70001000886101980168086820F001000860D0
:10CC800001980168086940F26F3290430861019889
:10CC90000168886820F440408860019890F881001D
:10CCA000042811D09DF80000800600280CD50199B9
:10CCB000D1F8840040F08000C1F884000198016838
:10CCC000886940F020008861019890F8810003286D
:10CCD00011D09DF80000400600280CD50199D1F82C
:10CCE000840040F00400C1F884000198016888695C
:10CCF00040F0400088619DF80100800700280CD5B5
:10CD00000199D1F8840040F00100C1F88400019835
:10CD10000168886940F4007088619DF80100C007CF
:10CD200060B10199D1F8840040F00800C1F8840096
:10CD300001980168886940F4807088610199002039
:0ECD4000A1F862000199A1F86A0002B07047E4
:10CD4E0080B584B00290029818B901208DF80F00BA
:10CD5E0043E1029800680021C4F20101884274D0B8
:10CD6E0002980068B0F1804F6FD00298006840F2D0
:10CD7E000041C4F20001884267D00298006840F674
:10CD8E000001C4F2000188425FD00298006840F6AC
:10CD9E000041C4F20001884257D00298006841F267
:10CDAE000001C4F2000188424FD00298006841F29F
:10CDBE000041C4F20001884247D00298006840F258
:10CDCE000041C4F2010188423FD00298006841F64A
:10CDDE000001C4F20001884237D00298006841F683
:10CDEE000041C4F2000188422FD00298006842F23E
:10CDFE000001C4F20001884227D00298006844F274
:10CE0E000001C4F2010188421FD00298006844F26A
:10CE1E000041C4F20101884217D00298006844F61E
:10CE2E000001C4F2010188420FD0029800684EF250
:10CE3E000001C4F20001884207D0029800684EF249
:10CE4E000041C4F20001884200D107E04DF25D209E
:10CE5E00C0F601004FF48B71F9F756FF0298806807
:10CE6E0078B10298806810280BD00298806820282C
:10CE7E0007D002988068402803D002988068602806
:10CE8E0000D107E04DF25D20C0F6010040F217110F
:10CE9E00F9F73AFF0298006948B102980069B0F5B7
:10CEAE00807F04D002980069B0F5007F00D107E0C2
:10CEBE004DF25D20C0F601004FF48C71F9F724FF9E
:10CECE00029801680120B1F1804F01901ED00298A6
:10CEDE000168012040F60042C4F200029142019026
:10CEEE0014D00298016801204EF20002C4F2000232
:10CEFE00914201900AD00298006841F60041CBF6AB
:10CF0E00FF710844B0FA80F0400901900198C00703
:10CF1E0040B90298C06848B10298C068B0F5803F29
:10CF2E0003D303E00298C06800B107E04DF25D2024
:10CF3E00C0F6010040F21911F9F7E6FE0298806979
:10CF4E0018B102988069802800D107E04DF25D206B
:10CF5E00C0F601004FF48D71F9F7D6FE029890F8E5
:10CF6E003D0030B90299002081F83C000298FAF792
:10CF7E00A8F90299022081F83D00029951F8040B9C
:10CF8E0000F02FF80299012081F848000299012043
:10CF9E0081F83E00029981F83F00029981F8400025
:10CFAE00029981F84100029981F84200029981F8B4
:10CFBE0043000299012081F84400029981F845004E
:10CFCE00029981F84600029981F8470002990120E2
:10CFDE0081F83D0000208DF80F009DF80F0004B081
:02CFEE0080BD04
:10CFF00083B002900191029800680090029800218D
:10D00000C4F2010188421FD00298B0F1804F1BD0BA
:10D01000029840F20041C4F20001884214D0029804
:10D0200040F60001C4F2000188420DD0029840F69B
:10D030000041C4F20001884206D0029840F200414B
:10D04000C4F20101884208D1009820F070000090DD
:10D050000198416800980843009002980021C4F2AA
:10D060000101884242D00298B0F1804F3ED0029830
:10D0700040F20041C4F20001884237D0029840F6E5
:10D080000001C4F20001884230D0029840F600410D
:10D09000C4F20001884229D0029840F20041C4F253
:10D0A0000101884222D0029844F20001C4F2010139
:10D0B00088421BD0029844F20041C4F20101884228
:10D0C00014D0029844F60001C4F2010188420DD048
:10D0D00002984EF20001C4F20001884206D0029884
:10D0E0004EF20041C4F20001884208D1009820F4B9
:10D0F000407000900198C168009808430090009823
:10D1000020F08000019949690843009001988068E7
:10D110000299C86201980068029988620298002109
:10D12000C4F2010188421BD0029840F20041C4F2CF
:10D130000101884214D0029844F20001C4F20101B6
:10D1400088420DD0029844F20041C4F201018842A5
:10D1500006D0029844F60001C4F20101884203D1CE
:10D1600001980069029908630299086840F0040078
:10D17000086002990120486100980299086003B094
:02D180007047F6
:10D1820080B584B00290029818B901208DF80F0082
:10D1920043E1029800680021C4F20101884274D080
:10D1A20002980068B0F1804F6FD00298006840F298
:10D1B2000041C4F20001884267D00298006840F63C
:10D1C2000001C4F2000188425FD00298006840F674
:10D1D2000041C4F20001884257D00298006841F22F
:10D1E2000001C4F2000188424FD00298006841F267
:10D1F2000041C4F20001884247D00298006840F220
:10D202000041C4F2010188423FD00298006841F611
:10D212000001C4F20001884237D00298006841F64A
:10D222000041C4F2000188422FD00298006842F205
:10D232000001C4F20001884227D00298006844F23B
:10D242000001C4F2010188421FD00298006844F232
:10D252000041C4F20101884217D00298006844F6E6
:10D262000001C4F2010188420FD0029800684EF218
:10D272000001C4F20001884207D0029800684EF211
:10D282000041C4F20001884200D107E04DF25D2066
:10D29200C0F6010040F23351F9F73CFD0298806874
:10D2A20078B10298806810280BD0029880682028F4
:10D2B20007D002988068402803D0029880686028CE
:10D2C20000D107E04DF25D20C0F6010040F234517A
:10D2D200F9F720FD0298006948B102980069B0F59B
:10D2E200807F04D002980069B0F5007F00D107E08A
:10D2F2004DF25D20C0F6010040F23551F9F70AFD0A
:10D30200029801680120B1F1804F01901ED002986D
:10D312000168012040F60042C4F2000291420190ED
:10D3220014D00298016801204EF20002C4F20002F9
:10D33200914201900AD00298006841F60041CBF672
:10D34200FF710844B0FA80F0400901900198C007CB
:10D3520040B90298C06848B10298C068B0F5803FF1
:10D3620003D303E00298C06800B107E04DF25D20EC
:10D37200C0F6010040F23651F9F7CCFC0298806900
:10D3820018B102988069802800D107E04DF25D2033
:10D39200C0F6010040F23751F9F7BCFC029890F850
:10D3A2003D0030B90299002081F83C0002980AF051
:10D3B20096FD0299022081F83D00029951F8040B72
:10D3C200FFF715FE0299012081F848000299012019
:10D3D20081F83E00029981F83F00029981F84000ED
:10D3E200029981F84100029981F84200029981F87C
:10D3F20043000299012081F84400029981F8450016
:10D40200029981F84600029981F8470002990120A9
:10D4120081F83D0000208DF80F009DF80F0004B048
:02D4220080BDCB
:10D4240080B584B00290029818B901208DF80F00DD
:10D4340043E1029800680021C4F20101884274D0DB
:10D4440002980068B0F1804F6FD00298006840F2F3
:10D454000041C4F20001884267D00298006840F697
:10D464000001C4F2000188425FD00298006840F6CF
:10D474000041C4F20001884257D00298006841F28A
:10D484000001C4F2000188424FD00298006841F2C2
:10D494000041C4F20001884247D00298006840F27B
:10D4A4000041C4F2010188423FD00298006841F66D
:10D4B4000001C4F20001884237D00298006841F6A6
:10D4C4000041C4F2000188422FD00298006842F261
:10D4D4000001C4F20001884227D00298006844F297
:10D4E4000001C4F2010188421FD00298006844F28E
:10D4F4000041C4F20101884217D00298006844F642
:10D504000001C4F2010188420FD0029800684EF273
:10D514000001C4F20001884207D0029800684EF26C
:10D524000041C4F20001884200D107E04DF25D20C1
:10D53400C0F6010040F2CF71F9F7EBFB0298806866
:10D5440078B10298806810280BD00298806820284F
:10D5540007D002988068402803D002988068602829
:10D5640000D107E04DF25D20C0F601004FF4FA61EE
:10D57400F9F7CFFB0298006948B102980069B0F549
:10D58400807F04D002980069B0F5007F00D107E0E5
:10D594004DF25D20C0F6010040F2D171F9F7B9FBFC
:10D5A400029801680120B1F1804F01901ED00298C9
:10D5B4000168012040F60042C4F200029142019049
:10D5C40014D00298016801204EF20002C4F2000255
:10D5D400914201900AD00298006841F60041CBF6CE
:10D5E400FF710844B0FA80F0400901900198C00727
:10D5F40040B90298C06848B10298C068B0F5803F4D
:10D6040003D303E00298C06800B107E04DF25D2047
:10D61400C0F6010040F2D271F9F77BFB02988069F1
:10D6240018B102988069802800D107E04DF25D208E
:10D63400C0F6010040F2D371F9F76BFB029890F841
:10D644003D0030B90299002081F83C0002980AF0AC
:10D6540045FC0299022081F83D00029951F8040B1F
:10D66400FFF7C4FC0299012081F8480002990120C7
:10D6740081F83E00029981F83F00029981F8400048
:10D68400029981F84100029981F84200029981F8D7
:10D6940043000299012081F84400029981F8450071
:10D6A400029981F84600029981F847000299012005
:10D6B40081F83D0000208DF80F009DF80F0004B0A4
:02D6C40080BD27
:10D6C60080B584B0039003980068C0680290039800
:10D6D6000068006901909DF80400800700281ED5A7
:10D6E6009DF808008007002819D5039801686FF097
:10D6F6000200086103990120087703980068806991
:10D70600800718B10398F9F7A2FC05E003980AF020
:10D71600E4FB03980AF0E1FB0399002008779DF8E3
:10D726000400400700281FD59DF808004007002880
:10D736001AD5039801686FF0040008610399022066
:10D74600087703980068806910F4407F03D0039837
:10D75600F9F77DFC05E003980AF0BFFB03980AF091
:10D76600BCFB0399002008779DF8040000070028F9
:10D776001ED59DF808000007002819D503980168F2
:10D786006FF0080008610399042008770398006881
:10D79600C069800718B10398F9F759FC05E00398AA
:10D7A6000AF09BFB03980AF098FB03990020087780
:10D7B6009DF80400C00600281FD59DF80800C00685
:10D7C60000281AD5039801686FF0100008610399C4
:10D7D6000820087703980068C06910F4407F03D0DA
:10D7E6000398F9F734FC05E003980AF076FB0398F2
:10D7F6000AF073FB0399002008779DF80400C00720
:10D8060058B19DF80800C00738B1039801686FF059
:10D81600010008610398F9F76CFA019800F080009E
:10D82600802804D09DF80500800600280CD59DF8B8
:10D8360008000006002807D5039801686FF4025017
:10D84600086103980AF049FB9DF80500C00760B11E
:10D856009DF808000006002807D5039801686FF4B4
:10D866008070086103980AF038FB9DF804004006B2
:10D8760000280CD59DF808004006002807D5039817
:10D8860001686FF04000086103980AF026FB9DF8D6
:10D896000400800600280CD59DF8080080060028A4
:10D8A60007D5039801686FF02000086103980AF015
:06D8B60014FB04B080BD6C
:10D8BC0080B586B0059004910598006A0290059990
:10D8CC00086A20F0010008620598406801900598EC
:10D8DC008069039003984FF68F71CFF6FE71084064
:10D8EC000390039820F003000390049801680398B8
:10D8FC0008430390029820F002000290049881687B
:10D90C0002980843029005980021C4F20101884254
:10D91C001BD0059840F20041C4F20101884214D09A
:10D92C00059844F20001C4F2010188420DD005981B
:10D93C0044F20041C4F20101884206D0059844F635
:10D94C000001C4F2010188421CD10498C06818B1CE
:10D95C000498C068082800D107E04DF25D20C0F69D
:10D96C00010041F66B31F9F7D0F9029820F008006C
:10D97C0002900498C168029808430290029820F023
:10D98C000400029005980021C4F2010188421BD0CA
:10D99C00059840F20041C4F20101884214D0059868
:10D9AC0044F20001C4F2010188420DD0059844F202
:10D9BC000041C4F20101884206D0059844F60001EA
:10D9CC00C4F20101884233D104988069B0F5007F1C
:10D9DC0002D00498806900B907E04DF25D20C0F6D2
:10D9EC00010041F67831F9F790F904984069B0F5E7
:10D9FC00807F02D00498406900B907E04DF25D20A9
:10DA0C00C0F6010041F67931F9F77FF9019820F45D
:10DA1C0080700190019820F4007001900498416985
:10DA2C00019808430190049881690198084301907A
:10DA3C000198059948600398059988610498406895
:0EDA4C000599486302980599086206B080BDEE
:10DA5A0080B586B0059004910598006A02900599F0
:10DA6A00086A20F480700862059840680190059859
:10DA7A00C069039003984FF68F71CFF6FE71084084
:10DA8A000390039820F00300039004980168039818
:10DA9A0008430390029820F4007002900498816869
:10DAAA00029840EA0120029005980021C4F201017F
:10DABA00884221D0059840F20041C4F2010188420F
:10DACA001AD0059844F20001C4F20101884201D13A
:10DADA00002088B9059844F20041C4F20101884245
:10DAEA0001D1002040B9059844F60001C4F20101B1
:10DAFA0088421FD10120E8B90498C06818B1049877
:10DB0A00C068082800D107E04DF25D20C0F6010088
:10DB1A0041F60241F9F7FAF8029820F400600290FF
:10DB2A000498C168029840EA01200290029820F401
:10DB3A008060029005980021C4F2010188421BD03E
:10DB4A00059840F20041C4F20101884214D00598B8
:10DB5A0044F20001C4F2010188420DD0059844F252
:10DB6A000041C4F20101884206D0059844F600013A
:10DB7A00C4F20101884235D104988069B0F5007F6A
:10DB8A0002D00498806900B907E04DF25D20C0F622
:10DB9A00010041F60F41F9F7B9F804984069B0F568
:10DBAA00807F02D00498406900B907E04DF25D20F9
:10DBBA00C0F6010041F61041F9F7A8F8019820F4DF
:10DBCA0080500190019820F4005001900498416916
:10DBDA00019840EA0110019004988169019840EA8D
:10DBEA000110019001980599486003980599C86148
:10DBFA00049840680599C86302980599086206B0B6
:02DC0A0080BDDB
:10DC0C0080B586B0059004910598006A029005993C
:10DC1C00086A20F4805008620598406801900598C5
:10DC2C00C0690390039848F6FF71CFF6FF61084076
:10DC3C000390039820F440700390049801680398B3
:10DC4C0040EA01200390029820F4005002900498BE
:10DC5C008168029840EA0130029005980021C4F2D4
:10DC6C00010188421BD0059840F20041C4F2010129
:10DC7C00884214D0059844F20001C4F20101884294
:10DC8C000DD0059844F20041C4F20101884206D03F
:10DC9C00059844F60001C4F2010188421AD1049897
:10DCAC004069B0F5807F02D00498406900B907E064
:10DCBC004DF25D20C0F6010041F64F41F9F725F811
:10DCCC00019820F48040019004984169019840EA41
:10DCDC008110019001980599486003980599C861D5
:10DCEC00049840680599086402980599086206B082
:02DCFC0080BDE9
:10DCFE0085B0049003910498006A01900499086A13
:10DD0E0020F4801008620498406800900498406DDA
:10DD1E000290029848F6FF71CFF6FF61084002901C
:10DD2E0003980168029840EA01200290019820F4BD
:10DD3E000010019003988168019840EA015001900B
:10DD4E0004980021C4F2010188421BD0049840F2CD
:10DD5E000041C4F20101884214D0049844F200013B
:10DD6E00C4F2010188420DD0049844F20041C4F27D
:10DD7E000101884206D0049844F60001C4F2010164
:10DD8E00884209D1009820F48020009003984169C0
:10DD9E00009840EA8120009000980499486002980B
:10DDAE0004994865039840680499C86501980499D8
:06DDBE00086205B0704789
:10DDC40080B586B004900391029200208DF807007C
:10DDD400049800680021C4F20101884264D00498C8
:10DDE4000068B0F1804F5FD00498006840F20041B1
:10DDF400C4F20001884257D00498006840F600013C
:10DE0400C4F2000188424FD00498006840F60041F3
:10DE1400C4F20001884247D00498006840F20041EF
:10DE2400C4F2010188423FD00498006841F6000121
:10DE3400C4F20001884237D00498006841F60041DA
:10DE4400C4F2000188422FD00498006842F2000115
:10DE5400C4F20001884227D00498006844F200010B
:10DE6400C4F2010188421FD00498006844F20041C2
:10DE7400C4F20101884217D00498006844F60001F6
:10DE8400C4F2010188420FD0049800684EF20001E8
:10DE9400C4F20001884207D0049800684EF20041A1
:10DEA400C4F20001884200D107E04DF25D20C0F6C3
:10DEB400010041F24C01F8F72CFF0398006838B1D7
:10DEC40003980068022803D0039800680A2800D148
:10DED40007E04DF25D20C0F6010041F24D01F8F774
:10DEE40018FF03984068012807D003984068022867
:10DEF40003D003984068032800D107E04DF25D2069
:10DF0400C0F6010041F24E01F8F703FF0398806860
:10DF140058B103988068042807D0039880680828BB
:10DF240003D0039880680C2800D107E04DF25D20EF
:10DF3400C0F6010041F24F01F8F7EBFE0398C06808
:10DF44000F2800D807E04DF25D20C0F6010041F231
:10DF54005001F8F7DEFE049890F83C00012803D144
:10DF640002208DF8170052E10499012081F83C0049
:10DF74000298A8B904980068039B19685A68DB687A
:10DF840000F049F904980168886920F00C00886160
:10DF940003988268049801688869104388612EE1B7
:10DFA400029804286BD1049800680021C4F201018E
:10DFB400884244D004980068B0F1804F3FD0049860
:10DFC400006840F20041C4F20001884237D004984E
:10DFD400006840F60001C4F2000188422FD0049882
:10DFE400006840F60041C4F20001884227D004983A
:10DFF400006840F20041C4F2010188421FD0049835
:10E00400006841F60001C4F20001884217D0049868
:10E01400006844F20001C4F2010188420FD0049860
:10E0240000684EF20001C4F20001884207D004984F
:10E0340000684EF20041C4F20001884200D107E0BA
:10E044004DF25D20C0F6010041F26601F8F761FE71
:10E0540004980068039B19685A68DB680AF042FE5A
:10E0640004980168886920F4406088610398826894
:10E0740004980168886940EA02208861BFE0029838
:10E0840008285AD1049800680021C4F2010188428A
:10E0940034D004980068B0F1804F2FD00498006801
:10E0A40040F20041C4F20001884227D0049800687D
:10E0B40040F60001C4F2000188421FD004980068B1
:10E0C40040F60041C4F20001884217D00498006869
:10E0D40040F20041C4F2010188420FD00498006864
:10E0E4004EF20001C4F20001884207D0049800688F
:10E0F4004EF20041C4F20001884200D107E04DF223
:10E104005D20C0F6010041F27601F8F702FE0498A2
:10E114000068039B19685A68DB6800F00FF90498DB
:10E124000168C86920F00C00C861039882680498EB
:10E134000168C8691043C86161E002980C285BD18A
:10E14400049800680021C4F20101884234D0049884
:10E154000068B0F1804F2FD00498006840F200416D
:10E16400C4F20001884227D00498006840F60001F8
:10E17400C4F2000188421FD00498006840F60041B0
:10E18400C4F20001884217D00498006840F20041AC
:10E19400C4F2010188420FD0049800684EF20001D5
:10E1A400C4F20001884207D0049800684EF200418E
:10E1B400C4F20001884200D107E04DF25D20C0F6B0
:10E1C400010041F28601F8F7A4FD04980068039B5E
:10E1D40019685A68DB680AF0BBFD04980168C869CD
:10E1E40020F44060C8610398826804980168C86993
:10E1F40040EA0220C86102E001208DF8070004997A
:10E20400002081F83C009DF807008DF817009DF868
:06E21400170006B080BDFA
:10E21A0087B006900591049203930698006A0190CC
:10E22A000699086A20F0010008620698806902903F
:10E23A00069901200022C4F20102914200904ED0B8
:10E24A0006990120B1F1804F009048D0069901202B
:10E25A0040F20042C4F20002914200903FD0069977
:10E26A00012040F60002C4F200029142009036D02A
:10E27A000699012040F60042C4F200029142009041
:10E28A002DD00699012040F20042C4F201029142C7
:10E29A00009024D00699012041F60002C4F200023F
:10E2AA00914200901BD00699012044F20002C4F268
:10E2BA0001029142009012D0069901204EF200020A
:10E2CA00C4F200029142009009D0069841F600413A
:10E2DA00CBF6FF710844B0FA80F04009009000982C
:10E2EA00C00740B1029820F00300029004990298F6
:10E2FA000843029003E0029840F00100029002985D
:10E30A0020F0F000029003980001C1B2029808437D
:10E31A000290019820F00A000190059800F00A0185
:10E32A000198084301900298069988610198069914
:06E33A00086207B0704705
:10E3400086B005900491039202930598006A0090AC
:10E350000599086A20F4807008620598C0690190E8
:10E36000019820F00300019003990198084301905F
:10E37000019820F0F000019002980001C1B20198CC
:10E3800008430190009820F420600090049800F069
:10E390000A01009840EA0120009001980599C8619F
:0AE3A00000980599086206B0704766
:10E3AA0080B586B00490039100208DF80B00049884
:10E3BA0090F83C00012804D102208DF8170000F0E3
:10E3CA0060BC0499012081F83C000499022081F87C
:10E3DA003D0003980068B0F5805F23D00398006879
:10E3EA0070281FD003980068B0F5005F1AD0039810
:10E3FA000068402816D003980068502812D0039865
:10E40A00006860280ED00398006858B10398006825
:10E41A00102807D003980068202803D003980068C2
:10E42A00302800D107E04DF25D20C0F6010041F22C
:10E43A005151F8F76BFC04980068806801900198C4
:10E44A004FF68871CFF6CE7108400190019820F4FA
:10E45A007F400190019804990968886003980068D0
:10E46A000090002800F0A2830098102800F09E83F4
:10E47A000098202800F09A830098302800F09683AC
:10E48A000098402800F007830098502800F0ED819A
:10E49A000098602800F074820098702800F0AF801D
:10E4AA000098B0F5805F24D00098B0F5005F00F0C6
:10E4BA0044810098B0F5801F00F078830098B0F18D
:10E4CA00101F00F0738300982021C0F210018842C7
:10E4DA0000F06C8300983021C0F21001884200F0ED
:10E4EA00658300984021C0F21001884200F05E83E3
:10E4FA00B8E3049800680021C4F20101884274D08C
:10E50A0004980068B0F1804F6FD00498006840F218
:10E51A000041C4F20001884267D00498006840F6BE
:10E52A000001C4F2000188425FD00498006840F6F6
:10E53A000041C4F20001884257D00498006841F2B1
:10E54A000001C4F2000188424FD00498006841F2E9
:10E55A000041C4F20001884247D00498006840F2A2
:10E56A000041C4F2010188423FD00498006841F694
:10E57A000001C4F20001884237D00498006841F6CD
:10E58A000041C4F2000188422FD00498006842F288
:10E59A000001C4F20001884227D00498006844F2BE
:10E5AA000001C4F2010188421FD00498006844F2B5
:10E5BA000041C4F20101884217D00498006844F669
:10E5CA000001C4F2010188420FD0049800684EF29B
:10E5DA000001C4F20001884207D0049800684EF294
:10E5EA000041C4F20001884200D107E04DF25D20EB
:10E5FA00C0F6010041F25D51F8F788FB35E3049853
:10E60A0000680021C4F20101884234D004980068ED
:10E61A00B0F1804F2FD00498006840F20041C4F254
:10E62A000001884227D00498006840F60001C4F22D
:10E63A00000188421FD00498006840F60041C4F2E5
:10E64A000001884217D00498006840F20041C4F2E1
:10E65A00010188420FD0049800684EF20001C4F20A
:10E66A000001884207D0049800684EF20041C4F2C3
:10E67A000001884200D107E04DF25D20C0F601009A
:10E68A0041F26451F8F742FB0398806870B103982D
:10E69A008068B0F5805F09D003988068B0F5005FA4
:10E6AA0004D003988068B0F5405F00D107E04DF2CE
:10E6BA005D20C0F6010041F26751F8F727FB039885
:10E6CA004068B0F5004F0DD00398406850B10398E8
:10E6DA00406838B103984068022803D0039840681C
:10E6EA000A2800D107E04DF25D20C0F6010041F290
:10E6FA006851F8F70BFB0398C0680F2800D807E0A9
:10E70A004DF25D20C0F6010041F26951F8F7FEFAB8
:10E71A0004980068039B5A689968DB680AF04BFB07
:10E72A000498006880680190019840F07700019091
:10E73A00019804990968886097E2049800680021A2
:10E74A00C4F20101884234D004980068B0F1804FC5
:10E75A002FD00498006840F20041C4F200018842B8
:10E76A0027D00498006840F60001C4F200018842EC
:10E77A001FD00498006840F60041C4F200018842A4
:10E78A0017D00498006840F20041C4F2010188429F
:10E79A000FD0049800684EF20001C4F200018842CA
:10E7AA0007D0049800684EF20041C4F20001884282
:10E7BA0000D107E04DF25D20C0F6010041F27C5124
:10E7CA00F8F7A4FA0398806870B103988068B0F5E6
:10E7DA00805F09D003988068B0F5005F04D0039881
:10E7EA008068B0F5405F00D107E04DF25D20C0F6C9
:10E7FA00010041F27F51F8F789FA03984068B0F5B1
:10E80A00004F0DD00398406850B10398406838B162
:10E81A0003984068022803D0039840680A2800D168
:10E82A0007E04DF25D20C0F601004FF4AC51F8F755
:10E83A006DFA0398C0680F2800D807E04DF25D20F2
:10E84A00C0F6010041F28151F8F760FA04980068B5
:10E85A00039B5A689968DB680AF0ADFA0498016864
:10E86A00886840F480408860FFE1049800680021CD
:10E87A00C4F20101884244D004980068B0F1804F84
:10E88A003FD00498006840F20041C4F20001884277
:10E89A0037D00498006840F60001C4F200018842AB
:10E8AA002FD00498006840F60041C4F20001884263
:10E8BA0027D00498006840F20041C4F2010188425E
:10E8CA001FD00498006841F60001C4F20001884292
:10E8DA0017D00498006844F20001C4F2010188428A
:10E8EA000FD0049800684EF20001C4F20001884279
:10E8FA0007D0049800684EF20041C4F20001884231
:10E90A0000D107E04DF25D20C0F6010041F29051BE
:10E91A00F8F7FCF903984068B0F5004F0DD003985A
:10E92A00406850B10398406838B10398406802289B
:10E93A0003D0039840680A2800D107E04DF25D2011
:10E94A00C0F6010041F29351F8F7E0F90398C06864
:10E95A000F2800D807E04DF25D20C0F6010041F211
:10E96A009451F8F7D3F904980068039A5168D26869
:10E97A000AF03BFA0498006850210AF05EFA74E142
:10E98A00049800680021C4F20101884244D0049826
:10E99A000068B0F1804F3FD00498006840F200410F
:10E9AA00C4F20001884237D00498006840F600019A
:10E9BA00C4F2000188422FD00498006840F6004152
:10E9CA00C4F20001884227D00498006840F200414E
:10E9DA00C4F2010188421FD00498006841F6000180
:10E9EA00C4F20001884217D00498006844F200017A
:10E9FA00C4F2010188420FD0049800684EF2000167
:10EA0A00C4F20001884207D0049800684EF200411F
:10EA1A00C4F20001884200D107E04DF25D20C0F641
:10EA2A0001004FF4AD51F8F771F903984068B0F559
:10EA3A00004F0DD00398406850B10398406838B130
:10EA4A0003984068022803D0039840680A2800D136
:10EA5A0007E04DF25D20C0F6010041F2A351F8F73C
:10EA6A0055F90398C0680F2800D807E04DF25D20D9
:10EA7A00C0F6010041F2A451F8F748F90498006879
:10EA8A00039A5168D26800F000F90498006860217E
:10EA9A000AF0D3F9E9E0049800680021C4F2010100
:10EAAA00884244D004980068B0F1804F3FD004985F
:10EABA00006840F20041C4F20001884237D004984D
:10EACA00006840F60001C4F2000188422FD0049881
:10EADA00006840F60041C4F20001884227D0049839
:10EAEA00006840F20041C4F2010188421FD0049834
:10EAFA00006841F60001C4F20001884217D0049868
:10EB0A00006844F20001C4F2010188420FD004985F
:10EB1A0000684EF20001C4F20001884207D004984E
:10EB2A0000684EF20041C4F20001884200D107E0B9
:10EB3A004DF25D20C0F6010041F2B051F8F7E6F857
:10EB4A0003984068B0F5004F0DD00398406850B163
:10EB5A000398406838B103984068022803D00398A4
:10EB6A0040680A2800D107E04DF25D20C0F6010096
:10EB7A0041F2B351F8F7CAF80398C0680F2800D8D1
:10EB8A0007E04DF25D20C0F6010041F2B451F8F7FA
:10EB9A00BDF804980068039A5168D2680AF025F90A
:10EBAA000498006840210AF048F95EE00498006879
:10EBBA000021C4F20101884244D004980068B0F1EF
:10EBCA00804F3FD00498006840F20041C4F200012F
:10EBDA00884237D00498006840F60001C4F2000168
:10EBEA0088422FD00498006840F60041C4F2000120
:10EBFA00884227D00498006840F20041C4F201011B
:10EC0A0088421FD00498006841F60001C4F200014E
:10EC1A00884217D00498006844F20001C4F2010146
:10EC2A0088420FD0049800684EF20001C4F2000135
:10EC3A00884207D0049800684EF20041C4F20001ED
:10EC4A00884200D107E04DF25D20C0F6010041F292
:10EC5A00C851F8F75BF804980068039909680AF044
:10EC6A00ECF802E001208DF80B000499012081F8EC
:10EC7A003D000499002081F83C009DF80B008DF8B6
:0AEC8A0017009DF8170006B080BDCA
:10EC940085B00490039102920498006A009004994C
:10ECA400086A20F0100008620498806901900198B5
:10ECB40020F4704001900299019840EA01300190DB
:10ECC400009820F0A00000900399009840EA0110F9
:10ECD400009001980499886100980499086205B02D
:02ECE400704777
:10ECE60080B584B002900191029800680021C4F2B8
:10ECF6000101884244D002980068B0F1804F3FD0AD
:10ED06000298006840F20041C4F20001884237D000
:10ED16000298006840F60001C4F2000188422FD034
:10ED26000298006840F60041C4F20001884227D0EC
:10ED36000298006840F20041C4F2010188421FD0E7
:10ED46000298006841F60001C4F20001884217D01B
:10ED56000298006844F20001C4F2010188420FD013
:10ED6600029800684EF20001C4F20001884207D002
:10ED7600029800684EF20041C4F20001884200D1B8
:10ED860007E04DF25D20C0F6010041F20861F7F799
:10ED9600BFFF01980068A0B101980068042810D050
:10EDA6000198006805280CD001980068062808D04C
:10EDB60001980068072804D001980068B0F5803FE4
:10EDC60000D107E04DF25D20C0F6010041F2096175
:10EDD600F7F79EFF01984068002846D001984068E2
:10EDE600102842D00198406820283ED001984068FB
:10EDF60030283AD001984068B0F5801F35D0019888
:10EE06004068B0F1101F30D0019840682021C0F250
:10EE16001001884229D0019840683021C0F21001C3
:10EE2600884222D0019840684021C0F210018842F1
:10EE36001BD001984068B0F5001F16D001984068B5
:10EE46001021C0F2200188420FD001984068402866
:10EE56000BD001984068502807D001984068602878
:10EE660003D001984068702800D107E04DF25D207C
:10EE7600C0F6010041F20A61F7F74AFF029890F8DE
:10EE86003C00012803D102208DF80F002FE00299E3
:10EE9600012081F83C000299022081F83D00029889
:10EEA600019900F028F858B10299012081F83D0037
:10EEB6000299002081F83C0001208DF80F0016E031
:10EEC60002980168C86820F04000C860029801688E
:10EED600C86820F48040C8600299012081F83D008E
:10EEE6000299002081F83C0000208DF80F009DF863
:06EEF6000F0004B080BD16
:10EEFC0080B588B00690059100208DF81300069817
:10EF0C0000688068039003984FF68F71CFF6CF712D
:10EF1C0008400390059841680398084303900398B0
:10EF2C004FF6F871CFF6FE71084003900598016812
:10EF3C00039808430390039806990968886005981C
:10EF4C0040680090002800F0C5820098102800F05E
:10EF5C00C1820098202800F0BD820098302800F073
:10EF6C00B9820098402800F0DE800098502800F00C
:10EF7C0085810098602800F027820098702840D086
:10EF8C000098B0F5801F00F0A5820098B0F1101F1A
:10EF9C0000F0A08200982021C0F21001884200F0FD
:10EFAC00998200983021C0F21001884200F09282C0
:10EFBC0000984021C0F21001884200F08B8200982A
:10EFCC005021C0F21001884200F084820098602128
:10EFDC00C0F21001884200F07D8200987021C0F2CE
:10EFEC001001884200F076820098B0F5001F00F006
:10EFFC00718200981021C0F22001884200F06A82D0
:10F00C00BEE2069800680021C4F20101884234D0A7
:10F01C0006980068B0F1804F2FD00698006840F237
:10F02C000041C4F20001884227D00698006840F6DF
:10F03C000001C4F2000188421FD00698006840F617
:10F04C000041C4F20001884217D00698006840F2D3
:10F05C000041C4F2010188420FD0069800684EF2BC
:10F06C000001C4F20001884207D0069800684EF2F5
:10F07C000041C4F20001884200D107E04DF25D204E
:10F08C00C0F6010041F6F641F7F73FFE0598C0685F
:10F09C0070B10598C068B0F5805F09D00598C0685C
:10F0AC00B0F5005F04D00598C068B0F5405F00D1A2
:10F0BC0007E04DF25D20C0F6010041F6F741F7F78D
:10F0CC0024FE05988068B0F5004F0DD00598806837
:10F0DC0050B10598806838B105988068022803D033
:10F0EC00059880680A2800D107E04DF25D20C0F633
:10F0FC00010041F6F841F7F708FE059800690F2862
:10F10C0000D807E04DF25D20C0F6010041F6F94150
:10F11C00F7F7FBFD06980068059B9A68D9681B6990
:10F12C0009F048FE2FE2069800680021C4F20101A4
:10F13C00884264D006980068B0F1804F5FD0069882
:10F14C00006840F20041C4F20001884257D0069892
:10F15C00006840F60001C4F2000188424FD00698C6
:10F16C00006840F60041C4F20001884247D006987E
:10F17C00006840F20041C4F2010188423FD0069879
:10F18C00006841F60001C4F20001884237D00698AD
:10F19C00006841F60041C4F2000188422FD0069865
:10F1AC00006842F20001C4F20001884227D00698A0
:10F1BC00006844F20001C4F2010188421FD0069895
:10F1CC00006844F20041C4F20101884217D006984D
:10F1DC00006844F60001C4F2010188420FD0069881
:10F1EC0000684EF20001C4F20001884207D0069874
:10F1FC0000684EF20041C4F20001884200D107E0E1
:10F20C004DF25D20C0F6010041F60551F7F77DFD8A
:10F21C00059800690F2800D807E04DF25D20C0F674
:10F22C00010041F60651F7F770FD059800680528B6
:10F23C0003D101208DF81F00A9E106980068006A2F
:10F24C00019006980168086A20F00100086206988F
:10F25C00006880690290029820F0F00002900598F6
:10F26C000169029840EA0110029002980699096817
:10F27C008861019806990968086284E1069800681B
:10F28C000021C4F20101884264D006980068B0F1F4
:10F29C00804F5FD00698006840F20041C4F2000134
:10F2AC00884257D00698006840F60001C4F200016D
:10F2BC0088424FD00698006840F60041C4F2000125
:10F2CC00884247D00698006840F20041C4F2010120
:10F2DC0088423FD00698006841F60001C4F2000154
:10F2EC00884237D00698006841F60041C4F200010C
:10F2FC0088422FD00698006842F20001C4F2000147
:10F30C00884227D00698006844F20001C4F201013B
:10F31C0088421FD00698006844F20041C4F20101F3
:10F32C00884217D00698006844F60001C4F2010127
:10F33C0088420FD0069800684EF20001C4F200011A
:10F34C00884207D0069800684EF20041C4F20001D2
:10F35C00884200D107E04DF25D20C0F6010041F675
:10F36C001F51F7F7D2FC05988068B0F5004F0DD00F
:10F37C000598806850B10598806838B10598806808
:10F38C00022803D0059880680A2800D107E04DF2C6
:10F39C005D20C0F601004FF4E951F7F7B6FC059873
:10F3AC0000690F2800D807E04DF25D20C0F601007F
:10F3BC0041F62151F7F7A9FC06980068059A916867
:10F3CC00126909F011FDDEE0069800680021C4F214
:10F3DC000101884244D006980068B0F1804F3FD0BC
:10F3EC000698006840F20041C4F20001884237D010
:10F3FC000698006840F60001C4F2000188422FD044
:10F40C000698006840F60041C4F20001884227D0FB
:10F41C000698006840F20041C4F2010188421FD0F6
:10F42C000698006841F60001C4F20001884217D02A
:10F43C000698006844F20001C4F2010188420FD022
:10F44C00069800684EF20001C4F20001884207D011
:10F45C00069800684EF20041C4F20001884200D1C7
:10F46C0007E04DF25D20C0F6010041F62D51F7F793
:10F47C004CFC05988068B0F5004F0DD0059880685D
:10F48C0050B10598806838B105988068022803D07F
:10F49C00059880680A2800D107E04DF25D20C0F67F
:10F4AC00010041F62E51F7F730FC059800690F2842
:10F4BC0000D807E04DF25D20C0F6010041F62F5157
:10F4CC00F7F723FC06980068059A91681269FFF714
:10F4DC00DBFB58E0069800680021C4F20101884269
:10F4EC0044D006980068B0F1804F3FD00698006871
:10F4FC0040F20041C4F20001884237D006980068FF
:10F50C0040F60001C4F2000188422FD00698006832
:10F51C0040F60041C4F20001884227D006980068EA
:10F52C0040F20041C4F2010188421FD006980068E5
:10F53C0041F60001C4F20001884217D00698006819
:10F54C0044F20001C4F2010188420FD00698006811
:10F55C004EF20001C4F20001884207D00698006800
:10F56C004EF20041C4F20001884200D107E04DF296
:10F57C005D20C0F6010041F64851F7F7C6FB02E0EA
:10F58C0001208DF813009DF813008DF81F009DF8D5
:06F59C001F0008B080BD55
:10F5A20080B582B00090009818B901208DF807004C
:10F5B20001E100988069002861D00098006841F25A
:10F5C2000001C4F2010188424FD00098006844F261
:10F5D2000041C4F20001884247D00098006844F616
:10F5E2000001C4F2000188423FD00098006844F64E
:10F5F2000041C4F20001884237D00098006845F209
:10F602000001C4F2000188422FD00098006841F244
:10F612000041C4F20101884227D00098006847F6F1
:10F622000001C4F2000188421FD00098006847F62A
:10F632000041C4F20001884217D00098006841F6E8
:10F642000001C4F2010188420FD00098006841F61F
:10F652000041C4F20101884207D00098006840F6D8
:10F662000041C5F60001884200D107E04DF6A22014
:10F67200C0F601004FF49F71F7F74CFB60E0009871
:10F68200006841F20001C4F2010188424FD00098A3
:10F69200006844F20041C4F20001884247D0009859
:10F6A200006844F60001C4F2000188423FD000988D
:10F6B200006844F60041C4F20001884237D0009845
:10F6C200006845F20001C4F2000188422FD0009880
:10F6D200006841F20041C4F20101884227D000983B
:10F6E200006847F60001C4F2000188421FD000986A
:10F6F200006847F60041C4F20001884217D0009822
:10F70200006841F60001C4F2010188420FD000985E
:10F71200006841F60041C4F20101884207D0009816
:10F72200006840F60041C5F60001884200D107E0BA
:10F732004DF6A220C0F6010040F24311F7F7EAFAB3
:10F742000098D0F8880030B90099002081F8840030
:10F752000098F7F768FE00992420C1F88800009805
:10F762000168086820F0010008600098806A10B102
:10F77200009800F024F80098F5F799FD012803D1CC
:10F7820001208DF8070016E000980168486820F40F
:10F792009040486000980168886820F02A008860DC
:10F7A20000980168086840F001000860009809F0BC
:0EF7B20004FD8DF807009DF8070002B080BD31
:10F7C00080B582B001900198806AFF2800D807E0D8
:10F7D0004DF6A220C0F601004FF44E61F7F79BFAF8
:10F7E000019890F82800000700281AD50198806B2E
:10F7F00020B10198806BB0F5004F00D107E04DF6C5
:10F80000A220C0F6010040F6E541F7F784FA01981E
:10F810000068406820F40040019A1168926B104320
:10F820004860019890F82800C007D0B10198C06ADC
:10F8300020B10198C06AB0F5003F00D107E04DF655
:10F84000A220C0F6010040F6EC41F7F764FA0198F7
:10F850000068406820F40030019A1168D26A1043B1
:10F860004860019890F82800800700281AD5019870
:10F87000006B20B10198006BB0F5803F00D107E02C
:10F880004DF6A220C0F6010040F6F341F7F743FA27
:10F8900001980068406820F48030019A1168126B6A
:10F8A00010434860019890F82800400700281AD5B6
:10F8B0000198406B20B10198406BB0F5802F00D1CA
:10F8C00007E04DF6A220C0F6010040F6FA41F7F736
:10F8D00022FA01980068406820F48020019A11689B
:10F8E000526B10434860019890F82800C006002829
:10F8F0001AD50198C06B20B10198C06BB0F5805F3C
:10F9000000D107E04DF6A220C0F6010040F60151FB
:10F91000F7F701FA01980068806820F48050019A96
:10F920001168D26B10438860019890F82800800617
:10F9300000281AD50198006C20B10198006CB0F530
:10F94000005F00D107E04DF6A220C0F6010040F6AE
:10F950000851F7F7E0F901980068806820F400503A
:10F96000019A1168126C10438860019890F8280081
:10F970004006002840F19E800198006841F2000195
:10F98000C4F20101884247D00198006844F2004166
:10F99000C4F2000188423FD00198006844F600019B
:10F9A000C4F20001884237D00198006844F6004153
:10F9B000C4F2000188422FD00198006845F200018E
:10F9C000C4F20001884227D00198006841F200414A
:10F9D000C4F2010188421FD00198006847F6000177
:10F9E000C4F20001884217D00198006847F6004130
:10F9F000C4F2000188420FD00198006841F600016E
:10FA0000C4F20101884207D00198006841F6004124
:10FA1000C4F20101884200D107E04DF6A220C0F6F1
:10FA2000010040F60F51F7F776F90198406C20B1CC
:10FA30000198406CB0F5801F00D107E04DF6A22080
:10FA4000C0F601004FF45161F7F765F901980068BD
:10FA5000406820F48010019A1168526C104348608D
:10FA60000198406CB0F5801F24D10198806C70B172
:10FA70000198806CB0F5001F09D00198806CB0F53A
:10FA8000800F04D00198806CB0F5C00F00D107E062
:10FA90004DF6A220C0F6010040F61551F7F73BF9EC
:10FAA00001980068406820F4C000019A1168926CC7
:10FAB00010434860019890F82800000600281AD5E5
:10FAC0000198C06C20B10198C06CB0F5002F00D136
:10FAD00007E04DF6A220C0F6010040F61D51F7F7F1
:10FAE0001AF901980068406820F40020019A116812
:0AFAF000D26C1043486002B080BDE4
:10FAFA0080B586B0DDF820C0049003918DF80B2004
:10FB0A00019304980068C06903990840401AB0FA42
:10FB1A0080F040099DF80B10884253D108980130B3
:10FB2A0000284ED005F0C7FB0199401A089988426F
:10FB3A0001D8089818B903208DF8170045E00498F1
:10FB4A0000680068400700283BD50398802838D011
:10FB5A000398402835D004980068C069C0F3C000F3
:10FB6A00012813D1049801680820009008620498BB
:10FB7A0009F0C7FB00980499C1F890000499002085
:10FB8A0081F8840001208DF817001EE004980068AF
:10FB9A00C069C0F3C020012813D1049801684FF44A
:10FBAA0000600862049809F0ACFB04992020C1F8AF
:10FBBA0090000499002081F8840003208DF8170032
:10FBCA0003E09EE700208DF817009DF8170006B0A5
:02FBDA0080BDEC
:10FBDC008EB003900398D0F8880021285BD103984D
:10FBEC00B0F86A00ADF80A00BDF80A00002852D03F
:10FBFC000398B0F8560090BB039800680830079043
:10FC0C00079850E8000F0690069820F40000019029
:10FC1C0001990398006808300D910C900C990D9A7D
:10FC2C0041E800200B900B980028E5D10398006860
:10FC3C000590059850E8000F0490049840F040009F
:10FC4C0000900099039800680A91099009990A9A02
:10FC5C0041E80020089008980028E7D11BE00398A1
:10FC6C000068C069000600280FD503980168006D74
:10FC7C00007888620399086D013008650399B1F822
:10FC8C0056000138A1F85600FFE7BDF80A0001380C
:0AFC9C00ADF80A00A8E70EB07047AB
:10FCA6008DB002900298D0F88800212843D102989E
:10FCB600B0F8560080BB029800680690069850E897
:10FCC600000F0590059820F0800001900199029898
:10FCD60000680C910B900B990C9A41E800200A9051
:10FCE6000A980028E7D1029800680490049850E822
:10FCF600000F0390039840F040000090009902988E
:10FD06000068099108900899099A41E8002007902F
:10FD160007980028E7D10EE002980168006D007888
:10FD260088620299086D013008650299B1F856009B
:0AFD36000138A1F856000DB0704727
:10FD400080B59AB005900598806B04900598C069BD
:10FD5000B0F5807F6FD004990020A1F85E00049870
:10FD600000680D900D9850E8000F0C900C9820F44E
:10FD7000807003900399049800681991189018995D
:10FD8000199A41E80020179017980028E7D10498A5
:10FD9000006808300B900B9850E8000F0A900A9802
:10FDA00020F0010002900299049800680830169132
:10FDB00015901599169A41E800201490149800287F
:10FDC000E5D10498006808300990099850E8000FC0
:10FDD0000890089820F0400001900199049800686C
:10FDE0000830139112901299139A41E80020119053
:10FDF00011980028E5D104992020C1F88C000498BE
:10FE0000C06E012817D1049800680790079850E841
:10FE1000000F0690069820F01000009000990498BA
:10FE2000006810910F900F99109A41E800200E90F1
:10FE30000E980028E7D10499002008670498C06E46
:10FE4000012805D10498B0F85C10F7F7F0F802E04B
:0AFE5000049808F045F81AB080BDD0
:10FE5A0080B582B001900198806B009000990120D2
:10FE6A0008670098C06E012806D10098B0F85C10A7
:10FE7A004908F7F7D7F802E0009808F02CF802B022
:02FE8A0080BD39
:10FE8C0080B5BAB0119011980068C06910901198A3
:10FE9C00006800680F901198006880680E901098A8
:10FEAC0040F60F0108400D900D98A8B99DF8400040
:10FEBC008006002810D59DF83C008006002804D44C
:10FECC009DF83B00C006002806D51198406F10B174
:10FEDC001198416F884726E30D98002800F0EF80B9
:10FEEC000E980121C1F20001084207D10F9840F28F
:10FEFC002011C0F20041084200F0E1809DF8400062
:10FF0C00C00770B19DF83D00C00750B11198016851
:10FF1C00012008621199D1F8900040F00100C1F85D
:10FF2C0090009DF84000800700280ED59DF8380001
:10FF3C00C00750B111980168022008621199D1F8DC
:10FF4C00900040F00400C1F890009DF8400040077C
:10FF5C0000280ED59DF83800C00750B111980168E3
:10FF6C00042008621199D1F8900040F00200C1F809
:10FF7C0090009DF840000007002815D59DF83C0026
:10FF8C008006002805D40E980121C1F20001084218
:10FF9C000AD011980168082008621199D1F89000D4
:10FFAC0040F00800C1F890009DF8410000070028BF
:10FFBC0010D59DF83F00400700280BD5119801681B
:10FFCC004FF4006008621199D1F8900040F02000C5
:10FFDC00C1F890001198D0F8900000286ED09DF8D0
:10FFEC004000800600280FD59DF83C0080060028B4
:04FFFC0004D49DF894
:020000040801F1
:100000003B00C006002805D51198406F10B111982B
:10001000416F88471198D0F890000C9011980068B3
:10002000806800F04000402804D09DF8300010F0B7
:10003000280F42D0119809F069F91198006880687A
:100040004006002835D51198006808302190219885
:1000500050E8000F2090209820F040000B900B9962
:10006000119800680830399138903899399A41E8E8
:100070000020379037980028E5D11198D0F88000FB
:1000800098B11198D0F8801040F23750C0F60100B6
:1000900008651198D0F8800005F026FF20B111986E
:1000A000D0F88000016D884702E0119807F018FF32
:1000B00002E0119807F014FF06E0119807F010FF16
:1000C00011990020C1F8900033E21198C06E012808
:1000D00040F0DE819DF84000C006002840F1D88144
:1000E0009DF83C00C006002840F1D28111980168BB
:1000F000102008621198006880684006002840F1CE
:1001000057811198D0F8800000681021C4F20201D4
:10011000884200F090801198D0F880000068282173
:10012000C4F20201884200F086801198D0F8800065
:1001300000684021C4F2020188427CD01198D0F8B6
:10014000800000685821C4F20201884273D01198DF
:10015000D0F8800000687021C4F2020188426AD0A1
:100160001198D0F8800000688821C4F2020188420A
:1001700061D01198D0F880000068A021C4F202017B
:10018000884258D01198D0F880000068B821C4F295
:10019000020188424FD01198D0F88000006840F2E8
:1001A0001041C4F20201884245D01198D0F8800075
:1001B000006840F22841C4F2020188423BD0119805
:1001C000D0F88000006840F24041C4F20201884249
:1001D00031D01198D0F88000006840F25841C4F244
:1001E0000201884227D01198D0F88000006840F2C0
:1001F0007041C4F2020188421DD01198D0F88000ED
:10020000006840F28841C4F20201884213D011987C
:10021000D0F88000006840F2A041C4F20201884298
:1002200009D01198D0F88000006840F2B841C4F2BB
:100230000201884206D11198D0F880000068406819
:10024000019005E01198D0F88000006840680190A6
:100250000198ADF82A00BDF82A00002800F091802E
:10026000BDF82A001199B1F85C10884280F28980AB
:10027000BDF82A001199A1F85E001198D0F880000D
:10028000C069B0F5807F6FD0119800681F901F98EB
:1002900050E8000F1E901E9820F480700990099974
:1002A00011980068369135903599369A41E80020CA
:1002B000349034980028E7D11198006808301D90D8
:1002C0001D9850E8000F1C901C9820F00100089029
:1002D0000899119800680830339132903299339A16
:1002E00041E80020319031980028E5D1119800684C
:1002F00008301B901B9850E8000F1A901A9820F0B5
:1003000040000790079911980068083030912F90AD
:100310002F99309A41E800202E902E980028E5D1A0
:1003200011992020C1F88C0011990020C8661198FD
:1003300000681990199850E8000F1890189820F04C
:10034000100006900699119800682D912C902C9918
:100350002D9A41E800202B902B980028E7D1119886
:10036000D0F88000F8F7C0FB1199022008671198B7
:10037000B0F85C10B0F85E20891A89B2F6F757FE23
:1003800015E0BDF82A001199B1F85C1088420ED131
:100390001198D0F88000C069B0F5807F07D111991D
:1003A000022008671198B0F85C10F6F740FEC0E034
:1003B0001199B1F85C00B1F85E10401AADF8160062
:1003C0001198B0F85E00002861D0BDF81600002832
:1003D0005DD0119800681790179850E8000F16909C
:1003E000169820F4907004900499119800682A914E
:1003F000299029992A9A41E80020289028980028D5
:10040000E7D11198006808301590159850E8000F52
:10041000149014984FF6FE71CEF6FF7108400390C9
:100420000399119800680830279126902699279AF9
:1004300041E80020259025980028E2D1119920203C
:10044000C1F88C0011990020C8661199486711986D
:1004500000681390139850E8000F1290129820F043
:10046000100002900299119800682491239023991A
:10047000249A41E80020229022980028E7D111997F
:10048000022008671198BDF81610F6F7D0FD50E06D
:100490009DF84200C00600280DD59DF83A004006A0
:1004A000002808D5119801684FF48010086211984F
:1004B00007F016FD3DE09DF840000006002810D52D
:1004C0009DF83C000006002804D49DF83A00000680
:1004D000002806D51198806F10B11198816F884758
:1004E00027E09DF840004006002808D59DF83C0014
:1004F0004006002803D5119800F02CF819E09DF86B
:1005000042000006002808D59DF83F00400600285C
:1005100003D5119807F0E4FC0BE09DF84300C007F9
:1005200038B19DF83F000006002802D5119807F069
:06053000D7FC3AB080BDCB
:1005360080B582B001900198806B009000990020F0
:0E054600A1F85E00009807F0C8FC02B080BD6E
:1005540080B588B00290029800680490049850E82E
:10056400000F0390039820F0400001900199029835
:100574000068079106900699079A41E800200590C3
:1005840005980028E7D102992020C1F88800029933
:0E05940000208867029807F0A1FC08B080BD27
:1005A20082B001900198406E38B901990120A1F8FA
:1005B2006A000199A1F8680031E010208DF803006B
:1005C2008DF80200019800688068C0F342608DF8DF
:1005D2000100019800688068400F8DF800009DF8C6
:1005E20002009DF800204DF60A33C0F60103995C23
:1005F20048434DF61231C0F601018A5CB0FBF2F0BD
:10060200019AA2F86A009DF803009DF801209B5C04
:100612005843895CB0FBF1F00199A1F8680002B07F
:0206220070471F
:1006240080B584B002900298006841F20001C4F2DF
:10063400010188424FD00298006844F20041C4F29C
:100644000001884247D00298006844F60001C4F2D1
:10065400000188423FD00298006844F60041C4F289
:100664000001884237D00298006845F20001C4F2C4
:10067400000188422FD00298006841F20041C4F280
:100684000101884227D00298006847F60001C4F2AD
:10069400000188421FD00298006847F60041C4F266
:1006A4000001884217D00298006841F60001C4F2A4
:1006B400010188420FD00298006841F60041C4F25B
:1006C4000101884207D00298006840F60041C5F64F
:1006D4000001884200D107E04DF2C420C0F60100B9
:1006E40040F23621F6F715FB029890F884000128B1
:1006F40003D102208DF80F0027E00299012081F830
:10070400840002992420C1F88800029800680068D7
:10071400019002980168086820F0010008600198BF
:1007240020F0005001900299002048660198029937
:100734000968086002992020C1F888000299002005
:1007440081F8840000208DF80F009DF80F0004B09C
:0207540080BD66
:1007560080B584B0029001910298006841F20001D0
:10076600C4F2010188424FD00298006844F2004169
:10077600C4F20001884247D00298006844F600019E
:10078600C4F2000188423FD00298006844F6004156
:10079600C4F20001884237D00298006845F2000191
:1007A600C4F2000188422FD00298006841F200414D
:1007B600C4F20101884227D00298006847F600017A
:1007C600C4F2000188421FD00298006847F6004133
:1007D600C4F20001884217D00298006841F6000171
:1007E600C4F2010188420FD00298006841F6004128
:1007F600C4F20101884207D00298006840F6004121
:10080600C5F60001884200D107E04DF2C420C0F6CB
:1008160001004FF41971F6F77BFA019898B1019827
:10082600B0F1005F0FD00198B0F1804F0BD0019866
:10083600B0F1C04F07D00198B0F1004F03D0019836
:10084600B0F1204F00D107E04DF2C420C0F6010000
:1008560040F26521F6F75CFA029890F884000128C8
:1008660003D102208DF80F002DE00299012081F8B6
:10087600840002992420C1F8880002980068006864
:10088600009002980168086820F00100086002984C
:100896000068806820F06040019908430299096861
:1008A60088600298FFF77AFE009802990968086046
:1008B60002992020C1F888000299002081F884005E
:0E08C60000208DF80F009DF80F0004B080BDDB
:1008D40080B584B0029001910298006841F2000151
:1008E400C4F2010188424FD00298006844F20041EA
:1008F400C4F20001884247D00298006844F600011F
:10090400C4F2000188423FD00298006844F60041D6
:10091400C4F20001884237D00298006845F2000111
:10092400C4F2000188422FD00298006841F20041CD
:10093400C4F20101884227D00298006847F60001FA
:10094400C4F2000188421FD00298006847F60041B3
:10095400C4F20001884217D00298006841F60001F1
:10096400C4F2010188420FD00298006841F60041A8
:10097400C4F20101884207D00298006840F60041A1
:10098400C5F60001884200D107E04DF2C420C0F64C
:10099400010040F29521F6F7BCF9019898B101984D
:1009A400B0F1007F0FD00198B0F1806F0BD00198A7
:1009B400B0F1C06F07D00198B0F1006F03D0019877
:1009C400B0F1206F00D107E04DF2C420C0F6010061
:1009D40040F29621F6F79DF9029890F884000128D8
:1009E40003D102208DF80F002DE00299012081F837
:1009F400840002992420C1F88800029800680068E5
:100A0400009002980168086820F0010008600298CC
:100A14000068806820F060600199084302990968C1
:100A240088600298FFF7BBFD009802990968086086
:100A340002992020C1F888000299002081F88400DE
:0E0A440000208DF80F009DF80F0004B080BD5B
:100A520080B58AB003900291ADF806200398D0F8D1
:100A62008C00202842D1029810B1BDF8060018B9B6
:100A720001208DF813003CE003990120C866039918
:100A82000020086703980299BDF8062008F063FE6B
:100A92008DF805009DF8050018BB0398C06E01286B
:100AA2001CD1039801681020086203980068069020
:100AB200069850E8000F0590059840F0100000904D
:100AC200009903980068099108900899099A41E8E9
:100AD2000020079007980028E7D102E001208DF856
:100AE20005009DF805008DF8130002E002208DF844
:0A0AF20013009DF813000AB080BD48
:100AFC0010B588B0DDF82CE0DDF828C0CDF81CE08E
:100B0C00CDF818C005930492039102900020019037
:100B1C00029847F20001C5F20021884206D00298E3
:100B2C0042F20041C4F60201884200D106E04DF6C3
:100B3C001A30C0F60100CE21F6F7E7F8039818B189
:100B4C000398B0F5803F00D106E04DF61A30C0F6A0
:100B5C000100CF21F6F7D9F8049818B10498B0F534
:100B6C00805F00D106E04DF61A30C0F60100D021AE
:100B7C00F6F7CBF8059838B10598B0F5804F03D04F
:100B8C000598B0F5004F00D106E04DF61A30C0F6CE
:100B9C000100D121F6F7B9F8069818B10698B0F50E
:100BAC00003F00D106E04DF61A30C0F60100D2210C
:100BBC00F6F7ABF80798800A00B906E04DF61A3044
:100BCC00C0F60100D321F6F7A0F80398049B059A10
:100BDC0006991843104308430799014301980843A9
:100BEC0001900298406842F60041CFF6C07108406F
:0E0BFC000199084302994860002008B010BD1E
:0E0C0A0081B000900098D0F8800001B07047D3
:100C180082B001900091009800680199C1F88000A5
:060C2800002002B070473D
:100C2E0080B584B003900291002001900298406834
:100C3E003F2800D807E04DF61A30C0F6010040F20A
:100C4E006511F6F761F80298806848B102988068DD
:100C5E00B0F5807F04D002988068B0F5407F00D157
:100C6E0007E04DF61A30C0F601004FF4B371F6F7F7
:100C7E004BF80298C06848B10298C068B0F5806F12
:100C8E0004D00298C068B0F5006F00D107E04DF6B1
:100C9E001A30C0F6010040F26711F6F735F80298E7
:100CAE00006920B102980069B0F5805F00D107E0BD
:100CBE004DF61A30C0F601004FF4B471F6F724F871
:100CCE000298006803998860029948688B68CA6820
:100CDE000969184310430143019808430190039892
:100CEE00C0684EF2C001CFF6FE710840019908436C
:0A0CFE000399C860002004B080BD17
:0E0D080081B0009000980069C0B201B0704741
:100D160080B584B003900291029840B102980428ED
:100D260005D00298082802D002980C2800D107E0C6
:100D36004DF61A30C0F601004FF4CA71F5F7E8FF18
:100D4600039802990844143001900198006804B091
:020D560080BD5E
:100D580080B584B003900291002001900298406809
:100D6800400E00B907E04DF61A30C0F6010040F217
:100D7800A911F5F7CCFF02988068B8B3029880688B
:100D8800102833D00298806820282FD002988068D5
:100D980030282BD002988068402827D00298806895
:100DA800502823D00298806860281FD00298806855
:100DB80070281BD002988068802817D00298806815
:100DC800902813D002988068A0280FD002988068D5
:100DD800B0280BD002988068C02807D00298806895
:100DE800D02803D002988068E02800D107E04DF6AB
:100DF8001A30C0F601004FF4D571F5F788FF029854
:100E0800C06818B10298C068022800D107E04DF602
:100E18001A30C0F6010040F2AB11F5F778FF0298DE
:100E2800006938B102980069042803D00298006963
:100E3800082800D107E04DF61A30C0F601004FF43B
:100E4800D671F5F764FF0298406918B102984069B5
:100E5800012800D107E04DF61A30C0F6010040F233
:100E6800AD11F5F754FF029800680399486202989B
:100E780040680399886202998868CB680A69496959
:100E88001843104301430198084301900398C06A2E
:100E980020F0FF00019908430399C862002004B0BC
:020EA80080BD0B
:100EAA0080B58AB0099008910898039010200190A3
:100EBA0004904FF480700590002006904FF4805003
:100ECA000790099803A9FFF7ADFE0199099841F225
:0E0EDA00883200F004F8029002980AB080BD41
:100EE80080B588B006908DF817100492049848F6DB
:100EF8005821C2F200410968C90844F6D352C1F228
:100F08006202A1FB02218909484301900198411E10
:100F1800019118B94FF000400790E5E00698406B42
:100F28000290029901204522C0F22002114200904D
:100F380004D09DF80900C0F3401000900098C00745
:100F48000028E3D10698406B4007002804D506998D
:100F5800042088630790C7E00698406BC00720B15B
:100F68000699012088630790BEE00699C520C0F263
:100F7800200088630698FFF7C3FE9DF81710884283
:100F880002D001200790AFE006980021FFF7BFFECE
:100F9800039003984EF20801CFF6FF51084202D1A0
:100FA80000200790A0E09DF80F000006002803D558
:100FB8004FF00070079097E09DF80F00400600285A
:100FC80002D5402007908FE09DF80F00800600288A
:100FD80002D58020079087E09DF80F00C006002802
:100FE80003D54FF4807007907EE09DF80F0000074E
:100FF800002803D54FF40070079075E09DF80F00A6
:101008004007002803D54FF4806007906CE09DF8F6
:101018000F00C00718B14FF40060079064E09DF816
:101028000E000006002803D54FF4805007905BE0BF
:101038009DF80E004006002803D54FF40050079095
:1010480052E09DF80E008006002803D54FF480403A
:10105800079049E09DF80E00C006002803D54FF41C
:101068000040079040E09DF80E004007002803D597
:101078004FF40030079037E09DF80E0080070028F5
:1010880003D54FF4802007902EE09DF80E00C0078E
:1010980018B14FF40020079026E09DF80D000006D7
:1010A800002803D54FF4801007901DE09DF80D002F
:1010B8004006002803D54FF40010079014E09DF86F
:1010C8000D008006002803D54FF4800007900BE040
:1010D8009DF80C000007002803D54FF40000079086
:0E10E80002E04FF480300790079808B080BDFA
:1010F60080B58AB009900891089803901120019054
:1011060004904FF480700590002006904FF48050B4
:101116000790099803A9FFF787FD0199099841F2FD
:0E1126008832FFF7DEFE029002980AB080BD0C
:1011340080B58AB009900891089803901220019014
:1011440004904FF480700590002006904FF4805076
:101154000790099803A9FFF768FD0199099841F2DE
:0E1164008832FFF7BFFE029002980AB080BDED
:1011720080B58AB0099008910898039018200190D0
:1011820004904FF480700590002006904FF4805038
:101192000790099803A9FFF749FD0199099841F2BF
:0E11A2008832FFF7A0FE029002980AB080BDCE
:1011B00080B58AB009900891089803901920019091
:1011C00004904FF480700590002006904FF48050FA
:1011D0000790099803A9FFF72AFD0199099841F2A0
:0E11E0008832FFF781FE029002980AB080BDAF
:1011EE0080B58AB009900891089803900720019065
:1011FE0004904FF480700590002006904FF48050BC
:10120E000790099803A9FFF70BFD0199099841F280
:0E121E008832FFF762FE029002980AB080BD8F
:10122C0080B588B007904FF4D570029008200390D9
:10123C004FF480700490002005904FF4805006907D
:10124C00079802A9FFF7EDFC079808F0B3FB019093
:06125C00019808B080BDFE
:1012620080B58AB0099008910898039037200190C0
:1012720004904FF480700590002006904FF4805047
:101282000790099803A9FFF7D1FC0199099841F247
:0E1292008832FFF728FE029002980AB080BD55
:1012A00080B588B007900691069801902920029099
:1012B0004FF480700390002004904FF4805005900C
:1012C000079801A9FFF7B3FC079808F0C7FB009047
:0612D000009808B080BD8B
:1012D60080B58AB00990089108980390062001907D
:1012E60004904FF480700590002006904FF48050D3
:1012F6000790099803A9FFF797FC0199099841F20D
:0E1306008832FFF7EEFD029002980AB080BD1B
:1013140080B588B00790002002903321009103919A
:101324004FF48071049105904FF480500690079813
:1013340002A9FFF77AFC0099079841F28832FFF777
:0A134400D1FD0190019808B080BDB2
:10134E0080B588B0079000200290022103914FF4DF
:10135E004071049105904FF480500690079802A9B1
:10136E00FFF75EFC079800F004F80190019808B0B2
:02137E0080BD30
:1013800085B0039048F65820C2F200400068C008BB
:1013900044F6D351C1F26201A0FB0110800941F271
:1013A0008831484301900198411E019118B94FF0CE
:1013B000004004902CE00398406B029001209DF8BF
:1013C000081011F0450F009004D09DF80900C0F3FB
:1013D000401000900098C0070028E4D10398406BAB
:1013E0004007002804D503990420886304900FE087
:1013F0000398406BC00720B10399012088630490D3
:1014000006E00399C520C0F2200088630020049004
:06141000049805B07047CE
:1014160080B588B007900691069801900920029041
:101426004FF440700390002004904FF480500590D4
:10143600079801A9FFF7F8FB0798FFF79EFF0090B2
:06144600009808B080BD13
:10144C0080B58AB009900891002003900321019186
:10145C0004914FF48071059106904FF480500790E1
:10146C00099803A9FFF7DDFB01990998089A00F088
:0A147C0004F8029002980AB080BD47
:1014860080B588B006908DF81710049248F658205B
:10149600C2F200400068C00844F6D351C1F26201AE
:1014A600A0FB0110800941F2883148430190019860
:1014B600411E019118B94FF0004007905AE0069876
:1014C600406B029001209DF8081011F0450F009026
:1014D60004D09DF80900C0F3401000900098C007A2
:1014E6000028E4D10698406B4007002804D50699E9
:1014F6000420886307903DE00698406BC00720B142
:10150600069901208863079034E00698FFF7F9FBF7
:101516009DF81710884202D0012007902AE006990C
:10152600C520C0F22000886306980021FFF7F0FB73
:1015360003909DF80D0010F0E00F06D1BDF80E00E7
:10154600049908800020079014E09DF80D004006DD
:10155600002803D54FF4005007900BE09DF80D00CE
:101566000006002803D54FF48050079002E04FF4A0
:0A15760080300790079808B080BD90
:1015800080B58AB009900891089803900D200190C9
:1015900004904FF480700590002006904FF4805026
:1015A0000790099803A9FFF742FB0199099841F2B6
:0E15B0008832FFF799FC029002980AB080BDC5
:1015BE0080B588B00790002002900D210091039114
:1015CE004FF48071049105904FF480500690079867
:1015DE0002A9FFF725FB0099079841F28832FFF721
:0A15EE007CFC0190019808B080BD5C
:1015F80080B584B0039000200290694634200860CA
:1016080048F26010C2F200404DF22F31C0F60101DD
:1016180042F6B802C2F200424FF4005302F0A1FFB2
:1016280000B10BE048F26010C2F20040019001984E
:10163800F3F71BFD0290029800B1FEE769463420DB
:10164800086048F29410C2F200404DF24231C0F6F0
:10165800010144F6B802C2F200424FF4005302F00E
:1016680080FF00B10BE048F29410C2F200400190F4
:10167800019800F006F80290029800B1FEE704B065
:0216880080BD23
:10168A0080B58CB00A90002309930A9808900898AC
:10169A0007A94FF4806202F0F0FE0990099810B190
:1016AA0002200B9026E007986946B4228A6101223B
:1016BA004A6100230B610A22CA608A604FF4806281
:1016CA004A60086047F67C10C2F200404DF6770186
:1016DA00C0F6010149F6E122C0F601020BF03DF91C
:1016EA000990099810B10E200B9003E000F08BFED0
:0A16FA0009980B900B980CB080BD0E
:1017040080B582B001900020009047F65C60C2F280
:10171400004006F0CFFA08B101200090009802B012
:0217240080BD86
:1017260080B586B005900491039202930020019043
:101736000499039A029B47F65C60C2F20040FAF7EE
:0E1746004CFD08B101200190019806B080BD55
:1017540080B586B005900491039202930020019015
:101764000499039A029B47F65C60C2F2004006F0BB
:0E177400D9FA08B101200190019806B080BD9D
:1017820080B582B0019048F21820C2F200400BF0FE
:06179200CEF802B080BD9C
:1017980080B582B0019048F23820C2F200400BF0C8
:0617A800C3F802B080BD91
:1017AE0080B590B0069005910492039300200290AC
:1017BE000398002869D00698D0F890000090002079
:1017CE00029002980499884255D2059A501C0590B1
:1017DE0040F20001C2F2004100200123FFF79CFFFE
:1017EE000190019810B19020079093E048F23820B4
:1017FE00C2F200404FF47A7103F0DCF810B1902081
:10180E00079087E040F20000C2F200400F904FF4C4
:10181E0000700E900E9801281CDB0E980F9901F0A7
:10182E001F0108440D900F980C90BFF34F8F0C982A
:10183E004EF65C71CEF2000108600C9820300C90D0
:10184E000D9820380D900D980028F0DCBFF34F8FC7
:10185E00BFF36F8F009940F20000C2F200404FF4C8
:10186E00007209F0D4F8009800F50070009002980C
:10187E0001300290A5E702980499884202D1002017
:10188E00019001E02120019042E00698D0F89010DE
:10189E00059A049B0020FFF73FFF0190019810B1BD
:1018AE009020079036E048F23820C2F200404FF404
:1018BE007A7103F07FF810B1902007902AE0069815
:1018CE00D0F89010049840020B910A900A980128C3
:1018DE001CDB0A980B9901F01F01084409900B9824
:1018EE000890BFF34F8F08984EF65C71CEF2000150
:1018FE0008600898203008900998203809900998B7
:10190E000028F0DCBFF34F8FBFF36F8F00200190E4
:0A191E0001980790079810B080BDF3
:1019280080B592B008900791069205930020049024
:101938000598002867D00898D0F8900002900020F9
:10194800049004980699884253D2029840F2000104
:10195800C2F2004100914FF40072019209F05AF866
:1019680000990198029A02F5007202921191109062
:10197800109801281CDB1098119901F01F010844E8
:101988000F9011980E90BFF34F8F0E984EF6687116
:10199800CEF2000108600E9820300E900F98203883
:1019A8000F900F980028F0DCBFF34F8FBFF36F8FB5
:1019B800079A501C079040F20001C2F20041002033
:1019C8000123FFF7C3FE0390039810B190200990FC
:1019D8005EE048F21820C2F200404FF47A7102F03B
:1019E800ECFF10B19020099052E004980130049067
:1019F800A7E704980699884202D10020039001E0E5
:101A08002120039042E00898D0F8901006984002F0
:101A18000D910C900C9801281CDB0C980D9901F085
:101A28001F0108440B900D980A90BFF34F8F0A9836
:101A38004EF66871CEF2000108600A9820300A90CC
:101A48000B9820380B900B980028F0DCBFF34F8FD1
:101A5800BFF36F8F0898D0F89010079A069B002064
:101A6800FFF774FE0390039810B1902009900FE0DF
:101A780048F21820C2F200404FF47A7102F09DFF3C
:101A880010B19020099003E000200390039809907A
:061A9800099812B080BDA8
:101A9E0080B59EB0DDF884C0DDF880C01990189135
:101AAE001792169348F23C30C2F20040006848F29A
:101ABE003831C2F200410968084348F23431C2F2AB
